:020000040040BA
:04C00000000919001A
:04C004006D85410005
:10C008000000000000000000000000000000000028
:10C018000000000000000000000000000000000018
:10C028000000000000000000000000000000000008
:10C0380000000000000000000000000000000000F8
:10C0480000000000000000000000000000000000E8
:10C0580000000000000000000000000000000000D8
:10C0680000000000000000000000000000000000C8
:10C0780000000000000000000000000000000000B8
:10C0880000000000000000000000000000000000A8
:10C098000000000000000000000000000000000098
:10C0A8000000000000000000000000000000000088
:10C0B8000000000000000000000000000000000078
:10C0C8000000000000000000000000000000000068
:10C0D8000000000000000000000000000000000058
:10C0E8000000000000000000000000000000000048
:10C0F8000000000000000000F87F00206D8541006E
:10C108009D834100AD834100BD834100CD83410043
:10C11800DD83410000000000000000000000000076
:10C1280000000000ED834100FD8341000000000095
:10C138000D8441001D8441002D8441003D8441004F
:10C148004D8441005D8441006D8441007D8441003F
:10C158008D844100000000009D844100AD844100B1
:10C1680000000000F16D4100FD6D4100000000007D
:10C178007D294100C5564100000000000000000074
:10C18800BD844100CD844100DD844100ED8441003F
:10C19800FD844100BD9941000D8541001D85410088
:10C1A800000000000000000000000000D92C410041
:10C1B8002D8541003D8541004D8541005D8541004B
:10C1C80069744100F0B50026A3B0434C22274348C8
:10C1D80007FB06412022F5B20FF056FE002868D171
:10C1E8003F4B404A1D7007FB054303F1200153F8FC
:10C1F800040B8B4242F8040BF9D11B8801261380EB
:10C20800384D394B95F820201B201A700DF048F84E
:10C21800002847D0354836490DF0ACF933482F4946
:10C228000DF0A8F9314833490DF0A4F92F483249E7
:10C238000DF0A0F9284C04F1CC0794F8202094F8CC
:10C24800213000922D49224602A80EF0B7FC223474
:10C25800264802A90DF08EF9BC42EED123482849A0
:10C268000DF088F916B92148264907E01C4B2649E4
:10C2780002A81A780EF0A2FC1C4802A90DF07AF95F
:10C288001A4822490DF076F995F8202095F82130C2
:10C298001F49009202A8134A0EF090FC134802A905
:10C2A8000DF068F904F04AFF1A4B00221A6023B017
:10C2B800F0BD052E01D0013687E72346094A04F16F
:10C2C800200153F8040B8B4242F8040BF9D11B8868
:10C2D8000026138094E700BF80C2410016FC41008D
:10C2E800BA34002098340020B851002000C2410020
:10C2F80008C2410043D841001FC2410032C2410078
:10C308004FC2410068C241004BC241006EC24100A9
:10C3180033C24100BC34002070B505461C488CB0BF
:10C32800407D08AC8DF80300086889880590ADF851
:10C33800181011689288CDF81A10ADF81E2003F174
:10C348001006224618685968083303C2B3421446D7
:10C35800F7D101AA0F4B05A80DF1030101F00CF864
:10C368000D4A03AE1368013313602A4601AB1C461D
:10C3780003CCB44210605160234602F10802F6D1A2
:10C38800206810602846A38893800CB070BD00BF59
:10C3980038720020B9340020BC3400202DE9F04B5D
:10C3A8008046894696B03D4C04AD93461E460FCC58
:10C3B8000FC50FCC0FC554F8043B239F2B600DAD60
:10C3C8000FCC0FC50FCC0FC52368354C2B60354DEE
:10C3D800354B4846019300954FF4FA730294414651
:10C3E800642200F069F828683B68834207D17A68BC
:10C3F8006B689A4203D1BA68AB689A4212D02B4B49
:10C4080021681A689142D4BF19601A6061685A6835
:10C4180038609142D4BF59605A60224B5A687A609A
:10C428009B68BB60BBF90030C3F10A02142A204A9A
:10C438008BBF002311681360013198BF1160126827
:10C44800802A11BF40F2FD73194A0021116008BF0C
:10C45800DB0100223BF912102498C91A40F8221077
:10C468000132082AF6D1209B48460093229B0DA949
:10C478000193219B0B4A0293092300F00FF91F9B9C
:10C48800009601931E9B4046029304A9094A09237A
:10C4980000F004F916B0BDE8F08B00BF4CC34100B2
:10C4A800CC340020E0340020D43400204025002083
:10C4B800DC340020C03400202DE9F04F85B08DE831
:10C4C8000F006E4B0E9E19680F981D4629B1002269
:10C4D80001312960144613461AE00B46684C694A34
:10C4E800694F42F8234042F2107247F82320674F01
:10C4F80047F82340664C44F82320664C002244F851
:10C508002320654C44F823200133032BE6D1DEE7D2
:10C518005C4F009D35F913C057F823506545B8BFE7
:10C52800654647F82350584FAB4657F823506545A2
:10C53800A8BF654647F82350A846544F019DC8EB4D
:10C548000B0835F913E057F8235044447545B8BF34
:10C55800754647F82350A9464D4D55F82370774541
:10C56800A8BF7746BA4645F823704A4D55F8237058
:10C578006744DFF824C145F823705CF823707744DA
:10C588004CF823700133CAEB0907032B3A44BFD197
:10C5980003680BB93223036043680BB9C8234360AF
:10C5A800109B1C605A60D0F800E00EEB4E0C6445FE
:10C5B8005EDC4768BA425BDC2B68DFF8D88093FB07
:10C5C800F1F383EAE379A9EBE379B9F5167F4FDC58
:10C5D800D8F8043093FBF1F383EAE37AAAEBE37A21
:10C5E800BAF5167F44DCD8F8088098FBF1F888EA99
:10C5F800E87BABEBE87BBBF5167F39DC029B994205
:10C608000CDD74450ADABA4208DAB9F5167F05D0A6
:10C61800BAF5167F02D0BBF5167F0FD1039B99425E
:10C6280029DD644527DABA4225DAB9F5167F22D022
:10C63800BAF5167F1FD0BBF5167F1CD02B6804EB0C
:10C64800440493FBF1F333606B6802EB420293FB03
:10C65800F1F37360AB6893FBF1F1B1600368A34237
:10C66800D4BF0360046043689342D4BF4360426010
:10C67800024B00221A6005B0BDE8F08F1C3500207F
:10C68800F0D8FFFF10350020F8340020EC340020EB
:10C69800203500202C350020043500202DE9F04FEE
:10C6A80089B00DF1080B82468846914600210C227C
:10C6B800584605AE1F46149D0FF02EFA304600214D
:10C6C8000C220FF029FA0023009301933AF9132062
:10C6D80059F82310521AD2034BF823200133032BA5
:10C6E800F4D15946404632461F2304F0A7FD009C6A
:10C6F800002156F82120A7F10608129842FA08F3FB
:10C7080040F8213082FB02230131920F42EA830272
:10C7180003291444EDD108A840F8204D01A904F0DC
:10C72800C8FD019C139B24FA08F21A601CB92C60FE
:10C738006C60AC6010E0002756F827302246D91705
:10C74800C907D80741EA530100230EF0D1FD45F887
:10C7580027000137032FEFD109B0BDE8F08F002380
:10C7680010B51360B9B14FF0804383424FEA5303C9
:10C7780001D94000F9E74008116853B15C18A0429C
:10C7880021BF401AC01A01EB4301116040005B0849
:10C79800F2E74900116010BD0346B0FBF1F001FB60
:10C7A800103330B5002494420BD0002B4FEA4000E0
:10C7B8004FEA430301DB8B4201D301305B1A01349A
:10C7C800F1E730BDB0FBF1F370B50024254601FB5D
:10C7D8001300954210D0064640000CB9DC0F00E06B
:10C7E8000124002EE4B24FEA430301DB884201D35F
:10C7F8000133401A0135ECE724B95A1C04D018B1AA
:10C80800013301E04FF0FF33184670BD70B5B0FB3F
:10C81800F1F401FB140300200546954210D01E4692
:10C828005B0008B9E00F00E00120002EC0B24FEA1B
:10C83800440401DB8B4201D301345B1A0135ECE778
:10C8480000280CBF20464FF0FF3070BD0B4610B5D6
:10C85800044681EAE171A1EBE371DB0F80EAE07045
:10C86800B3EBD47FA0EBE47005D0FFF7ABFF002853
:10C8780008DB404210BDFFF7C9FF0028B8BF6FF0C2
:10C88800004010BD4FF0004010BDF0B580EAE073E5
:10C8980081EAE176A6EBE176A3EBE073C50FB3FB83
:10C8A800F6F00024274606FB1033C90F974211D033
:10C8B8009E465B000CB9C40F00E00124BEF1000FD6
:10C8C800E4B24FEA400001DBB34201D301309B1BC5
:10C8D8000137EBE784B9421C0ED0002B05DB5B0067
:10C8E800B34202D802D1C30700D501308D4207D028
:10C8F80000280ADB4042F0BD8D4206D14FF0FF30E0
:10C908000028B8BF6FF00040F0BD4FF00040F0BD08
:10C9180038B505460C4680EAE07081EAE171A1EB82
:10C92800E471A0EBE570E40FFFF770FFB4EBD57F7F
:10C9380003D0002806DB404238BD0028B8BF6FF09E
:10C94800004038BD4FF0004038BD10B5044680EABD
:10C95800E070A0EBE470FFF759FF002C03DA002821
:10C9680006DB404210BD0028B8BF6FF0004010BD84
:10C978004FF0004010BD38B505460C4680EAE0701F
:10C9880081EAE171A1EBE471A0EBE570FFF704FF28
:10C99800E40FB4EBD57F18BF404238BDF0B5050CA5
:10C9A8000F0C80B289B201FB05F407FB00FE41437E
:10C9B80001EB0E4000EB0446240C04EB1E4407FB7D
:10C9C8000544884234BF01210021864238BF013125
:10C9D800214411601E60F0BD07B56A4601ABFFF740
:10C9E800DDFF0098000903B05DF804FB2DE9F04174
:10C9F80080EAE07581EAE176A5EBE075A6EBE176E1
:10CA0800ACB24FEA154E4FEA164CB5B205FB0EF61E
:10CA18000CFB04F8654305EB084404EB0647360CA9
:10CA280006EB18460CFB0E66AC4234BF0125002508
:10CA3800A74238BF0135741978B171B10028D4BF45
:10CA4800002001200029D4BF00210121884204D000
:10CA58007F420FB1E44300E0644214601F60BDE808
:10CA6800F08107B56A4601ABFFF7C0FF019B009A4A
:10CA7800002B05DA23F0004323B902F0010302E09A
:10CA8800002300E00123002A03EB020001DA13B1BE
:10CA980008B9002301E04FF0FF330093009B002BFF
:10CAA80003DB03D04FF0FF3000E0002003B05DF857
:10CAB80004FB07B56A4601ABFFF798FF019801032D
:10CAC80002D5C0F3120333B9C0F31403A3F5C0129F
:10CAD8005342534100E0012300990A0342EA1050EF
:10CAE800184413B1B0FA80F35B0903EB2153002B10
:10CAF80003DB03D04FF0FF3000E0002003B05DF807
:10CB080004FB07B56A4601ABFFF770FF009B01986D
:10CB18005A16002A04DB05D1400E40EAC31003E090
:10CB2800002001E04FF0FF3003B05DF804FB07B5CB
:10CB38006A4601ABFFF75AFF009B01985A17002A73
:10CB480004DB05D1400F40EAC30003E0002001E008
:10CB58004FF0FF3003B05DF804FB07B501AB6A4640
:10CB6800FFF744FF0098019B000140EA137003B0EF
:10CB78005DF804FB07B56A4601ABFFF70FFF0098A5
:10CB8800C00803B05DF804FB07B56A4601ABFFF7C0
:10CB98002DFF0198010102D520F0784333B920F028
:10CBA800604303F168425342534100E00123009976
:10CBB8000A0142EA1070184413B1B0FA80F35B0915
:10CBC80003EB2173002B03DB03D04FF0FF3000E0B1
:10CBD800002003B05DF804FB07B501AB6A46FFF718
:10CBE800DDFE0098019B000640EA132003B05DF8C3
:10CBF80004FB000038B5030A01330B4D03F1004470
:10CC0800013CDBB235F8131035F81430C0B29B0381
:10CC1800C3EB8131FFF7E0FF35F81430C0F38F30F4
:10CC2800184480B238BD00BF9C5B002038B5030AA9
:10CC380001330B4D03F10044013CDBB235F813100E
:10CC480035F81430C0B29B03C3EB8131FFF7C4FF42
:10CC580035F81430C0F38F30184480B238BD00BFA7
:10CC68009C59002007B501AB6A46FFF797FE00986C
:10CC7800019B400040EAD37003B05DF804FB884292
:10CC880002D8002018607047411A080D904235BF3D
:10CC9800C1F3130102F1FF30C9024FF000422CBF6B
:10CCA8001A6019607047013070B58500043D52F86C
:10CCB800203054591646A342084605DB191BFFF7D6
:10CCC800D1FF7459204470BDE11AFFF7CBFF201A39
:10CCD80070BD884202D8002018607047411A880E3B
:10CCE800904235BF21F07C4102F1FF3049014FF0FD
:10CCF80000422CBF1A60196070472DE9F04F89B0C7
:10CD0800069201F18042013A50F822208B46D20F58
:10CD18000092069903F18042013A51F822200590C9
:10CD2800D20F0192002213998A424FF0000104DACF
:10CD3800129840F822100132F5E70125594570DABA
:10CD4800059A009852F8212030B1AA1A013AAA424D
:10CD58002EBF002501250022100C92B20392139ACF
:10CD68000290521A9A42A8BF1A460492129A0127B0
:10CD780002EB810E002216460498864245DA069C8C
:10CD8800DEF800A054F82690019C4CB1C9EB0709C5
:10CD980009F1FF39B9452EBF002701274FF00009D7
:10CDA80002984FEA19441FFA89F900FB09F8039819
:10CDB8001AEB020200FB04FC2CBF012000200790A4
:10CDC8000398013600FB09FA4FEA08401AEB020AF9
:10CDD8002CBF012200224FEA0C4910EB0A002CBF9D
:10CDE8004FF0010A4FF0000A10EB09004EF8040B4F
:10CDF80002988146079809FB040404EB184404EBE5
:10CE08001C4414444AEB0402B6E70028ACBF0818D7
:10CE1800081C139C0131A042BCBF129C44F820207E
:10CE28008CE7009B019A934211D0129B0120043B8E
:10CE38000021139A91420ADA53F8042F0131821A19
:10CE4800013A82421A602CBF00200120F1E709B0A4
:10CE5800BDE8F08FF0B5002426469C4213DA50F85E
:10CE6800247051F824503D44354442F8245026B1EA
:10CE7800BD428CBF0026012603E0BD422CBF002620
:10CE880001260134E9E7F0BD10B502F18044013C08
:10CE980050F8243051F8244003F0004304F00044D3
:10CEA800A3420ED1002A0ADD013A50F8224051F877
:10CEB80022309C42F6D00AD84FF0FF3010BD002037
:10CEC80010BD002B14BF4FF0FF30012010BD012012
:10CED80010BD08B5FFF7D8FFC043C00F08BD2DE946
:10CEE800F04701F18044089F013C550950F824405F
:10CEF800BD424FEAE47E2C46A8BF3C460026A64227
:10CF080005DA4FF0000C43F826C00136F7E7BD42BA
:10CF180024EAE47439DA2944B942D4BFC4EB0101E4
:10CF2800C4EB0701B2EB45124FEA840501D11D4459
:10CF380020E05E190025AC46C2F120098C450CDAC8
:10CF480025FA09F850F82C5005FA02FA4AEA0808B6
:10CF580046F82C800CF1010CF0E70029A8BF6418F2
:10CF6800BC4212DA25FA09F50EFA02F2154343F823
:10CF780024500EE08A4205DA50F8226045F8226013
:10CF88000132F7E70029A8BF6418BC4203DA43F866
:10CF980024E00134F9E7BDE8F08708600123C017F1
:10CFA800934203DA41F823000133F9E7704708B5E3
:10CFB800FFF76AFF0028CCBF0020012008BD08B594
:10CFC800FFF762FFC00F08BD2DE9F04F01F1804562
:10CFD800013D540950F825708C424FEAE77733DA5F
:10CFE800099DA60025448D42A8BF0D46B2EB441208
:10CFF80001D106442AE050F82490C2F1200A0644E0
:10D00800A3F1040B4FF0000CE0460CF1010C0CEB03
:10D01800040EAE4529FA02FE08DA56F82C9009FAF1
:10D028000AF848EA0E0E4BF804EFEDE78D42ACBF64
:10D038003A4650F8252002FA0AF242EA0E0243F86C
:10D04800282008F101020AE0002208E01119A9428B
:10D0580005DA56F8221043F822100132F6E709994A
:10D068008A4203DA43F822700132F8E7BDE8F08F0C
:10D0780010B54C10C4EB00200144A0EBA0001160D7
:10D08800186010BD70B59C78002829D014B901200B
:10D098001C8098701E881E2E1CD00C8825044D8874
:10D0A80044BF6442A4B22804888844BF6D42ADB22C
:10D0B800010448BF404229B224B248BF80B2A1420D
:10D0C800A8BF214604B2A142A8BF2146B1FA81F106
:10D0D800490900E00021314489B21180198070BDEE
:10D0E80004B1987070BD28B10B6813604B68536029
:10D0F8008B68936070472DE9F04F8DB00B931368E0
:10D1080002920393013B04935368DDF86490189AE4
:10D11800013BDDF858A016680593D9F800300A6875
:10D128000A90049DDAF8000006EB030C55195C42DE
:10D13800C0EB0C0000EB0208A21A2844651B009201
:10D1480014D4B5422C46A8BF3446002A07DB009AFF
:10D15800B242A8BF3246002D174601DA04E0002784
:10D16800B542A8BF354607E0002505E0009A00242F
:10D17800002AECDA27462546B8F1000FA7EB05058B
:10D1880003EB040714DBB045C646A8BFB646002823
:10D1980006DBB042A8BF3046B8F1000F01DA04E060
:10D1A8000020B045A8BFB04608E04FF0000805E0F1
:10D1B80000284FF0000EECDA7046F046C8EB00008D
:10D1C800CEEB0C0C7A19C0EB0C084245A6EB040414
:10D1D800C8BFC7EB0805CEEB0404C8BFC2EB0C0000
:10D1E800641B221A1898D9F804E02F4445684E6841
:10D1F800DAF80400059905EB0E0C7118CEF100045D
:10D20800C0EB0C0000EB0609A61B641A0196084443
:10D2180013D4AC422146A8BF2946002E06DB019E46
:10D22800AE42A8BF2E46002C01DA04E00026AC422C
:10D23800A8BF2C4608E0002406E0019900294FF019
:10D248000001ECDA0E460C46B9F1000FA6EB040417
:10D258000EEB010814DBA9454E46A8BF2E46002850
:10D2680006DBA842A8BF2846B9F1000F01DA04E09E
:10D278000020A945A8BFA94608E04FF0000905E02D
:10D2880000284FF00006ECDA3046B146C9EB000042
:10D29800C6EB0C0CC0EB0C0B08EB0409D945A5EB4D
:10D2A8000101C8BFC8EB0B04A1EB0601C8BFC9EB5D
:10D2B8000C00091B002AA1EB00005ADD002858DDEC
:10D2C80044443A44013A2044F91A0138D31A0793DE
:10D2D800CEEB000308930691CEEB0403089A934221
:10D2E80047DC019A0699C2EB030BDAF8002002FB2F
:10D2F8000BFB189A1568179A5D4302EB8502099291
:10D30800079A914233DC0024A446A646009AC2EB51
:10D318000B020A440598844222DC0B9800EB820930
:10D328000A9800EB8C080020049EB0420BDC59F8E8
:10D33800207058F82060013087FB0667760D46EAB2
:10D34800C726B644F0E70398013420EAE076DAF815
:10D358000000324402440298B4440668921BD9E79C
:10D36800E9425CBF099A42F821E00131C8E701337C
:10D37800B4E70DB0BDE8F08F2DE9F04FADF6BC0D68
:10D38800389365910A92002330F81310CF4A22F897
:10D39800131001330E2B9046F6D1CD4ECD4DB6F875
:10D3A800D437D6F864740D9305F10C03009305F196
:10D3B8006003019305F11803029305F12403039315
:10D3C80005F16403049305F13003059305F13C036B
:10D3D8001046911D06930C322B46FEF7DFFF296895
:10D3E800D6F89421D5F804E08B1AD6F89821AC68C1
:10D3F800D6F89C019C46C2EB0E031A46231A0993E1
:10D4080081EAE173A3EBE1738EEAEE71A1EBEE71B1
:10D418009942B8BF194684EAE47BABEBE47B5945F3
:10D42800B8BF5946B8F80030B6F8FC06B6F8FE960C
:10D438001B1A9BB298B2040448BF5842B8F802308D
:10D4480048BF80B2C9EB03039BB21FFA83F919F4F2
:10D45800004F18BFC3F10009DFF874A29B4BBAF85C
:10D4680000879B8818BF1FFA89F9C8EB03081FFAC1
:10D4780088F81FFA88F31C0444BFC8F100039BB264
:10D48800B1F5600F0EDD0FFA89F900B28145A8BF2A
:10D49800814618B28145A8BF8146B9FA89F94FEA91
:10D4A800591901E04FF000096346002BB8BF5B42F1
:10D4B8009C46002A099BB8BF52429210002BB8BF65
:10D4C8005B4202EBAC0CB9F1000F14BF4FF4A01192
:10D4D8004FF400210CEBA30E14BF4FF4C0004FF41F
:10D4E8000010B1EBEE0FDAF8A04102F3308184EAC4
:10D4F800E473A3EBE4738342C2F2298101231493FA
:10D5080017930D9B002B179B18BF002309939DF8B9
:10D5180024303C930D9B262B3DD8179B002B3AD0EB
:10D52800099B6B49002B02F018804FF00053C1F89B
:10D5380064354FF06043C1F86835674B9F4282F20B
:10D548001480D1F86425D1F868359B1A634A934250
:10D5580002F31980D1F86835D1F864259B1AB3F124
:10D56800333F02F310805A4B5D49D3F868258A424D
:10D57800194642F30380D3F864255A4B9A42C2F203
:10D588000280D1F86435584A9342ACBF0023012386
:10D59800504A82F8A131D6F8B4324E4F5B10C5F824
:10D5A8002031D6F8B83207F590705B10C5F82431F1
:10D5B800D6F8BC3207F29B115B10C5F8283103F08E
:10D5C8002BFE95F89B31002B00F09880D7F8283176
:10D5D800D7F824614FEA430A4FEA6A03C3F10052BD
:10D5E80007F17C0003F1005307F18401FA67C7F8DB
:10D5F8008030D7F82051C6F1000903F0F1FD07F19A
:10D60800800007F1880103F0EBFD49464846FFF723
:10D61800BBFA294680462846FFF7B6FA8044002020
:10D628000146FFF7B1FA4044C7F80C0107F18C0135
:10D6380007F5867003F0D4FD05B9E6B3254BD3F89A
:10D648008C60760811D0314648461F22FFF71DF935
:10D65800314607461F222846FFF717F93146054687
:10D668001F220020FFF711F902E000273D46384647
:10D678001849D1F88860D1F88430760887FB068984
:10D6880085FB064580FB06674FEA987242EA8902E5
:10D698009B085210C1F82C31C1F83021B30FA20FEA
:10D6A80042EA850243EA870352105B10C1F834212D
:10D6B800C1F8383122E0BAF1000F4FF0005315DC01
:10D6C800C7F82C61C7F8303114E000BFD45D0020E2
:10D6D800BC510020F05D002048E17AE43333332365
:10D6E8006666661E9A9999F1666666E6C7F82C31F1
:10D6F800C7F83061C7F83461C7F83861BB4B93F895
:10D708009B215AB1D3F82C211192D3F830210C92D5
:10D71800D3F83421D3F838310B920BE0B44BD3F85B
:10D72800DC241192D3F8E0240C92D3F8E424D3F843
:10D73800E8340B920F930F9A0C9B002183FB024550
:10D74800002C75F10003B4BF6FF060400020221870
:10D7580045EB0103550F45EAC3050B9A119B83FB63
:10D768000223002A73F10001B4BF6FF0604000206B
:10D7780016184FF0000143EB0107720F42EAC70287
:10D78800AD1A6B000C9A1D93119B002183FB024577
:10D79800002C75F10003B4BF6FF060400020221820
:10D7A80045EB0103550F45EAC3050F9A0B9B00276C
:10D7B80083FB0223002A73F10001B4BF6FF06046B7
:10D7C8000026B01847EB0301430F43EAC1032B447B
:10D7D8005B0012935B4210930C9B83FB03010B9B32
:10D7E800420F42EAC10283FB0301430F43EAC1032C
:10D7F80013445B0003F160430E93179B002B41D049
:10D808000D9B072B3ED81D9B5D00109B85EAE57696
:10D818005F00A6EBE57641F0BC8643F24423002E78
:10D8280014BF1846002003B2392043436F4A5B13E4
:10D838005A3B82F897310E9B294628465E00FFF72F
:10D8480010F9394605463846FFF70BF901212844F7
:10D8580076AAFEF784FF769D002D01F0DF86002E64
:10D8680001F3E88641F0108746F2884010EA250067
:10D8780038BF3046392300B258435C4B401340420E
:10D8880083F89801594B5A4A9C46D2F8AC01D2F811
:10D89800B041D2F8B4111D9AD3F828E155428EFB55
:10D8A8000589B8F1000F79F10002B4BF6FF060424A
:10D8B800002218EB0206C3F89800C3F89C40C3F88E
:10D8C800A0104FF0000349EB0307720FDCF820317A
:10D8D8000E9E4FF0000983FB06ABBAF1000F7BF1F7
:10D8E8000006B4BF6FF060484FF000081AEB080656
:10D8F8004FEA567A42EAC7024BEB09074AEAC70AD7
:10D90800CAEB020A109A002783FB0289B8F1000FBC
:10D9180079F10003B4BF6FF06046002618EB0602E9
:10D9280049EB07034FEA527C4CEAC30C2F4B002704
:10D93800D3F824211B6E82FB0589B8F1000F79F119
:10D948000005B4BF6FF06046002616EB080647EBEB
:10D958000907750F45EAC7055B08C5EB0C0CA3F56D
:10D96800001585EAE573A3EBE573214E214DAB4223
:10D97800B6F8D657CCBF00230123142D319308BF26
:10D9880000232B449BB2A3F114073D937B427B41B8
:10D99800194D1A4F002B18BF3D46D6F880733D44E9
:10D9A800B5F1806F05DBB5F1804FA8BF4FF080451A
:10D9B80001E04FF0806525958000A40089001BBB1D
:10D9C80080EAE07584EAE473A3EBE473A5EBE07501
:10D9D8001D4481EAE173A3EBE1732B44084E094D22
:10D9E800259FB342D8BF3D460FE000BFF05D002041
:10D9F800BC51002065660600666666009A9999FF24
:10DA08006566660093180400259D0E9B002782FB1F
:10DA18000323002A73F10006B4BF6FF060460026A6
:10DA280012EB06084FEA587243EB070942EAC903AA
:10DA3800109A4FF000098EFB0267002E77F1000262
:10DA4800B4BF6FF060484FF0000816EB080647EBCC
:10DA58000907720F42EAC7029A1A82FB0589B8F1D0
:10DA6800000F79F10003B4BF6FF06046002618EB91
:10DA780006024FF0000749EB07034FEA527848EADD
:10DA8800C30313F008080AD05E0706D1002BD4BFE1
:10DA98004FF000084FF0010801E04FF0010808EBD3
:10DAA80023188AFB0523002A804473F10000B4BFC1
:10DAB8006FF06046002612EB060A4FF0000743EBB2
:10DAC800070B4FEA5A7242EACB0313F0080207D059
:10DAD800580704D1002BD4BF0022012200E0012204
:10DAE80002EB23131C448CFB0523002A73F100006E
:10DAF800B4BF6FF0604A4FF0000A1AEB02064FF00D
:10DB0800000B4BEB0307730F43EAC70313F0080737
:10DB180007D05A0704D1002BD4BF0027012700E003
:10DB2800012707EB23170F4488FB0801820F42EAFD
:10DB380081026FF000408B1790424FF0000171EBAB
:10DB4800030509DB44484FF0FF31824273EB0101C2
:10DB580003DA4FF0004200E0024684FB04AB4FEAD0
:10DB68009A7040EA8B006FF0004A4FEAAB71824529
:10DB78004FF0000B4FEAA2037BEB01020ADBDFF850
:10DB8800D8A04FF0FF3B504571EB0B0203DA4FF082
:10DB9800004000E0504687FB07AB03EBA0034FEAC9
:10DBA8009A7040EA8B006FF0004A4FEAAB718245E9
:10DBB8004FF0000B7BEB01020ADBDFF89CA04FF073
:10DBC800FF3B504571EB0B0203DA4FF0004000E0D9
:10DBD8005046224D03EBA003284605F16C0140F89E
:10DBE800683F03F0FDFAE96E1D48FEF7C3FF1D4BC1
:10DBF80080FB0301CD00B5F1004F07D8B5F1804F88
:10DC080094BFC5F1804305F1404306E0B5F1404FAC
:10DC18002CBF05F18043C5F140437F9300217CABC5
:10DC28004FF480627F98FFF72AF80F4A7C997F901B
:10DC3800FFF739F805F140430C4A013B934298BF7E
:10DC4800404243101393054BDB6E8BB1A6104FEA8D
:10DC5800A809BF109C0810E001000080F05D0020BA
:10DC68003D0AD7A3B7C17C512CC64100FEFFFF7FF8
:10DC78001F4699461E46134A1468B5F1004F8CBFDB
:10DC88004FF0000A4FF0010ABAF1000F01D105F177
:10DC980000457F957F9B0021B3F1804F84BFC3F17E
:10DCA80000437F934FF480627F987DABFEF7E7FFD8
:10DCB8007D99054A7F90FEF7F6FFBAF1000F05D16E
:10DCC800404203E050D641002CC641004FEA6008AC
:10DCD8001E2221464846FEF7B9FD80FB08ABBAF183
:10DCE800000F7BF10003B4BF6FF0404200221AEB33
:10DCF80002004FF000034BEB0301850F45EA810555
:10DD08001E2221463046FEF7A1FD80FB08ABBAF182
:10DD1800000F7BF10003B4BF6FF0404200221AEB02
:10DD280002004FF000034BEB0301860F46EA810621
:10DD38001E2221463846FEF789FD80FB080100288F
:10DD480071F10003B4BF6FF04042002212EB0008EB
:10DD58004FF0000343EB0109119A13994FEA9873A6
:10DD680082FB01ABBAF1000F7BF10002B4BF6FF088
:10DD780060484FF000081AEB080043EA89034FF0A7
:10DD880000094BEB0901420F42EAC1020C994FF01E
:10DD9800000981FB05ABBAF1000F7BF10001B4BFAC
:10DDA8006FF060484FF000081AEB08004BEB0901D0
:10DDB800470F47EAC107D71B0B9A4FF0000982FBB0
:10DDC80006ABBAF1000F7BF10002B4BF6FF06048F8
:10DDD8004FF000081AEB08004BEB0901420F42EA2A
:10DDE800C1020F994FF0000981FB03ABBAF1000F94
:10DDF8007BF10001B4BF6FF060484FF000081AEBE8
:10DE080008004BEB0901BA1A470F47EAC107D71BAD
:10DE1800119A4FF0000982FB05ABBAF1000F7BF1B4
:10DE28000002B4BF6FF060484FF000081AEB08001A
:10DE38004BEB0901420F42EAC10213980C994FF0CB
:10DE4800000B81FB000180468946002871F1000122
:10DE5800B4BF6FF0604A4FF0000A18EB0A0849EBAC
:10DE68000B094FEA587444EAC90414440B9A4FF05A
:10DE7800000B82FB0301002871F10002B4BF6FF0B0
:10DE8800604A4FF0000A10EB0A0841EB0B090F99A2
:10DE98004FEA587281FB0601804642EAC902894668
:10DEA800002871F10001B4BF6FF0604A4FF0000A1A
:10DEB80018EB0A084FF0000B49EB0B0922444FEA14
:10DEC800587444EAC904141B119A4FF0000982FBE4
:10DED80006ABBAF1000F7BF10002B4BF6FF06048E7
:10DEE8004FF000081AEB08004BEB0901420F42EA19
:10DEF800C1020C994FF0000981FB03ABBAF1000F86
:10DF08007BF10001B4BF6FF060484FF000081AEBD6
:10DF180008004BEB09014FEA507A4AEAC10A139804
:10DF28000B99CAEB020281FB000180468946002852
:10DF380071F100010F99B8BF6FF0604A81FB0501CC
:10DF4800A8BF4FF0000A18EB0A084FF0000B49EB86
:10DF58000B094FEA587A80464AEAC90A89460028D6
:10DF680071F100015244B4BF6FF0604A4FF0000AEB
:10DF780018EB0A084FF0000B49EB0B094FEA587AE7
:10DF88004AEAC90A9244119A4FF0000982FB030138
:10DF9800002871F10003B4BF6FF060484FF000082B
:10DFA80010EB080241EB09034FEA527E4EEAC30E1A
:10DFB8000C9B83FB0623002A73F10001B4BF6FF0AA
:10DFC8006040002012EB00084FF0000143EB01090C
:10DFD8004FEA58720B9B42EAC902964483FB052319
:10DFE800002A73F10001B4BF6FF06040002012EB0B
:10DFF80000084FF0000143EB01094FEA587242EA6A
:10E00800C902C2EB0E0E0F9B139ABE4D83FB028909
:10E01800B8F1000F79F10003B4BF6FF0604200223D
:10E0280018EB02004FF0000349EB030187FB078957
:10E0380084FB0423460F46EAC106D10F4FEAD87283
:10E0480042EA490241EA4301D21002EBE1028AFBAB
:10E058000A017644C30F43EA410386FB060102EB3B
:10E06800E302C30F43EA410305F5C67005F17001E9
:10E0780002EBE302C5F88C2103F0B2F82B6FA24A39
:10E0880093428DBF99464FF080590026601098BF83
:10E09800304649464FF01D028DBF7D10B2464D46B1
:10E0A8004FEA6A0A88BF7610FEF7D0FB49463E90D1
:10E0B8001D225046FEF7CAFB49463F901D223046B6
:10E0C800FEF7C4FB3E9BC0F100085E423F9B4946F9
:10E0D80040901D2228465F42FEF7B8FB87FB0745A4
:10E0E800299088FB0801874BD3F898C0C30FE00F2D
:10E0F80043EA410340EA45001844C0F1806040000B
:10E108008CFB00ABBAF1000F7BF10002B4BF6FF0DB
:10E118007E4400241AEB04004FF000054BEB050188
:10E1280086FB0745420EE00F0B9342EAC11340EA13
:10E13800450129984FF0000B80FB0845E00F40EAA5
:10E148004500704D0C18D5F89CE0640084FB0E4522
:10E15800002C75F10009B4BF6FF07E4A4FF0000A39
:10E1680014EB0A020C934FEA526445EB0B0344EAA2
:10E17800C3140C9B081A234486FB06451993E20F27
:10E188000B9B42EA45021A44C2F18062520082FBAC
:10E198000EABBAF1000F7BF10003B4BF6FF07E4401
:10E1A80000241AEB04024FF000054FEA40004BEB45
:10E1B80005038CFB00AB540EBAF1000F44EAC314FC
:10E1C8007BF10003B4BF6FF07E4200221AEB02001D
:10E1D8004FF000034BEB0301430E43EAC11386FBE8
:10E1E8000801E318299A1A93C30F43EA410382FBF3
:10E1F8000701C20F42EA41021A4452008CFB024551
:10E20800002C75F10003B4BF6FF07E400020221887
:10E218004FEA5264299A87FB088982FB06674FF008
:10E22800000145EB010344EAC314F20F4FEAD87327
:10E2380043EA490342EA47029A1A520082FB0E2334
:10E24800002A73F10001B4BF6FF07E400020161859
:10E258004FF0000143EB0107720E42EAC712A31800
:10E26800002B159303DB14BF0123002301E04FF0BB
:10E27800FF332F93254B2F991A6891421DBF002118
:10E2880008460A46199A01BFD3F83C13D3F840034D
:10E2980001EB22211A9A01BF00EB2220D3F8442374
:10E2A800159B02EB2322194BC3F83C13C3F8400318
:10E2B800C3F84423099B002B3DD0124BBCF1000F3F
:10E2C800C3F8F020BABFCCF10002C3F8AC20C3F801
:10E2D800ACC0BEF1000FBABFCEF10002C3F8B02047
:10E2E800C3F8B0E0BCF1000FC3F8E810C3F8EC00C5
:10E2F800044C02DA4FF0FF3301E009D00123E36553
:10E3080008E000BFF05D0020C3F52800BC510020E4
:10E31800C4F85CC0D4F8AC000146FEF7A2FBD4F800
:10E32800B0000146FEF79DFB159B002BD4BF0023D0
:10E33800012384F8A5310023284A1A44D2F83C1650
:10E348000DF5956299500433282BF5D10D9BA3F157
:10E358002709D9F1000343EB090332930D9B082BDE
:10E3680040F0CB8000231D4A0DF59A611A44D2F87B
:10E378001426002AB8BF5242CA500433282BF2D1BF
:10E38800DDF8D034002201320DF59A6151F82210DF
:10E398008B42B8BF0B46092AF5D1114A0024C2F8AE
:10E3A800B430104A83FB02239C460C4B03F52A70B9
:10E3B800B3F8DE27D3F8A41203F5C263C1C853F833
:10E3C800045F85EAE57EAEEBE57EE6450CDC12F1FE
:10E3D800000E18BF4FF0010E08E000BFBC5100202E
:10E3E800F05D0020CDCCCC4C4FF0010E724492B2BF
:10E3F80002F1FF38D8F1000E4EEB080EBEF1000F07
:10E4080002F01586002D2946C2F201860D1C18BFA0
:10E418000125BEF1000F42F0FC85002C04F1010437
:10E4280008BF00220A2CCAD1BD4BBE4CC3F8A412A7
:10E43800C4F8C410ED0F0146A3F8DE27C3F8A802FC
:10E44800C3F8AC62C3F8B07284F8A751C4F8C80026
:10E45800C4F8CC60C4F8D070FEF703FB0546D4F8C6
:10E46800CC000146FEF7FDFA0121284479AAFEF7FF
:10E4780076F97999D4F8CC004B001E22C4F8D8302C
:10E48800FEF763FA01461920FEF767FB00B263281E
:10E4980002F3C6856FF063039842B8BF18461D9B08
:10E4A800002BC2F2C08514BF01230023DDF8A81495
:10E4B80058430A4684F89A01002301330DF5956004
:10E4C80050F823008242B8BF02468142A8BF0146E5
:10E4D800092BF2D1934B521AC3F8B820D3F8AC20C9
:10E4E800002AB8BF5242C3F8BC20D3F8B0308D4AD6
:10E4F800002BB8BF5B42C2F8C030329B83B1389B57
:10E50800894A1978894B002918BF1346854AD2F8D9
:10E51800B810B3EB611FACBF0123002382F8A6310A
:10E528007F4B0F21D3F8E021D3F8DC411E92D3F8BA
:10E53800E421CDF82C451F92D3F8E821072020923A
:10E54800D3F8EC2185AE2192D3F8F0210025229250
:10E55800D3F8F4212392D3F8F8213392D3F8FC218D
:10E568003492D3F80022D3F80432359236931E9BA6
:10E57800CDF830351F9BCDF83435209BCDF8383594
:10E58800219BCDF83C35229BCDF84035239BCDF817
:10E598004435339BCDF85C25CDF85435349B8591B3
:10E5A800CDF85835369B8791CDF860355D4B6FF0C7
:10E5B8000601D3F898208B91D4338DA9CDF8642522
:10E5C8008D90012289A88692889289928A920193D5
:10E5D8000290039100960DF22C508BA987AA544BF8
:10E5E800CDF84855CDF84C55CDF850558C958E95AD
:10E5F800FEF781FD0DF22C5353F8251081EAE172E4
:10E60800A2EBE17243F8252001350F2DF2D1DDF898
:10E618002C65002301330DF22C5252F82320964228
:10E62800B8BF16460E2BF5D1002CBCBF6342C3936E
:10E638001E9BA8BFC394002BACBF1E9B5B42C49318
:10E648001F9B84EAE47A002BACBF1F9B5B42C593F7
:10E65800209BAAEBE47A002BACBF209B5B42C693BD
:10E66800219B0022002BACBF219B5B42C793229BBE
:10E67800002BACBF229B5B42C893239B002BACBFF3
:10E68800239B5B42C9930132C3AB53F822108A45DE
:10E69800B8BF8A46062AF6D13398349A0028B8BFFC
:10E6A8004042002AB8BF524291463599369A00290D
:10E6B800B8BF4942002AB8BF52424845B8BF484689
:10E6C8008842B8BF084690428146B8BF9146144A6E
:10E6D800144DD2F80812D5F898502491D2F80C129B
:10E6E80085EAE5772A91D2F81012A7EBE5772B9106
:10E6F800D2F81412B9452C91D2F81812D2F81C226B
:10E70800B8BFB9462E92249A2D91002AACBF249AFC
:10E7180052421A602A9B002BA8BF2A9B0AE000BF1E
:10E72800BC510020F05D002066662600B81E25005A
:10E73800ACC54100B8BF5B42C4932B9B002BACBF58
:10E748002B9B5B42C5932C9B002BACBF2C9B5B4245
:10E75800C6932D9B002BACBF2D9B5B42C7932E9B72
:10E76800002BACBF2E9B5B42C893724B249FD3F8FF
:10E778009C30002BB8BF5B42002FC993B8BF7F42C3
:10E7880000230133C3AA52F823209742B8BF174683
:10E79800062BF6D10DF50F7CDFF8988101217F94C7
:10E7A8000224CDF800C00B467FA880AA0194CDF8BA
:10E7B8002CC0DFF88CB18095FEF79FFAD8F89C3012
:10E7C80097AD7F93DBF82032012180937FA80B4619
:10E7D80080AA00950194FEF790FADDF82CC029462E
:10E7E800604699AA2346FEF735FBD8F8A0300121E8
:10E7F8007F93DBF840327FA8809380AA0B46009570
:10E808000194FEF77AFA99A829469BAA2346FEF7AF
:10E8180021FBD8F8D43050469B469DA92246FEF7E6
:10E82800BCFB0DF51F782B469DA821461E2200949F
:10E83800FEF755FB484641462246FEF7AEFB4046EA
:10E8480021461E229DAB0094FEF749FB01214FF0A3
:10E8580066337F937FA80B4680AACDF80080019489
:10E86800CDF800A2FEF749FA4846A3A92246FEF7CA
:10E8780094FB0DF52579A1ABA3A82146202200948D
:10E88800FEF72DFB384649462246FEF786FB4846EA
:10E8980021462022A3AB0094FEF721FBDFF8A4A0B9
:10E8A80001210B467FA880AACDF800900194CDF8ED
:10E8B800FCA18096FEF721FA5B461F4A002B86FBD7
:10E8C80002014FEA1072B8BF5B4242EA011293425A
:10E8D8009B461DDBB6F1A06F1AD828469DA9224693
:10E8E800FEF7F7FAA0B14046A1A92246FEF75FFB62
:10E8F80070B1A3A849462246FEF759FB40B1B7F5C7
:10E90800200F05DC9BA80D492246FEF750FB20B9D5
:10E918000B4BD3F89071013700E00027084B93F8B0
:10E92800042CC3F890710AB1149A6AB9B3F8D8578D
:10E938000BE000BFF05D0020DBF97E6294C541006A
:10E94800BC510020CDCCCC4C00254FF6FF730135CF
:10E95800B5F5803F08BF1D46ABB20E2B419394BF5F
:10E968000023012342930D9BA3F11200434243412C
:10E978003793002B00F08880DFF8C882199B0226A5
:10E988007F93D8F884330DF5117901218093CDF860
:10E9980000900B467FA880AA0196FEF7AEF91A9B55
:10E9A800A7AC7F93D8F88833012180938DE8500075
:10E9B8000B467FA880AAFEF7A0F948462146A9AAD7
:10E9C8003346FEF747FA159B01217F93D8F88C331D
:10E9D8007FA880938DE850000B4680AAFEF78DF93A
:10E9E8002146A9A8ABAA3346FEF734FAD8F88433EF
:10E9F800D8F8881383EAE372D8F88C03A2EBE372A1
:10EA080081EAE173A3EBE17380EAE074334103EB3D
:10EA1800A203A4EBE07403EBA404854BABA88549DF
:10EA28003246D3F8C490FEF7CAFA48B189EAE978C1
:10EA3800A8EBE978B8F5900F22DBB4F1607F1FDC12
:10EA4800ABA87D490222FEF7BAFAC8B9B4F5000F9F
:10EA580016DB199A1A9B002AB8BF5242002BB8BF7E
:10EA68005B429B1003EBA203159A002AB8BF5242DF
:10EA780003EBA203B3F5801FACBF0023012300E022
:10EA880001236B4A82F8A031694E0D9BD6F8AC4041
:10EA9800991E002CB8BF64424B424B410B944393E0
:10EAA800002B73D0109A129B199813EA220338BFCF
:10EAB800134601461293FEF73AF880461A984FEA31
:10EAC80058080146FEF733F808EB50008308304633
:10EAD80006F1940140F8903F02F082FB159BD6F8AE
:10EAE8009440002BB8BF5B4283FB0AABD6F8981062
:10EAF80084EAE4724FEA9A73A2EBE47243EA8B0366
:10EB080081EAE1709A42A0EBE17009DD129BB3F152
:10EB1800C05F05DDB0F1207FACBF0023012300E01A
:10EB28000023D6F89C2086F89F3182EAE271434B95
:10EB3800A1EBE27181FB03894FEA987242EA8902EC
:10EB4800D6F898309042ACBF00210121002B86F8FE
:10EB58009E1103DB14BF0123002301E04FF0FF33B4
:10EB6800374A0E9991420DDD364AD2F8EC248A1ABA
:10EB7800002A07DD109A5343334A9342ACBF00235F
:10EB8800012300E000232A4A82F89D310B9BDFF81D
:10EB9800A090B3F1107F09DAD9F89C3133F0FF0364
:10EBA80014BF4FF0010A4FF0000A01E04FF0000ACD
:10EBB800D9F898001E4E0146FDF7A3FF8046D9F804
:10EBC8009C004FEA58080146FDF79BFF08EB5000F0
:10EBD8008008C9F8740006F1780106F1740002F0A3
:10EBE800FFFAD9F87820099B82EAE274A4EBE27470
:10EBF80083B1164996F897318C4286F8993105DC2D
:10EC08005BB2472BD4BF0023012300E0002308494F
:10EC180081F8A931379BF3B10C4B05499C4217DCAD
:10EC280091F99931542BD4BF0023012311E000BF7F
:10EC3800F05D00209CC54100A4C54100CDCCCC0CA2
:10EC480033333303BC510020676666F6CCCC8C04A2
:10EC5800002381F8AB31B64BB64993F8E12B4492C7
:10EC680093F8E22B459293F8E32B469293F8E42B22
:10EC7800479293F8E52B489293F8E62B499293F83C
:10EC8800E72B4A9293F8E82B4B9293F8E92B4C9296
:10EC980093F8EA2B4D9293F8EB2B4E9293F8EC2BCA
:10ECA8004F9293F8ED2B509293F8EE2B519293F8E4
:10ECB800EF2B529293F8F02B539293F8F12B549236
:10ECC80093F8F22BD1F89810559293F8F32B00296A
:10ECD800569293F8F42B93F8051C579293F8F52B5A
:10ECE800589293F8F62B599293F8F72B5A9293F877
:10ECF800F82B5B9293F8F92B5C9293F8FA2B5D92C0
:10ED080093F8FB2B5E9293F8FC2B5F92ACBF012229
:10ED1800FF223992002900F0948093F8E03B8DF8A7
:10ED280028339DF810318DF829339DF814318DF86A
:10ED38002A339DF818318DF82B339DF81C318DF846
:10ED48002C339DF820318DF82D339DF824318DF822
:10ED58002E339DF828318DF82F339DF82C318DF8FE
:10ED680030339DF830318DF831339DF834318DF8DA
:10ED780032339DF838318DF833339DF83C318DF8B6
:10ED880034339DF840318DF835339DF844318DF892
:10ED980036339DF848318DF837339DF84C318DF86E
:10EDA80038339DF850318DF839339DF854318DF84A
:10EDB8003A339DF858318DF83B339DF85C318DF826
:10EDC8003C339DF860318DF83D339DF864318DF802
:10EDD8003E339DF868318DF83F339DF86C318DF8DE
:10EDE80040339DF870318DF841339DF874318DF8BA
:10EDF80042339DF878318DF843339DF87C318DF896
:10EE080044339DF8E4308DF845330023184600F567
:10EE18008451494E1C318E5DCAA9415C013006FB04
:10EE280001331E28D9B2CBB2F1D11A0644BF4B42E6
:10EE3800DBB25BB2182B3F49D4BF0023012381F812
:10EE4800AC31099B8BB104F17F423C4B013A9A42A9
:10EE5800384A07D892F9983113F1400FACBF002314
:10EE6800012300E0002382F8AA31C82F20DD429B4D
:10EE78001BB1642D01DC149BD3B92E4B93F8A02150
:10EE8800B2B9BAF1000F16D1D3F8A82112F0FF2FAA
:10EE980012D193F8AC311BB10B9BB3F1207F0BDA85
:10EEA800244B93F8AA31B3FA83FA4FEA5A1A03E0CB
:10EEB8004FF0000A00E092461D4C81A9B4F80837CB
:10EEC8001F4AADF80432B4F80A371E4DADF80632C1
:10EED800B4F80C37ADF808320D9B102B179B88BF80
:10EEE80000231C939DF8706004F614433046FEF727
:10EEF800C9F8B4F86237B5F89471ADF80C32B4F8C3
:10EF080064373046ADF80E32B4F8663783A9ADF8E9
:10EF1800103205F5C97204F54163FEF7B3F8022F04
:10EF280012D8B5F89231022B94BF002301230CE0CC
:10EF3800BC510020F05D002094C54100FEFF7F0613
:10EF4800845F0020F05D002001230C93C14B0B93DC
:10EF58001A46002350680DF5B76141F82300506A3E
:10EF6800D2A941F823000133082B02F10402F1D1A0
:10EF78000023B84A0DF5B7611A44506A194408626B
:10EF8800516CDAAA99500433202BF2D10023B14AEC
:10EF98000DF5B7611A44506C19440864516EE2AA21
:10EFA80099500433202BF2D10023AA4A0DF5B761FA
:10EFB8001A44506E19440866D2F88410EAAA995087
:10EFC8000433202BF1D10023A24A0DF5B7611A446E
:10EFD800D2F884001944C1F88000D2F8A410F2AA2B
:10EFE80099500433202BEFD100239A4A0DF5B761CD
:10EFF8001A44D2F8A4001944C1F8A000D2F8C410E9
:10F00800FAAA99500433202BEFD10023914A0DF529
:10F01800B7611A44D2F8C4001944C1F8C000D2F844
:10F02800E4100DF5816299500433202BEED10023B2
:10F03800884A0DF5B7611A44D2F8E4001944C1F8BA
:10F04800E000D2F804110DF5856299500433202BA5
:10F05800EED100237F4A0DF5B7611A44D2F80401B6
:10F068001944C1F80001D2F824110DF589629950AC
:10F078000433202BEED10023764A0DF5B7611A44EC
:10F08800D2F824011944C1F82001D2F844110DF531
:10F098008D6299500433202BEED100236D4A0DF573
:10F0A800B7611A44D2F844011944C1F84001D2F8B2
:10F0B80064110DF5916299500433202BEED1002292
:10F0C8000DF5B7639918634BD018D0F86401043272
:10F0D800202AC1F86001F3D193F8092C93F80C1C8D
:10F0E800002A00F08D8111B9012283F80C2C00232D
:10F0F8000DF5B76252F823200DF5E761002AB8BF75
:10F10800524241F823200133602BF1D1DDF83867F2
:10F11800002301330DF5E76252F823209642B8BF69
:10F1280016465F2BF5D14FF0333086FB0001830C78
:10F13800494843EA813386FB0001C3F3C03202EB3E
:10F1480023431493C30B43EA4143C3F3C03202EB96
:10F158002343189300240DF5B76353F824900F2E1A
:10F1680089EAE975D4BF4FF0000B4FF0010BA1B24B
:10F17800A5EBE975374ABBF1000F02D0149B9D42FD
:10F1880005DCB2F8DA37003318BF012300E00123A9
:10F19800B2F8DA2713449BB25F1E1D2F8CBF0027DD
:10F1A80001270F932D4B0FB9A3F89011DFF8A48016
:10F1B800B3F890C1A2B2484616927BABD8F8F416C1
:10F1C8007AAACDF844C0FDF753FFD8F8F8064FEAFD
:10F1D8000923184413934FEA6009DDF844C0BBF1D2
:10F1E800000F02D0189B9D4205DCB8F8DC370033CD
:10F1F80018BF012300E00123B8F8DC17154A0B44B7
:10F208001FFA83F808F1FF33152B144B11D8D2F8E5
:10F21800301389EAE970A0EBE97001447B98C3F8E0
:10F22800DC10D2F8342380EAE071A1EBE0710A44E3
:10F2380005E0D2F83013D2F83423C3F8DC10C3F851
:10F24800E0206CB1054BD3F8DC20D3F8E030119204
:10F25800129307E0BC51002033333373F05D002074
:10F26800129411947D4B93F80F2C002F00F0998085
:10F2780022B9C3F83823012283F80F2C169BCCEB54
:10F288000305ADB2754BAFB2D3F8382339B2744B1E
:10F298000029C3F8E4200CDA1122B5A80CF002FB0F
:10F2A800B59BC3EB0332C3EB021311332B449BB260
:10F2B80005E0B7A811220CF0F5FABDF8E03240F6E7
:10F2C8000F7B03FB0BFB4FEA0B4BBBF1004F07D83F
:10F2D800BBF1804F94BFCBF180430BF1404306E074
:10F2E800BBF1404F2CBF0BF18043CBF140437F93E0
:10F2F80000217EAB10227F98FDF7EBFC7E99594ADE
:10F308007F90FDF7D0FC389B1B7843B10BF1404B45
:10F31800554B0BF1FF3B9B4526D8404224E039B2C0
:10F3280000290DDA0B22B9A80CF0BCFAB99B03EB43
:10F33800830203EB4203C3F10B031D44ADB205E0A6
:10F34800BBA80B220CF0AEFABDF8F0522BB2002B82
:10F3580009DD053D012D06D9062BCCBF4FF04040F5
:10F368004FF0804000E0002089FB0001820F42EA54
:10F3780081023A49D1F83803002800EB020306DA83
:10F38800002A0BDA002BA8BF4FF0004306E005D097
:10F39800002A03DD002BD8BF6FF00043C1F83833D3
:10F3A80002E00AB183F80F7C2C4B24B1BDF83C2055
:10F3B800A3F8DA2701E0A3F8DA477A99274AC3F8CD
:10F3C800F4161399C3F8F8161199C3F83013129963
:10F3D800C3F8341314B1A2F8DC8701E0A2F8DC47C3
:10F3E8000134602C7FF4B7AE0F9B23B1192ED4BF24
:10F3F8000026012600E00F9E194B83F8AD6109E055
:10F4080041B193F80F1C09B183F80F2C134B00225C
:10F4180083F80C2C0D9B632B0CD1BAF1000F01D192
:10F428000C9B4BB10E4B93F8AD21002A40F0B481F0
:10F438000C9201E000230C931C9A084BB2B193F88C
:10F448000D2C22B9C3F8A022012283F80D2CD3F881
:10F45800A022034BC3F8A8200FE000BFBC51002036
:10F46800F05D0020E8C54100FEFFFF7F93F80D2CFA
:10F478001AB19DF8702083F80D2CB94C1D9AD4F858
:10F48800F0343C98D31ABD93109AD4F8F434BDA93B
:10F49800D31ABE930E9AD4F8F83495AED31AB14A5B
:10F4A800BF93FDF720FED4F8FC34BD9AD4F80015BC
:10F4B800D31ABE9AC093521AC192D4F80415BF9AAF
:10F4C8000224521A0121C2927F9380937FA80B468F
:10F4D80080AA00960194FDF710FCC19B012193AD11
:10F4E8007F9380937FA80B4680AA00950194FDF72F
:10F4F80004FC30462946ADAA2346FDF7ABFCAFAB6A
:10F50800ADA821461D220094FDF75EFDAF9875AAAF
:10F5180001217F90FDF723F9099A934B12B1759A4F
:10F52800C3F81C21D3F81C316393C09B002BB8BFD0
:10F538005B4218938A4BD3F80825002A03DC0E9AFD
:10F54800002A81F27B85D3F80C351493149A189B02
:10F558009342C0F2518101F080BDD1F864359F42D9
:10F5680000F30881C1F8647504E1804B9F42FDF601
:10F57800F1AFB7F1704F09DAFDF7F5BF7C4B9A424E
:10F5880004DDFDF7FEBF0123FEF702B80023FDF7F7
:10F59800FFBF4EB3B74200F0F780002F06DBBE4234
:10F5A80002DC304639460EE038461BE0B7F1004F22
:10F5B80014BFC7F1000B6FF0004B5E4500F0E88008
:10F5C8000FDA304659461022FDF7A2F980F31000F1
:10F5D80080B2FDF72BFB002FC0F3CF0003B20BDA8C
:10F5E80010E058463146EEE746F28843002FACBF9C
:10F5F80000201846FEF717B9B742BEF614A9C3F59E
:10F60800495303E05E4503DD03F54953033302E044
:10F61800C3F5C943073398B2FEF705B9002E03DCDA
:10F6280014BFFF20002000E0012043F2442340B231
:10F63800584389E0B54201F05E85002D14DBAE42E7
:10F6480002DC3046294601E0284631461022FDF703
:10F658005FF980F3100080B2FDF7CCFA002DC0F3FB
:10F66800CF0003B255DA5AE0B5F1004F14BFC5F127
:10F67800000B6FF0004B5E4501F0418502DA304621
:10F688005946E3E75846E0E7B54201F03C85002DCE
:10F6980011DBB6F1004F07D07642AE4201F0378554
:10F6A80007DA304629461DE06FF00046B54201F002
:10F6B8002E8528462BE0B5F1004F0BD0B6F1004F50
:10F6C800C5F1000B01D0764201E06FF000465E45BF
:10F6D8001CDC05E0B6F1004F6FF0004BF3D15E463D
:10F6E800304659461022FDF713F980F3100080B216
:10F6F800FDF780FA002DC0F3CF0398B219DBAE42B4
:10F70800CABFA0F54950584203381DE05846314653
:10F71800E8E7B542BEF6AEA8C3F5495003E05E453A
:10F7280003DD03F5495003300EE0C3F5C940073047
:10F738000AE05E4500B2C5BF00F549500330A0F5A8
:10F74800C9404042D8BF073880B2FEF793B80D9B36
:10F75800003318BF0123179300231493FDF7D1BE7C
:10F76800BC510020705F0020F05D0020CDCCCCECB7
:10F778009A999909D1F868359F42FDF6DEAE894B12
:10F78800C3F86875FDF7D9BE41F62210FEF74BB8ED
:10F7980044F66630FEF747B893F99A21232A1FDC0E
:10F7A800D3F8F020002A20DB14BF012300232824EB
:10F7B80016204FF42001B2F57A0F7B4D03DA95F944
:10F7C8009861A64205DC95F99841844203DD8A4296
:10F7D80001DADBB200E00023734A82F8963102E0D6
:10F7E800002283F89621012325E652424FF0FF3389
:10F7F8002D2420206D49DEE7099BB3B10023C19C6D
:10F80800694A1499002CB8BF6442C2F844110F9495
:10F81800002B41F04784634B0F99D3F81025914290
:10F828001392614A07DB01F027BCC19C002CB8BFCA
:10F8380064420F94EFE7099911B11399C2F8501176
:10F84800D3F81425C29B9A42B8BF1A462792099A40
:10F858002AB10025544A2799C2F8481100E0099DA9
:10F8680075991DB94F4AD2F8182500E000228A423E
:10F87800B8BF0A463B92099A52B14B4A3B99C2F823
:10F888003C11002D41F09483464AD2F81C2502E031
:10F89800002DF9D0099A9A42A8BF1A46099B3092BE
:10F8A8001BB1414B309AC3F84C21BD9A82EAE273EE
:10F8B800A3EBE2731B9355B93A4BD3F82035129357
:10F8C80012991B9B8B42C1F2788301F0FABB099B0A
:10F8D80033B11B9B1293344B1299C3F8541101E0B6
:10F8E8001B9B1293BE9B002BB8BF5B421193002D4C
:10F8F80041F0F4832B4BD3F82415169116981199DF
:10F9080081420999C1F26483002901F06683119943
:10F91800169125491698C1F86001D3F82835BF9982
:10F928009942B8BF1946099B26911BB11E4B2699CF
:10F93800C3F85811022601210DF515780B467F9260
:10F9480080927FA880AACDF800800196FDF7D5F9AE
:10F95800BE9B012193AF7F9380937FA80B4680AA1B
:10F9680000970196FDF7C9F9404631461D22B1AB13
:10F978000096FDF729FBB19B38467F9331461D223F
:10F98800B3AB0096FDF720FB7F98B39B74AA18448D
:10F9980001217F90FCF7E3FE749A4DB9014BD3F82F
:10F9A8002C3506E0BC510020F05D00200080BB0033
:10F9B80000239342B8BF13463A93099B002B01F0EA
:10F9C8001683DF4B3A9AC3F84021002D41F0098392
:10F9D800DC4BBF9AD3F830359A42A8BF1A46099B28
:10F9E80028921BB1D64B289AC3F85C21D64A3C987A
:10F9F800C0A9FDF778FBD54BD3F8D8203C92D3F8B3
:10FA0800E42064920C9A002A00F02184D3F8C800FC
:10FA1800D3F8CC10D3F8D0E0421060924A1061922B
:10FA28004FEA6E026292D3F8A82000275310C84A02
:10FA380083FB0289B8F1000F79F10003B4BFC54E0A
:10FA4800002618EB060249EB0703BD4F560DB7F821
:10FA5800942146EAC3261305BF4A4FF0000983FBE9
:10FA68000223002A73F10004B4BFDFF81C834FF0AF
:10FA7800000812EB080A43EB090B53469A0D42EAB9
:10FA88008B22CDF86C25B7F89221D046130548F69D
:10FA9800390283FB0223002A73F10004B4BFDFF8A4
:10FAA800EC824FF0000812EB080A4FF0000943EB14
:10FAB800090B5346D046A24FDA0CD7F8BC3042EABD
:10FAC8004B32CDF8702583EAE372A2EBE372A34BC5
:10FAD800521082FB0323002A73F10004B4BFDFF83D
:10FAE80074824FF0000812EB080A4FF0000943EB4C
:10FAF800090B5346D0465A0DD7F8C03042EACB22FC
:10FB0800CDF8742583EAE372A2EBE3725310944AAA
:10FB18004FF0000983FB0223002A73F10004B4BFED
:10FB2800DFF864824FF0000812EB080A43EB090B78
:10FB38005346D0469A0D824B42EA8B22CDF878255F
:10FB4800D3F8B4204FF000095310864A7C4F83FB4A
:10FB58000223002A73F10004B4BFDFF834824FF0A7
:10FB6800000812EB080A43EB090B53461A0D3C9B9D
:10FB780042EA0B32CDF87C255A1042F2A173D046E6
:10FB880082FB0323002A73F10004B4BFDFF8F88175
:10FB98004FF0000812EB080A4FF0000943EB090B7D
:10FBA8005346D0469A0D664B42EA8B22CDF8802503
:10FBB800D3F888214FF0000953126B4ACDF86865D5
:10FBC80083FB0223002A73F10004B4BFDFF8C0816D
:10FBD8004FF0000812EB080A43EB090B5346D046D6
:10FBE8001A0D639B42EA0B32CDF884255A125F4BFB
:10FBF8004FF0000982FB0323002A73F10004B4BF0D
:10FC0800DFF884814FF0000812EB080A43EB090B78
:10FC18004FEA9A5242EA8B22CDF88825D7F8442138
:10FC2800534B521282FB0323002A73F10004B4BF22
:10FC3800DFF854814FF0000812EB080A4FF0000972
:10FC480043EB090B4FEA9A5242EA8B22CDF88C25F6
:10FC5800D7F850214FF000095312464A384F83FB1A
:10FC68000223002A73F10004B4BFDFF8E8804FF0E4
:10FC7800000812EB080A43EB090B4FEA5A5242EA12
:10FC8800CB22CDF89025D7F848213B4B521282FB66
:10FC98000323002A73F10004B4BFDFF8F4804FF0A7
:10FCA800000812EB080A4FF0000943EB090B4FEA72
:10FCB8001A5242EA0B32CDF89425D7F83C214FF07E
:10FCC800000953122D4A1E4F83FB0223002A73F1A9
:10FCD8000004B4BFDFF8B0804FF0000812EB080A48
:10FCE80043EB090B4FEA9A5242EA8B22CDF898254A
:10FCF800D7F84C21224B521282FB0323002A73F1BE
:10FD08000004B4BFDFF880804FF0000812EB080A47
:10FD18004FF0000943EB090B4FEA9A5242EA8B2253
:10FD2800CDF89C25D7F854214FF000095312154AF5
:10FD3800034F83FB0223002A73F100042AE000BF6B
:10FD4800F05D0020BC510020645F0020F05D0020C1
:10FD5800F5670500FFFF1F007F6A17007998F8FF15
:10FD6800575BEDFF0947FFFF8115BB0647036E1B75
:10FD7800E3A5D60CA913B407371A69FD2BF6E7F4E7
:10FD88001D5A468E2D32ADFFFFFF3F00FFFF0700D3
:10FD9800FFFF0F00B4BFDFF8C4834FF0000812EB79
:10FDA800080A43EB090B4FEA1A5242EA0B32CDF824
:10FDB800A025D7F86021DF4B521282FB0323002ACB
:10FDC80073F10004B4BFDFF8BC834FF0000812EBF6
:10FDD800080A4FF0000943EB090B4FEA9A5242EA2E
:10FDE8008B22CDF8A425D7F858214FF000095312DB
:10FDF800D14AD24F83FB0223002A73F10004B4BF17
:10FE0800DFF880834FF0000812EB080A43EB090B78
:10FE18004FEA9A5242EA8B22CDF8A825D7F840211A
:10FE2800C74B521282FB0323002A73F10004B4BFAC
:10FE3800DFF854834FF0000812EB080A4FF000096E
:10FE480043EB090B4FEA5A5242EACB22CDF8AC25D4
:10FE5800D7F85C214FF000095312BA4A83FB0223FA
:10FE6800002A73F10004B4BFDFF818834FF00008CC
:10FE780012EB080A43EB090BB04B4FEA9A52D3F83E
:10FE8800783142EA8B22CDF8B02583EAE372A2EBFF
:10FE9800E3725312AC4A4FF0000983FB0223002A95
:10FEA80073F10004B4BFDFF8DC824FF0000812EBF6
:10FEB800080A43EB090B4FEA9A5242EA8B22CDF823
:10FEC800B425002301330DF5AD6252F82320132B1E
:10FED8001644F7D1994A9D4B92F89A71801117F000
:10FEE800800F334418BF7F424FEA83034FEAA119BA
:10FEF80001464FEAAE1818BFFFB2C2F80031FCF74E
:10FF0800D8FD494682464846FCF7D3FD414682441F
:10FF18004046FCF7CEFD0121504478AAFCF71FFCAF
:10FF28007FB28B4A3F0587FB0289B8F1000F79F150
:10FF38000003B4BF8748002018EB00024FF000010F
:10FF48007E4849EB0103910C41EA8331824AD0F89B
:10FF5800DC30CDF8F81483FB0289B8F1000F79F191
:10FF68000003B4BF7D4A002212EB080A4FF00003D9
:10FF780043EB090B4FEA1A5242EA0B32CDF8FC2444
:10FF8800774BD0F8E0204FF0000982FB0323002ACA
:10FF980073F10000B4BFDFF8C4814FF0000812EB22
:10FFA800080A43EB090B4FEA1A52644B42EA0B3238
:10FFB800CDF80025D3F8E4204BF21D0382FB032380
:10FFC800002A73F10000B4BFDFF890814FF00008F9
:10FFD80012EB080A4FF0000943EB090B4FEA1A52DB
:10FFE800649B42EA0B32002BCDF804255D4AB8BF6A
:08FFF8005B4283FB0289514BBF
:020000040041B9
:100000004FEAD84242EA4932CDF80825D3F8002118
:10001000574B4FF0000982FB0323002A73F10000C5
:10002000B4BFDFF870814FF0000812EB080A43EB11
:10003000090B4FEADA4242EA4B32CDF80C25609BBD
:100040004C4A4FF0000983FB0223002A73F10000A1
:10005000B4BFDFF810814FF0000812EB080A43EB41
:10006000090B4FEA1A5242EA0B32CDF81025619B78
:10007000414A4FF0000983FB0223002A73F100007C
:10008000B4BFDFF8E0804FF0000812EB080A43EB42
:10009000090B4FEA1A5242EA0B32CDF81425629B43
:1000A000364A4FF0000983FB0223002A73F1000057
:1000B000B4BFDFF8B0804FF0000812EB080A43EB42
:1000C000090B4FEA1A52609B42EA0B32002BCDF823
:1000D00018252B4AB8BF5B4283FB02894FEA1852AE
:1000E00042EA0932CDF81C25619A264B002AB8BF96
:1000F000524282FB032352EA030007BF904699460F
:10010000DFF890804FF0000912EB080A43EB090B6F
:100110004FEADA42629B42EA4B32002BCDF82025AF
:10012000194AB8BF5B4283FB02894FEA185242EA80
:100130000932CDF82425789A53082DE05BB1F3F904
:10014000C9E53910F05D002099AAAFFFDB8A82F182
:100150005DDC2EF93DDBFE01AF250A00FFFF030049
:10016000151DDEFEFFFF0F00E3C76C01575B190092
:1001700093E90600E763FFFF17F4FFFF7155FEFFE9
:1001800053052D00575BD5FF61600800FFFF3F005E
:10019000FFFF1F00FFFF07009E4A83FB02239046DC
:1001A000120D42EA0332CDF82825002301330DF564
:1001B0009F6252F823200C2B1144F7D1964B4FF03D
:1001C0000009D3F8A8205310944A83FB02ABBAF17C
:1001D000000F7BF10003B4BFDFF854824FF000083A
:1001E0001AEB08024BEB0903970D47EA83273C9B68
:1001F0004FF000099A108A4B82FB0323002A73F107
:100200000000B4BFDFF828824FF0000812EB080AA4
:1002100043EB090B834B4FEA9A5242EA8B220B4481
:1002200017447D489A12A7F5A017B2F57F3FC0F892
:10023000047101DBFF2303E0002AD4BF00231B1558
:1002400080F8A2317848794930441122FCF797FBB5
:10025000714BC3F80801704991F8A121D1F804311C
:10026000D1F80811002A18BF0B46B3F1C87FB4BFFC
:1002700023EAE3734FF0C8730C999B145FFA83FC75
:1002800041B3002B00F0C186002A40F0BD866249D0
:10029000659A91F8963112786BB15BB22AB1002B56
:1002A000ACBF0923082300F0B0BE002BACBF08236D
:1002B000092300F0AABE91F8A5312AB1002B14BF82
:1002C0000423032300F0A1BE002B14BF0323042347
:1002D00000F09BBE329B002B00F0AC800C9B4E4983
:1002E00091F8AD21002A4FD0D1F8E440CA6D84EADC
:1002F000E4706243002AD4BF0022012281F8A321C6
:10030000389AA0EBE47012782AB1012A40F23B122D
:1003100098BF932200E0CD2200F57A70C1103E48CC
:100320004FF00009D0F8DC00C01081FB000100286C
:1003300071F10004B4BF4FF0FF084FF0000818EB54
:10034000000649EB0107300A40EA0760801080FB95
:100350000201002871F10002B8BF40F6FF762E4A74
:10036000A8BF002610EB06084FF0000741EB070975
:100370004FEA1830D2F8E01040EA09508142D4BF69
:100380000021012182F8A4110C9A002A53D0224A9C
:1003900092F8A401114620B192F8A60108B10621F5
:1003A0000EE091F8A6111C4A31B192F8A31109B1DF
:1003B000092105E0042103E092F8A711B1B107215A
:1003C00082F89C11144A92F89A2151B20029CCBFAC
:1003D00000210121002915BF212624261E202B20C3
:1003E000022B05D0032B08BF304602E00221E7E7CD
:1003F0003720160644BF5242D2B252B29042064A49
:1004000001DB002103E009B1022100E0012182F8B3
:10041000A81110E0CF661200F05D0020DD0C1F0077
:10042000E17A14007E1DDBF53DDB0E013333030062
:10043000FFFF3F000C9BAF4EAF49306B47F6FF7A92
:100440008842B8BF0846776B5045A8BF50468F42D8
:10045000B8BF0F46B66B5745BE46A8BFD646B14299
:10046000B8BF31465145A8BF51468146F34688463C
:10047000424292B290B2CEF100070FFA80FABFB2B8
:100480001FFA87FEBAF1000FC1F10006B6B2B8BF7D
:100490001FFA89F00FFA8EF9B1B2B9F1000FB8BFA7
:1004A0001FFA8BFE0FFA81FB0FFA8EFEBBF1000FD5
:1004B00000B2B8BF1FFA88F18645B8BF864608B2B9
:1004C0008645B8BF86460A990A980B70894BBEF1DB
:1004D000030F93F89C11D8BF0022417093F8A81124
:1004E000C8BFD2B2817093F89A11C1BFFFB2F6B201
:1004F000CAF3072AC9F30729CFBFCBF3072B174647
:1005000016469246DCBF914693460C0654BF0A98A5
:100510004942C1700A9981F804C093F8A1311BB116
:10052000744B93F8A23100E00A994B71714B0A9811
:1005300093F89811817193F897110272C1710D9A15
:10054000179986726D4E80F80BA080F80DB0477237
:1005500080F80C900A441FFA82FAD6F86012D3F899
:10056000A0209869521AC3F8A420D6F86422D96949
:10057000C2EB000BD6F868228A1A196AD6F86C32D8
:100580001792CB1A1C99329396F80E2C334699B1D8
:1005900022B9C6F87C23012286F80E2C099A0AB1EA
:1005A000002206E0D3F84823D3F87C339A4208DBD4
:1005B000524BC3F87C2304E01AB19DF8703086F8E2
:1005C0000E3C4E4E4B4FD6F8E43201461C93FCF7DE
:1005D0004CFAF8690146FCF748FA38680146FCF71E
:1005E00044FA804678680146FCF73FFA8044B868D0
:1005F0000146FCF73AFA0121404477AAFCF7B3F828
:100600003F4BB6F8BC171A88B6F8BE07511A89B224
:1006100038915988B6F8C077081A80B23C9098880B
:10062000B6F8C8E7C71BBCB2DF886094CEEB0707FB
:10063000BCB2B6F8CAE71F896194CEEB0707BCB21B
:100640005B89B6F8CC776294DB1B9BB26393D6F8D8
:100650007C326493D6F880326593D6F88432669300
:10066000D6F888326793D6F88C326893D6F89032F1
:100670006993D6F894326A93D6F898326B93D6F889
:100680009C326C9396F8FD3B6D9396F8FE3B6E930F
:1006900096F8FF3B6F9396F8003C709396F8013CF8
:1006A000719396F8023C729396F8033C7393D6F8D4
:1006B0003435002B03DBC19E002E04DD2BB9C19B1A
:1006C000DB43DB0F02E0012300E00023BF9E13B1F8
:1006D000084BC3F86C61094BD3F83835002B03DBAA
:1006E000C29E002E04DD6BB9C29BDB43DB0F0AE028
:1006F000012308E0F05D00200080FFFFBC510020D6
:10070000D45D00200023BE9E13B1B24BC3F86861D4
:10071000DFF8C4C2C19BDCF83CE5DCF84475C29E3E
:10072000DCF84885BEF1000FA3EB0707C8EB06080D
:1007300004DB002F04DDBEF1000F07D1002F05DB25
:10074000DFF890E2CEF86431012300E00023DFF807
:1007500088E2DEF84CC5BCF1000F05DBB8F1000FF4
:1007600005DDBCF1000F09D1B8F1000F06DBDFF8A1
:1007700064C2CCF8706163B9012300E01BB9DEF8F4
:10078000846153B901E04FF0FF36934BD3F8889161
:1007900005E04FF0FF36B14601E04FF0FF39DFF8DA
:1007A00038E2DEF85035002B04DB109C002C04DD11
:1007B0002BB902E0109B002B01DB002302E0DEF8E6
:1007C0008C310133CEF88C3115B9DEF8543500E0A8
:1007D0000023119C9C42A8BF1C460D941DB97E4B62
:1007E000D3F8583500E000231B9C9C42A8BF1C4650
:1007F00009941DB9784BD3F85C3500E000230F9CB9
:10080000A342A8BF23460F931DB9734BD3F860359D
:1008100000E00023189C9C42A8BF1C4611940DB117
:10082000002302E06C4BD3F85C347F937F9B749C75
:10083000A34228BF23460A930DB1002302E0664B72
:10084000D3F860347F937F9C759B9C4228BF1C46E5
:100850000C9B18948BB15F4B93F8A1416CB9D3F802
:100860000041C3F8F44093F998412405C3F8F840D7
:1008700093F997412405C3F8FC40584B03F17404E5
:1008800053F8045FA34243F8045CF9D1524B0E9C29
:10089000B3F802E7BAF1960FC3F8D84484BF002436
:1008A000A3F8D447A3F8FCE64A4CB3F804E7A3F84E
:1008B0000417D3F8C0122568A3F80227C3F8B412AE
:1008C000D3F8A421D3F8C412C3F89451C3F8A021DB
:1008D0006568D3F8A821C3F8B812D3F8C812C3F8D2
:1008E0009851A3F8FEE6C3F8A421B3F806E7A2697D
:1008F000C3F8BC12A568D3F8CC12C3F8A82198BFDE
:10090000A3F8D4A7C3F89C51A3F800E7A3F80607FF
:10091000C3F8C012D3F8D012DFF8BCC0C3F8C412B9
:10092000D3F8D412C3F8C812D3F8D812C3F8CC1233
:10093000D3F8DC12C3F8D012D3F8E012C3F8D41203
:10094000E168C3F8D8122169C3F8DC126169C3F801
:10095000E0122999C3F8DC143E99C3F8E0143F99DA
:10096000C3F8E4144099C3F8E814D3F8B811C3F8F5
:10097000AC11D3F8BC11C3F8B011D3F8C011C3F84F
:10098000B411D3F8C411C3F8B811D3F8C811C3F81F
:10099000BC11D3F8CC11C3F8C011D3F8D011C3F8EF
:1009A000D021E269C3F8C411D3F8D411C3F8D4211B
:1009B000226AC3F8C811D3F8D811C3F8D821259AF0
:1009C000C3F8CC11C3F88023319B4BB1BDF8F43090
:1009D00008E000BFF05D0020BC5100202056002040
:1009E000BDF8C4302F9AACF8D637BD4B1A6003F56A
:1009F000C76103F2146252F8040F8A4242F8040CF1
:100A0000F9D1B84AD2F8A410C3F83816B64B03F19E
:100A1000240153F8040F8B4243F8040CF9D1B04B76
:100A2000D2F8A04003F5D261C3F8604603F26462D5
:100A300052F8040F8A4242F8040CF9D1A94AD2F8BC
:100A40009800C3F89006A94B03F12C0153F8045FFA
:100A50008B4243F8045CF9D1A14BD2F89C1003F50A
:100A6000DE65C3F8C01603F2C46252F804EFAA426E
:100A700042F804ECF9D11E9AC3F8F046C3F8DC2121
:100A80001F9AC3F80402C3F8E021209AC3F81C128D
:100A9000C3F8E421219AC3F8E821229AC3F8EC2193
:100AA000239AC3F8F021649AC3F8F421349AC3F866
:100AB000F821359AC3F8FC21369AC3F800222A9A05
:100AC000C3F808222B9AC3F80C222C9AC3F81022E0
:100AD0002D9AC3F814222E9AC3F81822844B03F1DE
:100AE0001C0253F8041F934243F8041CF9D17C4BB9
:100AF000249A03F51771C3F83C2203F5107252F8DB
:100B0000040F8A4242F8040CF9D1679AC3F85C22B8
:100B10009DF8082183F8042CBDF80421A3F8D827F8
:100B2000744AA2F1CC03D3F890130C33C3F87813B2
:100B3000D3F88813C3F87C13D3F88C13C3F880134D
:100B40009342F0D1664B199AC3F850241A9AC3F80D
:100B50005424159AC3F858240E9AC3F8EC249DF82F
:100B6000102183F8E02B9DF8142183F8E12B9DF8E8
:100B7000182183F8E22B9DF81C2183F8E32B9DF8C4
:100B8000202183F8E42B9DF8242183F8E52B9DF8A0
:100B9000282183F8E62B9DF82C2183F8E72B9DF87C
:100BA000302183F8E82B9DF8342183F8E92B9DF858
:100BB000382183F8EA2B9DF83C2183F8EB2B9DF834
:100BC000402183F8EC2B9DF8442183F8ED2B9DF810
:100BD000B82183F8EE2B9DF84C2183F8EF2B9DF87C
:100BE000502183F8F02B9DF8542183F8F12B9DF8C8
:100BF000582183F8F22B9DF85C2183F8F32B9DF8A4
:100C0000602183F8F42B9DF8642183F8F52B9DF87F
:100C1000682183F8F62B9DF86C2183F8F72B9DF85B
:100C2000702183F8F82B9DF8742183F8F92B9DF837
:100C3000782183F8FA2B9DF87C2183F8FB2B9DF813
:100C4000E42083F8FC2B93F8062C83F8052C93F80A
:100C5000072C83F8062C93F8082C83F8072C9DF8B2
:100C6000DC2083F8082C03F15402B3F80E17063386
:100C7000A3F80217B3F80A17A3F80417B3F80C1770
:100C8000A3F806179342F0D1154BBDF8E010A3F876
:100C90005C17BDF8F010A3F85E17BDF88011A3F83B
:100CA0006017B3F868170633A3F85C17B3F8641736
:100CB000A3F85E17B3F86617A3F860179342F0D154
:100CC000074BBDF884210C49A3F8B627BDF888214D
:100CD000A3F8B827BDF88C21A3F8BA2700230DE0AC
:100CE000BC510020F05D0020F85700205058002033
:100CF000DC53002088520020285E0020D2AA0B98E6
:100D000052F823204260DAAA52F823204262E2AA73
:100D100052F823204264EAAA52F823204266F2AA3B
:100D200052F82320C0F88420FAAA52F82320C0F8F1
:100D3000A4200DF5816252F82320C0F8C4200DF5DF
:100D4000856252F82320C0F8E4200DF5896252F83C
:100D50002320C0F804210DF58D6252F82320C0F83D
:100D600024210DF5916252F823200133C0F844216B
:100D700051F8042F082BC0F86421024602F1040246
:100D80000B92BBD1C44C9DF80C3184F8093C94F80B
:100D90000D3C43B1C1481C99FBF722FED4F8A032A8
:100DA0001844C4F8A0021D9BBD4AC4F8F034109B3F
:100DB000C4F8F4340E9BC4F8F834BD9BC4F8FC347A
:100DC000BE9BC4F80035BF9BC4F804350E9BC4F825
:100DD0000835149BC4F80C35139BC4F81035279BB9
:100DE000C4F814353B9BC4F81835309BC4F81C3547
:100DF000129BC4F82035169BC4F82435269BC4F8F2
:100E000028353A9BC4F82C35289BC4F83035D4F8E3
:100E10007032D2F8A000C4F86432D4F87432C4F846
:100E20006002C4F86832D4F87832C4F86C3293693E
:100E3000C4F87032D369C4F87432136AC4F87832D3
:100E4000984B03F1300253F8041F934243F8041CFB
:100E5000F9D1179A8BEAEB74002AB8BF52425110AD
:100E6000A4EBEB7401EB640232998B4B0029B8BF01
:100E7000494202EB6102C3F8782303F54B7103F595
:100E8000397252F8044F8A4242F8044CF9D1779AE9
:100E90000136C3F82C23B3F8C227A3F8BC27B3F854
:100EA000C427A3F8BE27B3F8C627A3F8C0277E4AF5
:100EB0001188A3F8C2175188A3F8C4179188A3F822
:100EC000C617B3F8CE17A3F8C817B3F8D017A3F80E
:100ED000CA17B3F8D217A3F8CC17D188A3F8CE1746
:100EE00011895289A3F8D017A3F8D227669AC3F8BC
:100EF0007C22339AC3F88022659AC3F884226A9AC6
:100F0000C3F888226C9AC199C3F88C22689AC3F8F6
:100F10009802C3F89022699AC098C3F894226B9AF9
:100F2000C3F83415C3F89C229DF8CC21C3F83C7556
:100F300083F8FD2B9DF8B421C3F8400583F8FE2B00
:100F40009DF84821C3F8441583F8FF2B9DF8BC2178
:100F5000C3F84C8583F8002C9DF8C02183F8012C40
:100F60009DF8C42183F8022C9DF8C82183F8032C36
:100F7000C29AC3F83825C3F8482509F10102C3F81D
:100F80008461C3F88821109AC3F850250D9AC3F8DC
:100F90005425099AC3F858250F9AC3F85C25119A6D
:100FA000C3F860250A9AC3F85C24189AC3F8602431
:100FB0000DF6BC0DBDE8F08F03EAE3733093FEF746
:100FC00074BC099B002B7EF48AACBE9B002BB8BF7F
:100FD0005B421193FEF792BC00297EF49EACFEF7B3
:100FE000A0BC11991691FEF79CBCBF9B03EAE3736A
:100FF0002893FEF7FBBC002D3EF4EEACBF9B03EA4A
:10100000E3732893FEF7F6BC0223329A002A7FF49A
:1010100066A9FFF7BCB94FF0FF35186DD3F88060B3
:10102000D3F8B070FDF7FDB96420FDF73CBA4FF07E
:10103000FF33FDF73FBA0029BDF6ECA94FF0FF35AD
:10104000FDF7EFB9099B23B1189B14930123FEF719
:10105000DABBC19C189B002CB8BF64420F94149358
:101060005DE0099B1BB1189B1493FEF7CBBBC19CA1
:10107000189B002CB8BF64420F941493FEF7CFBBAB
:10108000099921B10F99C2F850110A4600E00F9A50
:101090001392FEF7D9BB00BFBC510020CDCCCCCC05
:1010A000F05D002004550020D45D0020099B002B3A
:1010B00035D00F9B0125C2F85031C29B23EAE37261
:1010C00027920F9A1392FEF7C9BB099B002B7EF45F
:1010D00004ACBE9B002BB8BF5B4211931B9B1293C9
:1010E000FEF70CBC099B1BB3154B1199C3F860119B
:1010F000BF9B169123EAE3732693FEF71BBC41F6D0
:101100002210FCF7BBBB44F66630FCF7B7BB4BF2D2
:101110009A40FCF7B3BB4EF2DE60FCF7AFBBC29B5C
:10112000012523EAE37227920F9A1392FEF79CBBE4
:10113000119B1693BF9B23EAE3732693FEF7FEBB36
:10114000F05D0020244B4FF00052C3F864254FF0AF
:101150006042C3F8682503F2DE7100221F4830F8B0
:101160001200013221F8020FB2F5807FA1F80002CF
:10117000F4D14FF400121A49C3F8A422C3F8A822EC
:10118000C3F8AC22C3F8B022164A1A20C2F8C41021
:10119000C2F8C810C2F8CC10C2F8D010C2F8E400EF
:1011A000C2F8DC00C2F8E0004FF00052C3F8DC24C3
:1011B0004FF000620021C3F880230122A3F8141C21
:1011C000A3F8101CC3F8E014C3F8E414C3F8E8143F
:1011D0001A6083F8042C7047BC51002094C341006E
:1011E00033330300F05D002010B5002302680B606C
:1011F0004FF0804393424FEA530301D95200F9E77D
:10120000520808684BB11C18A24222BF00EB4300F1
:10121000121B086052005B08F3E74000086010BD35
:10122000036853B1436843B1836833B1044B1A6810
:101230001AB901220A701A60704700230B707047B8
:10124000383500202DE9F84305460C4698460768D6
:101250000E6840684968A36880FB0101C6FB07016E
:101260009146AA68C3FB020142460AF037F8C9F862
:10127000000028696168EF6880FB010126686A69DF
:10128000C6FB0701A368C3FB020142460AF026F829
:10129000C9F80400EB696068AF6983FB0001266848
:1012A000A268C6FB07012D6AC2FB050142460AF08F
:1012B00015F8C9F80800BDE8F88310B500230268E6
:1012C0000B604FF0804393424FEA530301D9520021
:1012D000F9E7520808684BB11C18A24222BF00EB84
:1012E0004300121B086052005B08F3E740000860EF
:1012F00010BD0000014B0360704700BF050000A552
:1013000008B530B104F0D7FABDE80840022005F076
:10131000C4BC022005F0CDFCBDE8084004F0C8BA0A
:1013200008B50020FFF7ECFF0A200AF061FFBDE8D6
:1013300008400120FFF7E4BF08B50020FFF7E0FFF9
:10134000014B00221A7008BD3C35002008B500F0A2
:101350005FFA034B00201870BDE80840FFF7D0BFCC
:101360003C35002013B53C4C237800283AD1013B92
:10137000092B6FD8DFE803F0050E1D242D6E6E6C6F
:101380006E34082007F01CFEFFF7D6FF002007F0A0
:101390002DFA5FE0314B18689B8800900820ADF86B
:1013A000043007F00DFEFFF7C7FF684607F0F8F9B5
:1013B00050E0082007F004FEFFF7BEFF002005E024
:1013C000082007F0FDFD00232370012007F032FA0A
:1013D00040E0082007F0F4FDFFF7AEFF00200FE02B
:1013E000002017E0043B082B34D8DFE803F00C059D
:1013F0001633313312331F00082007F0E1FD0120BE
:1014000007F006FA26E0082007F0DAFD0020207039
:10141000DCE7012000F0C4FE1CE04FF41640002180
:10142000012204F087F90723237013E04FF41640DC
:101430000021012204F07EF90D23237000F0ACFAA4
:1014400008B109F0E1F8FFF777FF00F0E1F901E0FA
:1014500000F05CFE02B010BD3C35002054D64100C7
:1014600070470000037810B50446002B6BD002F0E3
:1014700069FC63780F2B66D8DFE803F00865652CFC
:1014800032346539654365516565655E2E4B1B7861
:10149000013B0B2B57D8DFE803F006081156131752
:1014A000565619560F17082000E0062000210A465C
:1014B000BDE8104000F0C6B90E20F7E70A20F5E7B6
:1014C000012022490422F3E70C20EFE7BDE8104099
:1014D00000F03ABE6068A178BDE8104000F040BE60
:1014E000012000E00020BDE8104000F017BE0820F9
:1014F00007F066FDFFF720FF6068BDE8104007F0C9
:101500004FB9082007F05CFDFFF716FF6368BDE8E0
:1015100010401878003018BF012007F067B9FFF7B6
:101520000BFF094B04221A7000210A200A46BDE86D
:1015300010400B4600F078B9082007F041FDBDE8E7
:101540001040FFF7F9BE10BD3C3500205AD64100CF
:1015500007B5124B1B78013B042B19D8DFE803F0C9
:10156000030715151100002007F040F910E00C4B9F
:1015700018689B8800906846ADF8043007F010F9B1
:1015800006E0002007F044F902E0002007F052F9DD
:10159000FFF7D2FE03B05DF804FB00BF3C3500202E
:1015A00054D6410010B10120FFF7AABEFFF7C4BE18
:1015B000074B10B5082204461A700AF03BFC421C87
:1015C0002146BDE810401020D2B200F03BB900BF68
:1015D0003C35002003460A460349092008700120D3
:1015E000194600F02FB900BF3C35002008B5FFF7C1
:1015F00097FE024B09221A7008BD00BF3C3500203F
:1016000038B505460C46064B0A221A7002F09AFBC2
:1016100029462246BDE83840022000F013B900BF39
:101620003C35002008B5FFF77BFE054B01221A7000
:10163000082040F2DC51BDE8084007F095BC00BF2F
:101640003C35002008B5FFF76BFE024B06221A70EE
:1016500008BD00BF3C35002008B5FFF761FE024B16
:101660000C221A7008BD00BF3C35002008B508F0F8
:10167000BFFF18B9BDE80840FFF7EEBF08BD000086
:1016800008B5FFF74DFE054B02221A70082040F204
:10169000DC51BDE8084007F067BC00BF3C350020C6
:1016A00008B5FFF73DFE054B05221A70082040F2F1
:1016B000DC51BDE8084007F057BC00BF3C350020B6
:1016C00008B5FFF72DFE054B03221A70082040F2E3
:1016D000DC51BDE8084007F047BC00BF3C350020A6
:1016E00000B50E4B89B01B78072B0FD1202168461F
:1016F00003F0ACFF6946C0B204F07EF904F0B4F820
:1017000040B10120002107F0C3FB03E00D2B01D005
:1017100000F09CF809B05DF804FB00BF3C350020E8
:10172000034B0022A3F80621A3F80E221A7070477B
:101730003E35002037B5044612488DF80440006855
:1017400002AB00908DF8052053F8080D0E4C9B88D5
:101750001546A4F805300623C4F80100A4F80631A4
:101760003AB1E01D0AF066F9B4F806212A44A4F85B
:1017700006210648B4F8061103B0BDE8304004F075
:1017800021B800BF5FD641003E3500203F35002024
:101790000720C82107F0E8BBF7B51B4B00251868E8
:1017A000019004F061F8064656B34DBB174C013E5C
:1017B000B4F80E7204F01EF8B4F80E322744032B6E
:1017C00087F80801B6B20ED8E21892F8081102AAFA
:1017D0001A4412F8042C914206BF5A1CA4F80E2297
:1017E000A4F80E52E0E75A1C93B2052BA4F80E326F
:1017F000DAD994F80D51063BEB1A5D425D41D3E70F
:10180000284603B0F0BD00BF65D641003E3500203C
:1018100008B504480121002203F08CFFBDE8084010
:10182000FFF77EBF0018150010B51C46FFF782FFBA
:10183000FFF7AEFF024A012382F81042137010BD79
:101840003E3500200323FFF7EFBF00007FB504F013
:101850000BF8002853D02E4C23782546012B2DD091
:1018600002D3022B06D04AE002232370FFF7F8FDD3
:10187000FFF78EFFFFF790FF002840D0072007F00A
:101880009FFB012404A901F8094D95F80C0122469B
:10189000FFF750FF95F80C3100268DF809301D4BED
:1018A00002A8039395F80D312E708DF808408DF83D
:1018B0000A30FFF7D7FDA5F80E6220E0FFF76CFFB6
:1018C000E8B1072007F07CFB94F80E01012812D044
:1018D00094F8100278B10023601CB4F80611A4F843
:1018E0000E3203F06FFFFFF753FF94F81032013B05
:1018F00084F8103203E0FFF735FDFFF711FF03F026
:10190000B3FF18B10120002107F0C2FA04B070BD86
:101910003E3500204C3600201FB51E4C2378012B8D
:1019200002D0022B18D032E094F8100278B10023D4
:10193000601CB4F80611A4F80E3203F043FFFFF761
:1019400027FF94F81032013B84F810321FE0FFF7B4
:1019500009FDFFF7E5FE1AE000238DF80730B4F823
:101960000E32052B06D994F80C010DF10701012266
:10197000FFF7E0FEFFF7D4FE002302A88DF8083041
:101980008DF8093003938DF80A30FFF76BFD04B032
:1019900010BD00BF3E3500202DE9F047FAB005AD7F
:1019A0002A469B4B1BAF03F1240E1E467446186853
:1019B000596803C29868106003F10C023B46106836
:1019C0005168083203C372451F46F7D12068616829
:1019D00008AB03C3A0680BAA18608E4B1C4618689E
:1019E000596803F1200E03C29868106054F80C0F78
:1019F0000EAA616803C2A06817AC106003F1180258
:101A0000274610685168083203C772453C46F7D133
:101A10001068918892793860B98018685968BA71ED
:101A200011AA03C298687C4B106003F1180721AA21
:101A3000144618685968083303C4BB422246F7D1DC
:101A400019889B780DF1040AA37053462180734CCA
:101A50000DF1A008206861684FF0600903C34A4691
:101A600004F10801404609F0E5FF682740ABE119A1
:101A70003A46184609F0DEFF0DF10C0E7246034699
:101A80005D951825ADF87A511BAD54F8D00F5F95D0
:101A900008AD61950BAD616863950EAD6595C82580
:101AA00003C2ADF89A510C210F2500240122022017
:101AB0004FF0320CADF87211ADF88211ADF88A1109
:101AC000ADF89211ADF8A251ADF8AA1117AD11A958
:101AD0008DF86801ADF86AC18DF878218DF88821FC
:101AE0008DF898018DF8A0216B918DF8B001ADF8BB
:101AF000B2C15B948DF870418DF880418DF89041B2
:101B0000679469958DF8A8416D94ADF8DA7114AFBA
:101B100077933B461B21ADF8BA1121A96F918DF83F
:101B2000C80108214FF4FA70ADF8C211ADF8CA012E
:101B3000ADF8E211306871688DF8B82103C3B06860
:101B40008DF8C041CDF8C4A173948DF8D041ADF8A3
:101B5000D291CDF8D4818DF8D8218DF8E041CDF81F
:101B6000E4E1186003F094FE2D4E03F07DFE70B1A9
:101B700003F040FE3B5D834203D10134E4B2012512
:101B800009E0013E14BF01250025002405E0013EC7
:101B900014BF012500250B2C01D8002DE5D15AAC2E
:101BA000A1464FF000087DB319F83830022B03D15D
:101BB00060880AF01DFB20E023B96068618803F0AB
:101BC00001FE1AE0164F00266388B34215D9A5B16D
:101BD00003F04AFE48B103F00DFE63689B5D83424B
:101BE00008D10136B6B20E4FEEE7013F14BF012512
:101BF0000025E9E70A4F0025E6E708F10108B8F1FA
:101C0000100F04F10804CED128467AB0BDE8F08761
:101C100069D6410099D64100C0D64100DBD64100CB
:101C2000FFFF0F0010B5084B5524AA2218715971F7
:101C30001C705A709C70DA7006311846BDE810406E
:101C4000C9B2FFF7DDBC00BF683700204FF48060E9
:101C5000002107F01DB9000073B50546184C00239C
:101C600029460D22204623610AF05CF929460C2200
:101C700014480AF057F928460AF0DCF8063083B217
:101C80000B2B114E04D80022F25401339BB2F7E71C
:101C9000284601A907F012FC00B901900198019BA8
:101CA0001021C6F8120004206361FFF7BBFF074B49
:101CB00006221A70FFF7CAFF08F046F902B070BD9D
:101CC000503700206E37002068370020673800202A
:101CD00030B585B06B46144A1068516803C311894A
:101CE000927A19809A70114B00211D6801201DF80D
:101CF0000130EA18527802F00302022A14BF1A4691
:101D0000A3F120020A4BCB5C0131EC18647804F09B
:101D10000304022C08BF203B9A4218BF00200B2965
:101D2000E5D105B030BD00BFB3D74100443000203D
:101D30005037002070B506468EB00D46144608F0A8
:101D400003F90D2E00F2F780DFE816F00E00F50023
:101D50001C00F5003A005600690081009600A300BF
:101D6000BF00D600F500EF00002D40F0E48007F042
:101D70008BFB0EAB23F8320D1A88724B0120DA80F0
:101D80000221D6E0042D40F0D68007A903AA02ABB9
:101D9000207807F08AFB6B4A07AB03CBC2F806003A
:101DA0001868BDF81030C2F80E000398C2F80A1087
:101DB000C2F812000298D382906116210320B8E085
:101DC000102D40F0B880604B20681A46616803C24D
:101DD000A068106000201873A27B617B120442EAA5
:101DE0000122217B0A43E17B186142EA0162184625
:101DF0005A6107F033FC9EE0002D00F09C805248B1
:101E00002946224607F098FBFFF762FF002800F002
:101E10009280204608F008FC08F012FA8BE0042DAE
:101E200040F0898007AD2078294603AA02AB07F06D
:101E30003CFB00287FD095E807000AAB83E8070049
:101E4000002218468DF8342007F0DAF973E0042DEB
:101E500071D107AD2078294603AA02AB07F025FB14
:101E6000002868D095E807000AAB83E80700002245
:101E70008DF83420184609E0002D5CD10AA83349BA
:101E80000D220AF04FF88DF834500AA8FFF7E4FE4F
:101E900056E0062D4FD1237805A803F5FA63ADF877
:101EA000163063788DF81530A3788DF81430E37808
:101EB0008DF81A3023798DF8193063798DF8183040
:101EC000234B1B685B6F984735E0062D33D1237891
:101ED000A22B30D16378732B2DD1A3788F2B2AD1ED
:101EE000E378B42B27D12379762B24D16379902BF7
:101EF00021D107F0B3FD1EE0062D1CD12378862BDF
:101F000019D16378A42B16D1A378792B13D1E37858
:101F1000F62B10D12379832B0DD16379422B0AD173
:101F20000A20192107F020F805E0064B01219971DC
:101F30000E20FFF777FE074B05221A70FFF786FE8B
:101F40000EB070BD6837002050370020B3D7410075
:101F50002C72002067380020024B00221A70FFF715
:101F6000F5B900BF67380020F0B53E4C89B0237842
:101F7000092B71D8DFE803F0740508273174743A2F
:101F80007064FFF733FB6BE00022374B0B2A1344DE
:101F900093F83630B3FA83F34FEA531303D0013288
:101FA000002BF2D000E033B168463049304A314B63
:101FB00008F008FE03E068462D4909F0DDFE68469A
:101FC000FFF7F6FA4CE0092042F2283106F0CCFF88
:101FD00029480421FFF7FEFA42E001F097F80523B3
:101FE0002370FFF733FE07F0B7FF39E0234D2E696A
:101FF0006B699E4222D29E1BF12E28BFF126FFF76D
:1020000067FE30B928462969F1221D4B07F06EFAA8
:102010000BE01C4F4821384603F006FE3946A7F86E
:1020200048004A22164809F005FD2B690520334473
:10203000F1B22B61FFF7F6FD06230EE005230CE05D
:102040000020FFF7AFFA00232370FFF7FFFD01F038
:10205000BBF800F07DFD03E000232370FFF7F6FDE1
:1020600009B0F0BD6738002000FC4100BFD7410037
:10207000C5D7410036FC41005AD6410050370020F8
:102080006E3700203872002038B50E4C23783BB9EB
:1020900007F05EFF01232370BDE83840FFF7D6BD8F
:1020A000023B012B0CD800200025FFF77BFA25709E
:1020B000FFF7CCFD2946BDE83840012007F03EBFC0
:1020C00038BD00BF6738002010B5074C2378032BBC
:1020D00008D10020FFF766FA00232370BDE8104006
:1020E000FFF7B4BD10BD00BF6738002008B508F089
:1020F0004DFABDE8084007F0FFBC0000024B18781D
:10210000C31E58425841704767380020024B0322D3
:102110001A70FFF79BBD00BF6738002008B530B9C3
:102120000A2006F06FFF60B90922064B04E0054B58
:102130001A78032A05D104221A70BDE80840FFF777
:1021400085BD08BD67380020044B1A78012A03D1E9
:1021500002221A70FFF77ABD704700BF673800206F
:1021600038B50D4B05461B780C46052B13D10529B8
:1021700011D90A49042209F02BFC60B96979063C9F
:10218000A14208D1287909B90A4600E0AA1DBDE894
:102190003840FFF7CFBD38BD673800207ADD4100F9
:1021A000054B08B9052203E01A78062A03D1072255
:1021B0001A70FFF74BBD704767380020024B187844
:1021C000B0FA80F0400970476738002038B5194BE5
:1021D0000D461970044610B101280CD038BD0220FC
:1021E00021B3012107F030FE2046214607F02CFEE6
:1021F000012021461AE0A1B1FFF780FF054628B96A
:10220000214607F021FE0220294605E00020214654
:1022100007F01AFE2146022007F016FE01200021D9
:1022200004E0084607F010FE29460220BDE83840C9
:1022300007F00ABE6C38002038B52F4C2F4B22789F
:10224000AABB1B7843BBFFF7B9FF30B9012107F0E8
:10225000FBFD0220012107F0F7FD08F033FB042805
:102260000CBF00200220012107F0EEFD00F066FF08
:1022700018B10120014607F0E7FD214B1B785BB147
:102280000020012107F0E0FD0120014607F0DCFD00
:102290000220012107F0D8FD1A4B0F201B780BB943
:1022A000192100E00A2106F05FFE012322E01D78DB
:1022B0005DB90220294607F0C7FD2846294607F0E8
:1022C000C3FD0120294607F0BFFD0F4B1B7863B902
:1022D0000C4D0F202B780BB9C82108E00A2106F01D
:1022E00043FE2B78013B2B7003E00F20192106F0F1
:1022F0003BFE0023237038BD773800206C38002067
:1023000068380020733800207138002070470000C2
:1023100038B5134D02202B7833B9012107F094FD15
:1023200001232B70192205E0002107F08DFD002309
:102330002B704B220B4B1C78013CE4B21C7044B157
:10234000094B01211970094B1B881344084A13805B
:1023500038BD0220214607F077FD2C7038BD00BF44
:102360007738002072380020703800206A3800204A
:1023700074380020034B042219781A7009B9FFF74A
:10238000C7BF70477238002008B508F09BFA0146B5
:1023900038B907F059FDBDE808400120014607F0B3
:1023A00053BD0020012107F04FFD054B01221A709B
:1023B000044B054A1B8803F6B833138008BD00BFE1
:1023C000763800206A3800206E380020104A114903
:1023D0001388087801339BB210B51380144638B1C6
:1023E0000D4A12889A4203D100230B70FFF7CCFFED
:1023F0000A4B1A7852B10A4A21881288914205D1B3
:10240000BDE8104000221A70FFF782BF10BD00BF68
:102410006A380020763800206E380020703800209E
:102420007438002008B5084B1A7862B901220B20D5
:1024300064211A7006F098FD0F2006F0C1FDBDE87A
:102440000840FFF7F9BE08BD7138002008B5054BFC
:1024500000220F201A7006F0B3FDBDE80840FFF718
:10246000EBBE00BF7138002008B50020012107F045
:10247000EBFCBDE808400220012107F0E5BC0000AC
:10248000014B01221A70704768380020014B072267
:102490001A707047733800202DE9F04F83461C46B0
:1024A00095B0019102920025DFF858A14D492A46C6
:1024B0004D4808F087FBDFF85091DAF80020D9F892
:1024C0000000D66848490122B047484AC0B210709F
:1024D0005646C84617460392F0B907F06DF8DAF889
:1024E0000010D9F800008969884707F073F8039A4B
:1024F00001351278ABB262B9B5F5FA7FD4D105A82F
:1025000006F050FF3A493B4A05AB374808F05AFB02
:1025100002E0B3F5FA7FF2D055238DF81430002590
:10252000022359460DF117008DF815308DF816501D
:1025300009F022FC01990DF1370009F01DFC029B06
:102540006288CDF84330A379622A8DF847306379E9
:1025500088BF30328DF8483023798DF84C208DF8C3
:10256000493023788DF84A3063788DF84B302B460C
:10257000214D2B706B70AB70EB7007F01DF833685A
:102580001949DB680B22D8F800009847387007F02B
:1025900021F8336802210A461B6C134898473368B8
:1025A00005A9D3F828C0D8F800003922134BE0471A
:1025B000336838709E6A2946D8F8000004220F4B11
:1025C000B047627923793C2101FB0233A2794FF4B1
:1025D000616101FB02330A4A3870136015B0BDE82F
:1025E000F08F00BFD2D74100DC610020A05F002047
:1025F000E1D74100E7D74100A15F0020A85F00209C
:10260000D46100202C720020902500201FB50B788B
:10261000002B4FD0022B8DF802300CBF4B790023DA
:102620004A780EBFADF807308DF807308DF80830C6
:10263000224B8DF803201A780B7902FB0333C3F386
:1026400007238DF80630CB7942798DF80A308B79E3
:102650008DF80930CB788DF805308B783C218DF8DA
:10266000043000238DF80B308DF80C30037901FB1A
:10267000023382794FF4616101FB0233104A6946EB
:102680001268934236BFC2F5A3429B1A9B18ADF85D
:1026900000300C4B0D221B689C6A0B4B18680B4BCF
:1026A000A0470B4B0B4A18705388BDF8000001334C
:1026B000538000E0184604B010BD00BFB8510020A0
:1026C000D46100202C72002090250020A85F0020FB
:1026D000A05F0020A15F00202DE9F341427903793A
:1026E0003C2101FB023382794FF4616101FB02332B
:1026F000304A314F1268314D934236BFC2F5A34282
:102700009B1A9B182E4C2B803B6839215B692068F3
:1027100098472C4E3B680422D3F828C030702749D4
:10272000294B2068E0473B6830705B6900212068D6
:102730009847307003F06AFA4FF000086B880D2656
:1027400073431FFA88F23D339A4208F101080CD214
:102750003B6820681E690DF1050101221B4BB04743
:102760009DF8050003F03AFAE8E7002003F036FA96
:10277000002003F033FA03F051FA02AD0F4A25F8B6
:10278000020D51883B6871435B6920683D31984771
:102790003B68294602229E6A20680B4BB04706F030
:1027A0000BFF3B6820689B69984706F013FF02B057
:1027B000BDE8F081D46100202C720020A15F0020D0
:1027C00090250020A05F0020A85F0020D861002095
:1027D00002462DE9F0411A4E1A4D336890B08846F2
:1027E000DB681146286801229847174FC4B23C7035
:1027F00004BB33682868D3F810C001A93922134BF1
:10280000E047C0B2387060B9336828681C6969460F
:102810000E4B0422A047BDF8003038700124C8F8E0
:10282000003006F0C9FE336828689B69984706F0B7
:10283000D1FE00E00024204610B0BDE8F08100BFCA
:102840002C72002090250020A05F0020D86100207D
:1028500000B58BB007F07EFB01A806F0A3FD40B1E8
:1028600005A80549054A01AB08F0ACF905A806F032
:10287000C7FC0BB05DF804FBE1D74100E7D741008E
:1028800007B506F075FDC72801D8FFF7E1FF6846D8
:1028900003F0ECFA054B03F11C0003F13C019A69CB
:1028A0006B46FFF7F9FD03B05DF804FB38720020BA
:1028B00007B5684603F0DAFA6846FFF70DFF03B084
:1028C0005DF804FB13B5044606F052FDC72801D895
:1028D000FFF7BEFF684603F0C9FA2378022B04D144
:1028E0006379D22B84BFD223637168462146FFF7F8
:1028F0008DFE02B010BD4FF4E130002100F074B83D
:1029000070B50C46064600F00BF9A04228BF2046E1
:1029100084B24CB13546AB1B9BB2A34204D200F04B
:10292000C5F805F8010BF6E7204670BD4FF40060CE
:10293000002106F0ADBA00000A4B13B50A4A002484
:102940001C8001231380094A09481480094A6946FA
:102950008DE80C00224601F0F8FE074B1C7002B017
:1029600010BD00BF783800209A3800209C38002025
:10297000004102407A3800209E38002008B51448F3
:1029800005F0FCFC030722D5124A138801339BB2E1
:10299000138013889BB21E2B0EDC0F4A0F4913883D
:1029A0009BB20B440E490B6001234B60138801332B
:1029B00003F01F03138006E00548082105F0DCFC46
:1029C000084B01221A70BDE80840FFF7AFBF08BDF1
:1029D00000400240783800209A3800207A380020E1
:1029E000004102409E38002030B50D4687B0C0231C
:1029F0000024009001930E204FF40063029303948F
:102A00000494059404F078FA4FF0006160221648AF
:102A1000234604F0D3F815486946154A15B105F068
:102A200095FC01E005F058FC4FF0FF310F4805F030
:102A3000A3FC0E4805F098FC0C4805F098FC0D4BE3
:102A40004FF480421021C3F8802183F80E131A60DE
:102A5000FFF772FF0848012101F082FE03480821B8
:102A600005F088FC07B030BD000E0E40004002406B
:102A70000048E80100E100E00041024007B5002203
:102A80008DE803000848694601F054FE06484FF4FB
:102A9000807101F065FE044801F072FE0028FAD151
:102AA00003B05DF804FB00BF0041024038B5154B90
:102AB000154D1A88154892B2AC5C1A88082101326B
:102AC00002F01F021A8005F057FC114BE4B21A887D
:102AD000013A92B21A800F4B1B7863B10E4A0F492C
:102AE00013889BB22B440B6001234B601388013386
:102AF00003F01F0313800548082105F03BFC204626
:102B000038BD00BF9C3800207A38002000400240C9
:102B1000783800209E3800209A380020004102407A
:102B200038B5074D0821284605F026FC054B2846F8
:102B30001C880821A4B205F01DFC204638BD00BF4A
:102B400000400240783800200E2004F0F3B9000065
:102B500008B5054801234FF00061602204F02EF80B
:102B6000BDE80840FFF7F0BF000E0E4010B50E4C58
:102B70000E48012101F0C5FE2046042101F090FD20
:102B80002046052101F08CFD094A00231370094AF3
:102B90001D201370084A137004F0CCF9BDE81040F2
:102BA000182004F0C7B900BF0080034000000140B6
:102BB0009F380020A2420020A34200201FB5394BBD
:102BC00018689B8800901D20ADF8043004F094F93B
:102BD000354801F070FD3448042101F05DFD3248B4
:102BE000052101F059FD694606222F4801F017FD25
:102BF0002D4801F04CFD2D4B002202932C48402320
:102C000002A9039301F0A1FD2948012101F0A8FDCB
:102C1000284A00231370284A23481370274A4FF08C
:102C2000FF31137001F04EFD4FF000611E4801F0BE
:102C300047FD234B4FF000522021C3F8802183F839
:102C40001D131A601F4B204A196891420AD01C6854
:102C500040F6C41240F2E2431C498C420CBF1C46B1
:102C6000144601E040F2E244182004F045F9184807
:102C70000121184A01F030FE012124FA01F2144822
:102C800001F046FE22461248012101F048FE10489C
:102C9000012101F02FFE04480521002201F0B8FCBB
:102CA00004B010BDEAD7410000800340A2380020E4
:102CB000008103409F380020A2420020A342002050
:102CC00000E100E040070E4060079A286009902864
:102CD0000000014001C006001FB52E4C6846214689
:102CE00001F0F2FC6268009B002A42DA1A014FD51B
:102CF000294A14241378132B03BF284914200B7876
:102D0000137803BF013393FBF0F200FB123301335E
:102D10001ABFDBB21370DBB2214A08BF0B70117807
:102D2000204BC901595A2048C1F3033104291178B5
:102D300013BF03EBC111C901595A4988C1F30B01F3
:102D400001801178013191FBF4F004FB1011C9B23C
:102D500011701278154803EBC21302A900220293E6
:102D60004023039301F0F1FC07F0A0FD00F098F977
:102D70000EE0DB010CD5204601F096FC80B2030B7F
:102D8000042B05D1084BC0F30B00188007F08EFD13
:102D900004B010BD008003409F380020A3420020F3
:102DA000A2420020A2380020A03800200081034069
:102DB00010B50A4C0A490B4A0823204601F00CFCC6
:102DC0004FF4401201232046002101F053FC20461D
:102DD00001F06CFC044B00221A7010BD008003400F
:102DE0000048E8010024F400A4420020012838B57E
:102DF00005460A4C02D0022807D009E023780BB11F
:102E0000FFF7B4FEFFF7DAFE02E02378002BF9D0DB
:102E1000237845EA0300207038BD00BFA44200209B
:102E2000044A137823EA0000107008B9FFF79EBE29
:102E3000704700BFA442002010B506F08FFD034B81
:102E40001C7806F08DFDE4B2204610BD9F380020AE
:102E500038B5054606F082FD0023174A1749107859
:102E6000144603EB801031F81000C0F3033005283E
:102E700015BF107812785A1C03EB821218BF02EBB0
:102E8000801231F81220C2F30B02EA520233402BB7
:102E9000E3D10B4A14211378013BDBB21370237882
:102EA000013393FBF1F201FB1233DBB22370BDE877
:102EB000384006F055BD00BFA3420020A2380020D4
:102EC0009F380020014B188880B27047A03800203E
:102ED000C1F5FF437F33984206DC064B5B1A9842EC
:102EE00005DB084400B2704747F6FF7070470148A1
:102EF000704700BF0080FFFF2DE9F04391B0FFF75E
:102F00009BFF8046002800F0A28002F01DF90C24EF
:102F1000B0FBF4F0002784B2FBB2434580F08D8013
:102F2000032C07D904204B494B4A043C02F01BF9FF
:102F3000A4B23DE0474E484D94B9738A3353B28AE8
:102F400033195A80F28A9A806B8A2B53AA8A2B19DA
:102F50005A80EA8A0634182C9A80EED1002427E0A1
:102F6000204631462A4602F0FEF85FFA84FE062328
:102F7000621E5A4303FB0EF336F802C0B01826F85F
:102F800003C0B0F802C0F118A1F802C080880EF1A9
:102F9000010E8880A85AA918E852EA184B885FFAEF
:102FA0008EFE53808B88BEF1040F9380DFD1D5E76E
:102FB0006846FFF74DFF06F0D1FC284B5D781A7884
:102FC0001E46AA4207D0132D0CBF00226A1C5A705D
:102FD0004FF0010901E00025A94606F0C1FCB9F156
:102FE000000F28D0702303FB05631A4A023302F155
:102FF000180152F8040B8A4243F8040BF9D17023EC
:1030000003FB0563144A1A3302F1180152F8040B4A
:103010008A4243F8040BF9D1702303FB05656B4624
:10302000323510AE1A4603CAB242286069601346B0
:1030300005F10805F6D101376EE7012C07D901200B
:103040000449054A013C02F08EF8A4B2F5E711B03C
:10305000BDE8F083D4440020284300209A250020B6
:10306000054B1B7833B9054A11204EF660211370C9
:1030700005F07ABF704700BF41430020F2440020B2
:1030800010B5044602F004F80120FFF7AFFE0CB1C2
:1030900002F0E6F8014B01221A7010BDF544002041
:1030A00008B5104B01221A700F4B1B78C3B90F4B98
:1030B0001B78934214D10E4B1B68D3F8A03098476D
:1030C00030B1022806D102F0A1F818B102F095F84B
:1030D000FFF712FFBDE808400220002105F0D8BE2E
:1030E00008BD00BFA542002040430020F544002059
:1030F0002C72002008B50120FFF792FE01F0FCFFC2
:10310000014B00221A7008BDF544002008B5FFF7F6
:10311000F1FF112005F054FF122005F051FF064B7E
:103120001A782AB100221A70BDE8084000F086BE65
:10313000BDE80840FFF7BCBBF4440020014B187801
:10314000704700BFF44400200A4B10B51C78012CD6
:103150000FD1094A127862B902221A70FFF780FF74
:1031600001F0CAFF2046FFF75BFEBDE8104002F009
:103170009DB810BDF54400204143002008B5074B21
:103180001B78022B09D1112005F01AFF02F0C2F8BA
:10319000BDE808400120FFF773BF08BDF5440020DB
:1031A000074B1B7853B930B1064A12204EF6602106
:1031B000137005F0D9BE122005F002BF704700BFA2
:1031C00041430020F344002038B5032006F06CF89A
:1031D000104C2070002006F067F80F4B18701D4649
:1031E00018B1C82000F0BCFD08E0F8F7EFFFFFF7CA
:1031F00047FB237813B90120FFF7D2FF2B780BB9D7
:1032000023780BB1002000E00120BDE83840FFF733
:1032100037BF00BF41430020F444002030B5584C74
:10322000A1B0FFF773FFB4F900302BB9B4F9023045
:1032300013B9B4F9043013B1514807F0A9F90B20C0
:1032400006F032F8002800F087804E4D4E484F4976
:1032500006F094F9AA7AEB7A4D4943EA022212B2B7
:10326000684607F0AFFC4848694606F087F92A7BB4
:103270006B7B484943EA022212B2684607F0A2FC7F
:103280004148694606F07AF9AA7BEB7B424943EA5A
:10329000022212B2684607F095FC3B48694606F0E8
:1032A0006DF92A7C6B7C3D4943EA022212B26846E2
:1032B00007F088FC3A4D3448694606F05FF9324819
:1032C000384906F05BF9AA78EB78324943EA0222E2
:1032D00012B2684607F076FC2B48694606F04EF9B4
:1032E0002A796B792C4943EA022212B2684607F028
:1032F00069FC2548694606F041F9AA79EB79274926
:1033000043EA022212B2684607F05CFC1E48694696
:1033100006F034F91C48244906F030F9B4F90020CD
:103320001C49684607F04EFC1748694606F026F926
:10333000B4F902201849684607F044FC124869466F
:1033400006F01CF915496846B4F9042007F03AFC68
:103350000D48694606F012F907F018F9134B1020D2
:103360001B68D3F89830984707F0AAFA10B106F016
:1033700075FB03E006F0C5FD06F0BEFB21B030BDD5
:10338000EC44002000FC4100F0D74100FCD7410094
:1033900004D841000FD841001AD8410025D8410077
:1033A00000F8410030D8410039D841002C7200208B
:1033B0002DE9F04F8FB0002706F0D0FA954A157826
:1033C0001446132D537802D100253BB103E001359B
:1033D0009D4205D0EDB21570012603E01D4600E0C8
:1033E00000252E4606F0BCFA002E00F00781002FC3
:1033F00040F0048170235D436019014604462C317E
:103400001430B4F8702005F07BF9824E01270028B3
:10341000D2D105F13207183537442E4463887E4AED
:10342000A588E188ADF81830B4F81C90638BB4F827
:103430001EB092F800E0ADF81A50ADF81C10ADF8CF
:103440002030ADF82290ADF824B008B22AB20FFABD
:1034500083FABEF1000F25D010F5004F1ABF494284
:1034600089B247F6FF7112F5004F1ABF6D42ADB237
:1034700047F6FF751AF5004F0CBF47F6FF735B4226
:10348000ADF81A1018BF9BB206A808A93A46ADF8C5
:103490001C50ADF82030ADF822B0ADF8249000F00B
:1034A0008FFCA4E0DFF87C81019298F80A1098F86C
:1034B0000B3043EA012109B2FFF70AFD009098F8AA
:1034C0000C0098F80D1041EA002109B25046FFF7B0
:1034D000FFFC824698F80E0098F80F1041EA002190
:1034E00009B20FFA89F0FFF7F3FC814698F8100053
:1034F00098F8111041EA002109B20FFA8BF0FFF79A
:10350000E7FC009B019A13F5004F1ABF5B429BB288
:1035100047F6FF7312F5004F0EBF47F6FF756D4279
:10352000ADB21AF5004F804608BF47F6FF70ADF800
:103530001C503A4DADF81A30A978EB781CBFCAF18F
:10354000000080B243EA012109B200B2FFF7C0FCDB
:1035500029796B79ADF8200043EA0121404609B290
:10356000FFF7B6FCA979EB79ADF8220043EA012117
:1035700009B24846FFF7ACFC08AAADF824003B4668
:1035800002A806A9F8F7CCFE0AAA904602AB0DF1F4
:10359000100E154618685968083303C573452A4646
:1035A000F7D1186828609B88AB809DF833109DF890
:1035B00030201B4B42EA01221A809DF834109DF8FE
:1035C000312042EA01225A809DF835109DF83220C0
:1035D00042EA01229A8005F07FFB40B99DF828302D
:1035E0002BB10120FFF7DCFD4046FFF76BF90634F5
:1035F000B44207F110077FF411AFDCE6064B1B78ED
:103600002BB105F0B5FE132801D8FFF707FE0FB068
:10361000BDE8F08F9A250020F444002000F8410016
:10362000EC44002000FC410038B506F055FC07F0E2
:1036300047F918B1BDE83840FFF7F0BD084B094C19
:103640001B68B4F811505B6D984706F0F9FDA4F8BB
:10365000115006F09BFFBDE8384006F04DBA00BFA0
:103660002C72002038720020064A13780133DBB236
:10367000012B137001D1FFF7D1BD11204EF660214F
:1036800005F072BCF2440020064A13780133DBB225
:10369000012B137001D1FFF7C1BD12204EF660213E
:1036A00005F062BCF34400202DE9F04F00252E46C2
:1036B000914B9BB001221A7001950020014606F043
:1036C000C3FB0120002106F0BFFB0220012106F010
:1036D000BBFB8A4A00231370894A1370894A13601E
:1036E000894A1360FFF770FD884C237823B906F0F0
:1036F00001F934462646F7E7854B1F7897B9854B85
:10370000197881F0010119702DB9284606F09CFB4B
:103710000220294604E0022006F096FB384639468E
:1037200006F092FB4FF0000884F80080FFF784FB5E
:103730008146002800F0738201F006FD0C24B0FBE6
:10374000F4F084B25FFA88F34B4551D2032C07D9C9
:1037500004207149714A043C01F005FDA4B241E026
:103760006D4F9CB97B8A3B53BA8A3B195A80FA8ABF
:103770009A806A4B5A8AE252998A1A195180DB8AD6
:103780000634182C9380EDD100242BE0634A2046A8
:10379000394601F0E8FCE2B20623611E5943534367
:1037A00037F801C007EB010E27F803C0BEF802C0CE
:1037B000F818A0F802C0BEF804E00132A0F804E056
:1037C0005648D2B230F801C000EB010E20F803C019
:1037D000C118BEF80230042A4B80BEF804308B803A
:1037E000DAD1D1E70AA8FFF733FB08F10108A9E70E
:1037F0004B4B4C4F02930DF136030493019B059301
:1038000000230393029937F8023C31F802AC09888F
:103810003A8806910299B7F802804988ADF82030BD
:1038200007913B49ADF822200978ADF824800029A2
:1038300040F02F8103F5CD7080B2B0F54D7FDFF8F9
:10384000F0C00AD802F5CD7080B2B0F54D7F04D833
:103850000FFA88FEBEF1000F04DD0025ACF8005021
:10386000A84608E1BCF8000006254543DFF8C4B0CF
:103870000BEB05092BF80530A9F8022012B25243D0
:103880001BB203FB03230EFB0E33274AA9F8048067
:10389000DFF8A48022F805A048F820305319BDF8BD
:1038A000182001305A8080B2BDF81C201F289A8051
:1038B000434604D8ACF8000001258846DBE00A4600
:1038C00053F82100013189B220290244F8D192FB3A
:1038D000F1F14FF001080022202A2FD053F82200E6
:1038E000124D401A0028B8BF40420132A842C8BF5A
:1038F0004FF0000892B2EFE740430020024400205E
:10390000CC440020D044002004440020A5420020E4
:10391000CA440020CB440020D44400202843002087
:103920002A430020D644002008440020A08601003D
:10393000C844002042430020A8420020B8F1000FF4
:1039400000F0958000231D4699469A469E461946EA
:103950001A4606205843DFF8A8B301330BEB000CDE
:103960003BF900B09BB25A44BCF902B0BCF904C0A8
:103970005944DFF890B3E6440BEB000C3BF9000030
:10398000202B8244BCF902008144BCF904000544A8
:10399000DFD192FBF3F291FBF3F15243C2F58002C7
:1039A00001FB1121C4489EFBF3FE03804FF0100B76
:1039B0004FF4006391FBF3F20BF1FF3B13444FF024
:1039C000020C1BF0FF0B93FBFCF3F3D17344604636
:1039D00059460793CDF818C006F036FA079BDDF874
:1039E00018C05B429BB203F5FA7292B2B2F57A7FCD
:1039F0000CD90121584606F027FA642008F0F8FB9C
:103A00005846594606F020FAD84630E001200146D3
:103A10000693CDF81CC006F017FA4FF47A7008F040
:103A2000E7FB5946012006F00FFADDF81CC0012122
:103A3000604606F009FA069B4FF0200B19469F4896
:103A400006F000FB9AFBFBF1494289B29C4806F064
:103A5000F9FA99FBFBF1494289B29A4806F0F2FA69
:103A600095FBFBF56942984889B206F0EBFA924B58
:103A700000221A800125954B83F80080B8F1000FD1
:103A800000F09180FFF742FB4FF00008FFF79CFB2E
:103A900089E08F4A136833B1013B13601BB98D4A2B
:103AA0001370012303938C4B04981A888B4BA0F15D
:103AB000100C1B883CF802EF0498724528BF724630
:103AC000734538BF73468445F4D18448DFF808E273
:103AD00003809B1AC82BAEF800200BDD7C4B202204
:103AE0001A607C4B01221A704FF6FF73AEF800305B
:103AF000002303807A4A136833B1013B13601BB97A
:103B0000784A1370012303930023774808AA32F8F8
:103B1000132030F913800FFA82FCE045C8BF20F86B
:103B2000132072484FEA430E3EF900800133E0450E
:103B3000B8BF2EF80020032BE7D1DFF8A881684B2F
:103B400098F80090D3F800C00023684A664832F91C
:103B500013A030F913E0CEEB0A0E42F2107AD645EC
:103B60000FDD47F6FF7E8946A0F800E0A0F802E0EE
:103B7000A0F804E04FF400401080508090804FF097
:103B8000200C0133032BE0D1554B88F80090C3F88B
:103B900000C0504B1B781BB1524B93F8008000E0E3
:103BA000984608F00108002006F046FF012806F1BB
:103BB0000106814617D1019B01330193059BB3F5A3
:103BC000C87F12D10020014606F03EF94846002188
:103BD00006F03AF90220002106F036F905F08CFFD4
:103BE00040F2911300E000230193414B9F420CD01F
:103BF000029B063706330293049B10330493B8F1FB
:103C0000000F02D1019B0593FCE5072C09D9042084
:103C10003849394A043C01F0A6FAA4B2F5E78046D7
:103C2000039005F067FE354B741C9E4203D9FFF7E5
:103C30006DFA05F061FFB8F1000F03D1039B002B73
:103C40003FF458ADFFF762FAB8F1000F1DD14046BE
:103C5000012106F0F9F80120414606F0F5F8414649
:103C6000022006F0F1F840F6B83008F0C1FA4046FC
:103C7000414606F0E9F80120414606F0E5F8022049
:103C8000012106F0E1F8264617E50020014606F07E
:103C9000DBF80120014606F0D7F80021022006F0EB
:103CA000D3F840F6B83008F0A3FA05F075FC05F03B
:103CB00023FF1BB0BDE8F08FC84400200AFC410080
:103CC0000CFC41000EFC410010FC4100CA440020E5
:103CD00004440020CC440020622E0020CE4400206A
:103CE000D0440020024400205C2E002094250020B7
:103CF000E8440020D4440020284300201FBF0200D5
:103D000042430020084400201FB50D4B1B78012BB7
:103D100013D18DF8013003230A228DF80230684652
:103D200000238DF800208DF803308DF805308DF8D4
:103D300006308DF80730FEF7C5FD05B05DF804FBD1
:103D4000F544002008B50120FFF72AFA112005F0FC
:103D500059F918B1BDE80840FFF782B908BD000065
:103D600010B5044686B004A802F080F89DF8103023
:103D700020468DF808309DF8113011218DF809305A
:103D80009DF812300C4A30338DF80A309DF8163009
:103D90008DF80C309DF815308DF80D309DF81430ED
:103DA0008DF80E3003AB009302AB00F0DBFF034B4A
:103DB00000221A8006B010BD45D84100F64400200C
:103DC00010B51D4C8AB02388ADF804300388ADF8D7
:103DD00006304388ADF808308388ADF80A300B8888
:103DE000ADF80C304B88ADF80E308B88ADF8103044
:103DF000002301A91944D05A0233102BC881F8D1ED
:103E000006F066FD0023ADF8220001208DF8243075
:103E100006F012FE012808BF9DF8243001A804BF57
:103E200043F001038DF8243001F014F823880133A6
:103E300023800AB010BD00BFF644002001F042B854
:103E400010B50446152003F057F8204600F09AFC00
:103E5000204600F0A4FC204600F0B4FC204600F010
:103E6000B6FC0021204600F0B7FC204600F09CFC88
:103E7000204600F09EFC2046BDE81040012100F0E5
:103E8000B6BC0000F8B505460C461F461646012292
:103E90001346096800F005FD28462168082200F055
:103EA000EBFC0E4A2846B2FBF7F22168D2B200F0D2
:103EB000EDFC28462168082200F0BEFC2846216857
:103EC000720800F0A3FC06F001022846216882F087
:103ED0000102BDE8F84000F0A4BC00BF0048E801C2
:103EE00038B50D46044600F069FC296818B10F2961
:103EF0000CD8204606E0032908D8012303FA01F173
:103F00002046C943BDE8384000F066BC38BD10B556
:103F10000446204600F076FC0028FAD020460F2107
:103F200000F05AFC2046BDE8104000F034BC0020F0
:103F3000704700000030044B18BF01201870034B7D
:103F400001221A70704700BFEC610020642E00202F
:103F500010B5054C00212046122207F0E1FDF023A8
:103F600023700A23E37110BD20450020024B00227C
:103F70001A7001F0A7BD00BFF944002007B5094B36
:103F8000022000930121084A1F2304F045F830B9AC
:103F90000649022003B05DF804EB04F051B903B008
:103FA0005DF804FBED424100344500207D3F4100B7
:103FB0000B4A002310B513700A4A137002F0B2F8CE
:103FC000094B10B91870002408E00138187001F08E
:103FD00073FD04460028F6D0FFF7D0FF204610BD41
:103FE000F9440020FA440020F8440020FFF7C6BF3F
:103FF00007B5094B812000930021084A0D2304F0E6
:104000000BF830B90649812003B05DF804EB04F0E9
:1040100017B903B05DF804FBED3F4100A02E00206E
:10402000F13F410038B5094B094D9A681C463AB139
:1040300095F90C30002BB4BF8120022003F02EFF35
:104040006B686360BDE83840FFF7D2BFA02E002048
:104050003445002008B5064B1B7843B1022003F01D
:104060001DFFBDE808400220024904F0E9B808BD80
:10407000FA4400205540410008B5064B1B7843B177
:10408000812003F00BFFBDE808408120024904F0C5
:10409000D7B808BDFA4400207940410038B50D4634
:1040A000044650B9FFF754FF044B9A681C73521B27
:1040B0009A60BDE83840FFF7B5BF38BDA02E00209C
:1040C00008B5174B1A7812F0800F02F060020DD07D
:1040D000202A22D15A78FE2A1FD1D88801281CD143
:1040E0005A88D2B90F4A98819A6008BD202A14D103
:1040F0005A78FF2A11D1D88878B95B8873B90A4AEF
:1041000002201370094A137004F00EF8812004F0A5
:104110000BF8FFF733FF012008BD002008BD00BFEA
:1041200014720020F8440020FA440020F9440020D2
:1041300038B50C460546FFF70BFF074B01221A73F3
:10414000064B0022DA701A715A719A71220A9D7018
:104150001A735C7338BD00BFA02E002020450020DC
:1041600002204FF46851FFF7E3BF06204FF42051BF
:10417000FFF7DEBF04200021FFF7DABF07B50B46CB
:104180000849024600918120012103F045FF30B922
:10419000FFF7F0FF03B05DF804EBFFF743BF03B098
:1041A0005DF804FB9D40410005204FF41051FFF7DE
:1041B000BFBF000008B5084B1B7B59400B0603D45A
:1041C000064B9B68834205D2FFF7EEFFFFF72AFFFD
:1041D000002008BD012008BD34450020A02E00208D
:1041E0002DE9F041064600212148142207F098FCF1
:1041F0001F4DDFF880802EB198F8171005F10803E5
:10420000082403E098F813102B1D042498F81120BB
:1042100002F03F021C2A01D03F2A07D11C221A704B
:104220000A225A700C340522DA70E4B2A14228BF87
:1042300021460F4608468021FFF7BCFFB0B198F831
:104240000D0001F07CFF002814BF8023002326B15D
:10425000023C24022C80EB7002E0013C2C70AB701D
:104260003946BDE8F0410248FFF788BFBDE8F0815C
:10427000FC4400203445002038B50546164C60B992
:10428000607B01F05CFF40B107204FF41C51FFF749
:104290004FFFBDE83840FFF7C5BE104B627C002DD4
:1042A000DA70A27C18BF80219A70E27C08BF0021DE
:1042B0005A70227D1A700A4BA27D5A70E27D1A70E4
:1042C00018884002FFF776FF20B1064B01221D70CF
:1042D000054B1A7038BD00BF344500201C45002036
:1042E0001845002032450020F944002070B5002810
:1042F00040F0E8801F2904D1734C744B22689A4225
:1043000008D0734B01221A70FFF7A4FEBDE870407D
:10431000FFF7B2BE6F4B627B1B7802F00F02934235
:10432000627302D2FFF740FFC4E0A3686A4DAB603E
:10433000E37B1E2B00F0B0800DD8122B2CD004D8BC
:10434000002B67D0032B19D0AFE01A2B5ED01B2BAC
:1043500000F08D80A9E02A2B00F0A38006D8252B41
:1043600065D0282B40F0A18001209AE02F2B00F08F
:1043700093805A2B40F09980012047E0E47C802113
:10438000122C28BF12242046FFF714FF002800F04B
:1043900099805248214635E0E57C8021242D28BFB4
:1043A00024252846FFF706FF002800F08B80237C99
:1043B0009B07B7D1637C002BB4D1607B01F0C4FEB6
:1043C000474E431C00F111023446186859680833FF
:1043D00003C493422646F7D100224249D3B288183B
:1043E000007C28B1222803D00132102AF5D11346CF
:1043F000102B05D0CA18202001331074DBB2F7E768
:1044000029463848BDE87040FFF7B8BEBDE87040A7
:10441000FFF7E6BE104601F087FE0228044623D0CF
:1044200003281ED0002849D0FFF7A4FE42E0082050
:104430008021FFF7BFFE002844D02B4D607B29462A
:1044400001F077FE02280FD003280AD00028EBD114
:104450004FF400336B602B6828461BBA2B60082191
:10446000D0E7FFF782FE25E0FFF77AFE22E0002684
:10447000FFF76EFD2E73FFF7D5FDE37C03F003031A
:10448000022B02D0032B02D070BD012000E0304689
:10449000BDE8704001F096BAFFF75AFD00232B7378
:1044A00008E0BDE87040FFF7E7BE05204FF400517B
:1044B000FFF73EFEBDE87040FFF7B4BDFFF748FDD3
:1044C0002C73F7E770BD00BF3445002055534243BD
:1044D000FA440020F8440020A02E002020450020AF
:1044E0008C2E00207C2E00201045002038B5164B65
:1044F0001D783DB300221A70144B15491878154ADF
:10450000154B28B1487B11681A8801F025FE04E09C
:10451000487B11681A8801F031FE022804460AD04F
:10452000032805D050B9FFF713FD0C4B1C7307E0AF
:10453000FFF71BFE04E0FFF713FE01E0FFF71AFE92
:10454000FFF770FD284638BDF944002032450020B1
:10455000344500201C45002018450020A02E0020D6
:10456000F7B5194C1E4623788E46154627460BB9DB
:10457000002026E00021154B884214BF8120022034
:104580008E4218BF3346724600932B46217003F0CB
:1045900043FD10B90123237013E076B93B78002B5B
:1045A000FCD00B4B1A78002AE2D10A4918788A68A5
:1045B00080F00100521B8A6003E0064B9A68521B90
:1045C0009A6003B0F0BD00BF642E0020353F41006B
:1045D000EC610020A02E002030B5520040F20225F0
:1045E000B1FBF2F10124046000244460C0F82051C2
:1045F000C0F80441C0F8144145684A1E1B0403F486
:10460000702312022B4392B213434360204630BD05
:104610004368D2011943D2B2114341607047072A5F
:1046200070B54FF000030BD8DCB2944207D2CC5CDB
:1046300085689E00B4402C4384600133F4E770BD6C
:10464000CC5C85689E00B44001332C43082B846009
:10465000F6D10024E3B2A2F10805AB4204F1010453
:1046600007DACE5CC5689B0006FA03F32B43C360F0
:10467000F0E770BD10B544680906224301F070618F
:104680001B070A4303F040531343436010BD4368C4
:1046900023F400034360704701238B40036170479C
:1046A00001238B4043617047006A7047036C43F0FD
:1046B000807303647047436843F00043436070476E
:1046C000416270478162704710B50C6BCA6B046021
:1046D000426010BD0368090201F4706123F4706345
:1046E0000B43036070470068C0F30320704700006D
:1046F000A1F10E03012B10B5044612D90A4B120288
:1047000022F07F421B68094822F0FF0242F0B442C7
:10471000C9B20360114300209847A06800F006006A
:1047200010BD4FF0FF3010BD080080005445002040
:10473000C068704719B10B6883604B68C3601AB1D9
:10474000136883615368C361704719B10B680360D4
:104750004B6843601AB11368036153684361704743
:1047600021F0FE01C905C90D0162704721F4FE71F7
:1047700021F001018905890D01627047406A704787
:10478000C06870478023036070470123036070474F
:104790000223036070474FF08073036070474368E3
:1047A00043F0010343607047436823F00203436012
:1047B0007047436823F00403436070474068C0F3C8
:1047C00080007047436843F01003436070474368BC
:1047D00023F08003436070474368090423F4702387
:1047E0004360436801F470210B43436070474368A2
:1047F00023F07F434360436843EA016141607047AF
:10480000006970470069C0F3402070478900014487
:104810000B6B12B143F0010301E023F001030B63C2
:104820007047890001440B6B12B143F0020301E0B1
:1048300023F002030B637047042A09D100EB8101C6
:104840000B6B23F008030B630B6B43F0040311E0C5
:104850004AB900EB81010B6B23F008030B630B6B70
:1048600023F0040306E0082A05D100EB81010B6B5D
:1048700043F008030B63704700EB81010B6B23F0DF
:10488000F0030B630B6B1A430A63704700EB810163
:104890000B6B23F47F430B630B6B43EA02220A6327
:1048A000704700EB8101086B10B580B208630C6B98
:1048B00044EA036343EA02420A6310BD836823F0BB
:1048C0007F4323F4805343F025438360704743685C
:1048D00023F4805343607047022910B500D9FEE7E6
:1048E00089010224431844504FF0FF319962196A3C
:1048F0005A6010BD022900D9FEE789010523435003
:104900007047022900D9FEE789010223435070470E
:10491000022900D9FEE700EB8110426170470229AD
:1049200000D9FEE700EB8110C2617047022900D96F
:10493000FEE700EB811042627047022900D9FEE7D2
:1049400000EB8110006A7047084BB3FBF1F188421D
:1049500008D3C1EB0133984204D8B0FBF1F0C0F3A7
:104960000B0070474FF6FF70704700BF0020A10793
:1049700010B5044CC2F30B0204EA0343134319437A
:10498000416010BD0000FF0F014B0360704700BF86
:10499000010000A5044B1868044B98420CBF4FF46B
:1049A00000404FF48040704740070E40600A9B284B
:1049B000B1F5800F30B500D2FEE7B1F5840F00D914
:1049C000FEE7A1F58004C4F30F24C9B208B1034D7A
:1049D000056002B1148003B1198030BD000A0E4099
:1049E000034613B50C46002201A819461346FFF7EB
:1049F000DFFF01982146FFF76DFE002002B010BDD9
:104A000007B500220146134601A8FFF7D1FF019820
:104A1000FFF769FE03B05DF804FB00002DE9F04FDD
:104A2000044685B0009303A80DF10A038846174693
:104A3000214602AAFFF7BCFF0398FFF754FE0621A8
:104A400081460398FFF746FE002F44D0BDF80A5078
:104A50003E46C5F5807C674528BF6646BDF808A080
:104A6000DFF884B00AF58044240221462A465846DD
:104A7000CDF804C006F0DEFF414632460BEB0500E0
:104A800006F0D8FFDDF804C07019C6EB0C026119FE
:104A9000314492B2584406F0CDFF224604F58071AD
:104AA000C4EB0B00805842F8040B8A42F8D1009BFB
:104AB00003980BB1032100E001215246FFF718FED5
:104AC00070B9BDF80830B0440133BF1BADF80830F1
:104AD000ADF80A00B8E703984946FFF7FBFD3846F2
:104AE00005B0BDE8F08F00BF584500202DE9F74321
:104AF0000C46054690469946FFF74CFFC0F30F263B
:104B0000FFF748FFB5FBF0F101FB10502D1AFFF73E
:104B100041FFB4FBF0F707FB1047FFF73BFF013CF9
:104B20002044C41BB8F1000F01D0C8F80050B9F1FF
:104B3000000F01D0C9F8004001A829466A460023A9
:104B4000FFF736FF002021460DF102020346FFF772
:104B50002FFFBDF80020BDF8023093420AD901981A
:104B60000821FFF7C5FD30B9BDF800303344ADF87A
:104B70000030EEE7002003B0BDE8F0832DE9F743F5
:104B80000C46054690469946FFF704FFC0F30F26F2
:104B9000FFF700FFB5FBF0F101FB10502D1AFFF7F6
:104BA000F9FEB4FBF0F707FB1047FFF7F3FE013CFB
:104BB0002044C41BB8F1000F01D0C8F80050B9F16F
:104BC000000F01D0C9F8004001A829466A46002319
:104BD000FFF7EEFE002021460DF102020346FFF72B
:104BE000E7FEBDF80020BDF8023093420AD90198D3
:104BF0000921FFF77DFD30B9BDF800303344ADF831
:104C00000030EEE7002003B0BDE8F083012810B5C6
:104C100004460FD809480D210022FFF769FD58B955
:104C20000648FFF785FD0123A34018420CBF012071
:104C3000002010BD112010BD102010BD000A0E4034
:104C4000012810B504460ED8FFF7E0FF012801D176
:104C5000002010BD05480C212246FFF749FD002821
:104C6000F6D0102010BD112010BD00BF000A0E406C
:104C700010B50446054803F083FB0028FAD021460E
:104C8000BDE81040014803F07FBB00BF0040024078
:104C900038B505460C46BCB10C4B0D481B6829467F
:104CA000D3F8883001229847034608B1012038BD67
:104CB000012007494FF40072FFF752FC0028F5D09D
:104CC000013C0135A4B2E6E7204638BD2C72002035
:104CD000F061002070B505460C46DCB100200E499D
:104CE0004FF400720346FFF73BFC08B9012070BD8A
:104CF0000A4B09481B682946D3F88C300122984793
:104D00000646054805F090FC002EEFD1013C013528
:104D1000A4B2E2E7204670BDF06100202C720020B2
:104D20000246014804F0B6BD5846002007B502A966
:104D300001F8010D0120FFF7F3FF03B05DF804FB5C
:104D400037B50546030A02AC04F8013D21460120AF
:104D5000FFF7E6FF012021468DF80750FFF7E0FF3F
:104D600003B030BD2DE9F04F0C469946834690467E
:104D700087B001A8109F04F03BFC012201A9324832
:104D800004F04CFD06AD4FF0000A10202F49FFF74C
:104D9000C7FF05F816AD29460120FFF7C1FF2226FF
:104DA00029460120FFF7BCFF04FB066629460120C7
:104DB000FFF7B6FF2946012006ADFFF7B1FF05F862
:104DC00015AD29460120FFF7ABFFC6F3074329467F
:104DD00001208DF80330FFF7A3FFC6F30723294610
:104DE00001208DF80330FFF79BFF294601208DF845
:104DF0000360FFF795FF99F80000FFF797FF99F818
:104E00000100FFF793FF99F80200FFF78FFF387852
:104E1000FFF78CFF7878FFF789FFB878FFF786FFF8
:104E20005846FFF78DFF2046FFF78AFF04EB04107A
:104E30004000414680B2FFF773FF10200449FFF79E
:104E40006FFF07B0BDE8F08F5846002087DA4100B9
:104E500097DA410010B504460088FFF771FF6088BB
:104E6000FFF76EFFA088FFF76BFFE088FFF768FF92
:104E70002089FFF765FF6089FFF762FFA089FFF7D0
:104E80005FFFE089FFF75CFF208AFFF759FF608A28
:104E9000FFF756FFA08AFFF753FFE08AFFF750FFA6
:104EA000208BFFF74DFF608BFFF74AFFA08BFFF7CA
:104EB00047FFE08BFFF744FF94F82000BDE8104067
:104EC000FFF734BF014804F0C7BC00BF58460020BC
:104ED00000F0CABF08B5054B054A1B6810681B6E79
:104EE000984700280CBF0220002008BD2C7200202B
:104EF000F0710020034B1B685B6D5B0003600020BA
:104F0000704700BFF071002000207047F8B50646DA
:104F10000C46E4B10F4B072C1B6898BFE5B25F6EDF
:104F20000D4B88BF082518680C492B463246B847F8
:104F3000034608B10120F8BD012008496A02FFF7C5
:104F40000FFB0028F6D0641B2E44A4B2E1E72046F4
:104F5000F8BD00BF2C720020F0710020F06100202D
:104F6000F8B506460C46FCB1072C94BFE5B20825FF
:104F700000200E496A020346FFF7F2FA08B9012041
:104F8000F8BD0B4B09491B6832469F6E094B1868E8
:104F90002B46B8470746054805F046FB002FEED1E3
:104FA000641B2E44A4B2DEE72046F8BDF061002069
:104FB0002C720020F071002070B506460D46144694
:104FC000012000F051FA30462946224600F0A0FAAE
:104FD000BDE87040012000F057BA38B505460C46D0
:104FE000012000F041FA28462146012200F05CFA37
:104FF000BDE83840012000F047BA37B500F0CEF9DF
:105000000024F52001A90122FFF7D6FF9DF80450E6
:10501000682D03D00134B4F5803FF2D1032301A9F8
:105020006B208DF80430FFF7D8FF322007F0E0F84E
:10503000102301A96A208DF80430FFF7CEFF272343
:1050400001A919208DF80430FFF7C7FF182301A923
:105050001B208DF80430FFF7C0FF1C2001A98DF83C
:105060000400FFF7BAFF002301A91A208DF80430CD
:10507000FFF7B3FF43236B2001A98DF80430FFF73E
:10508000ACFFA5F168035842584103B030BD0000A1
:1050900013B5032302AC04F8043D21466B20FFF74F
:1050A0009CFF322007F0A4F8002321466C208DF8E5
:1050B0000430FFF792FF7823214623208DF8043037
:1050C000FFF78BFF542321466A208DF80430FFF749
:1050D00084FF0849102338200B70FFF77EFF012062
:1050E00000F07CF9BA2021460122FFF765FF02B0EB
:1050F00010BD00BF8148002037B5002000F06EF9D8
:1051000002AC142304F8043D21466A20FFF765FF32
:105110000025214623208DF80450FFF75EFF094942
:1051200038200D70FFF759FF21460122BA20FFF702
:1051300043FF43236B2021468DF80430FFF74DFFDA
:1051400003B030BD8148002007B5F22001A902223A
:10515000FFF732FF9DF804009DF8053043EA002078
:1051600003B05DF804FB2DE9F043884691461546EF
:105170000E460627474385B00024BC423AD0F420AF
:1051800001A90C22FFF718FFB8F1000F15D09DF808
:1051900004209DF8053043EA022328F804309DF8E6
:1051A00006209DF8073043EA022373809DF808200B
:1051B0009DF8093043EA0223B380B9F1000F15D0FE
:1051C0009DF80A209DF80B3043EA022329F80430A9
:1051D0009DF80C209DF80D3043EA02236B809DF86A
:1051E0000E209DF80F3043EA0223AB8006350634CB
:1051F0000636C2E705B0BDE8F08308B500F01AFA3C
:10520000BDE80840002000F03FB9000008B50348A1
:10521000FFF7B4FA00F0010008BD00BF00810040B4
:1052200013B5142302AC04F8043D21466A20FFF7AD
:10523000D4FE0023214623208DF80430FFF7CDFE55
:105240007823214623208DF80430FFF7C6FE54232F
:105250006A2021468DF80430FFF7BFFE02B010BD72
:1052600013B5192302AC04F8043D21462120FFF7B1
:10527000B4FEEA23214622208DF80430FFF7ADFE6C
:10528000044938200B7843F020030B70FFF7A5FE8C
:1052900002B010BD81480020034938200B7843F04C
:1052A00001030B70FFF799BE8148002037B500233A
:1052B00002AC04F8043D21466B20FFF78EFE32203D
:1052C00006F096FF072321466C208DF80430FFF787
:1052D00084FE192321461F208DF804300125FFF795
:1052E0007CFE214620208DF80450FFF776FE084909
:1052F000402338200B70FFF770FE284600F06EF850
:10530000BA2021462A46FFF757FE03B030BD00BF42
:1053100081480020FFF7F0BE034B0122202000212E
:105320001A7003F0B5BD00BF8048002007B5BA2051
:1053300001220DF10701FFF73FFE104B00221A700A
:105340009DF80730D80601D5FFF76AFF9DF80730B2
:10535000590601D5FDF712FF9DF807309A060AD5C8
:10536000E12001A90122FFF727FE9DF80430DB07A9
:1053700001D5FDF7E9FE03B05DF804FB804800208D
:10538000014B1878704700BF804800200B2803D1DC
:10539000022901D1FFF7C0BF7047000007B50B4BD2
:1053A0000B21009302227023094801F003FD094BF1
:1053B0004FF400622021C3F8802183F80B131A6098
:1053C000054B00221A6403B05DF804FB8D534100C5
:1053D000000E0E4000E100E000040E4018B1044849
:1053E000022101F043BC0248022101F042BC00BF8F
:1053F000000E0E40F0B5184C85B02046FFF7C8F9F6
:105400002046FEF71DFD04AD144F012345F8043D71
:105410000026204629463B4600960222FEF732FD32
:1054200020462946009603220D4B0396FEF72AFDDF
:105430000222204629463B4600960392FEF722FDB3
:10544000084B4FF40012C3F880212046C3F8802097
:10545000FFF79BF905B0F0BD0080004040420F000F
:105460000024F40000E100E013B50446152001F02B
:1054700043FD02A941F8044D0248FEF731FD02B098
:1054800010BD00BF0080004007B502A941F8040D1F
:105490000448FEF73CFD152001F04CFD03B05DF81B
:1054A00004FB00BF0080004030B514460D468DB0AF
:1054B0000CAB03F8290D04930691012307921248BF
:1054C00004A906AA0593FFF735F903AB08930E4824
:1054D000022308A9013C0AAA09930A950B94FFF735
:1054E00034F9094840F20111FFF73AF90748FFF78C
:1054F00087F90206FAD54306F8D5034840F202219F
:10550000FFF734F90DB030BD00810040008000404D
:1055100030B50D4614468BB0FF238DF8053001AB36
:10552000029302238DF8040003930491531E124842
:1055300002A904AA0593FFF7FDF801230E4806A966
:1055400008AACDF818D0079308950994FFF7FDF83D
:10555000094840F20111FFF703F90848FFF750F935
:105560000206FAD54306F8D5034840F20221FFF7B8
:10557000FDF80BB030BD00BF00810040008000404E
:1055800008B540B300F094F94FF020510C2001F021
:105590009CFB4FF020510D2001F097FB4FF0205164
:1055A0000E2001F092FB2149162001F08EFB1F49CD
:1055B0000A2001F08AFB4FF060510B2001F085FBBF
:1055C0004FF06051092001F080FBBDE80840022047
:1055D000164901F07ABB4FF000610C2001F075FB19
:1055E0004FF000610D2001F070FB4FF000610E20C4
:1055F00001F06BFB0E49162001F067FB4FF0805164
:105600000A2001F062FB4FF000610B2001F05DFB0E
:105610004FF08051092001F058FB02204FF040511B
:1056200001F053FBBDE8084000F045B90100002837
:105630000100000808B50448FFF7E2F80206FAD5B1
:105640004306F8D508BD00BF0080004070B50C4689
:10565000064600F009F9A04228BF204684B24CB1AA
:105660003546AB1B9BB2A34204D200F0C3F805F849
:10567000010BF6E7204670BD0120002103F008BCB5
:105680000A4B13B50A4A00241C8001231380094ADF
:1056900009481480094A69468DE80C002246FFF744
:1056A00054F8074B1C7002B010BD00BF84480020A6
:1056B000884A002086480020008102408848002057
:1056C0008248002008B5154802F058FE030723D58C
:1056D000134A138801339BB2138013889BB2B3F52E
:1056E000FF7F0EDC0F4A104913889BB20B440F4911
:1056F0000B6001234B6013880133C3F3080313804D
:1057000006E00648082102F037FE094B01221A7014
:10571000BDE80840FFF7B0BF08BD00BF00800240F1
:1057200084480020884A00208848002000810240E8
:1057300082480020F0B5164687B000240090C023B0
:105740004FF400650F200F460193029503940494D3
:10575000059401F0D1FB1EB1012E02D1029400E0AC
:10576000029514486946144A17B102F0EFFD01E0B2
:1057700002F0B2FD4FF0FF310E4802F0FDFD0D4882
:1057800002F0F2FD0B4802F0F2FD0C4B4FF4004228
:105790001021C3F8802183F80F131A60FFF770FF00
:1057A00007480121FEF7DCFF0248082102F0E2FD74
:1057B00007B0F0BD008002400048E80100E100E0D1
:1057C0000081024007B500228DE8030008486946C1
:1057D000FEF7B0FF06484FF48071FEF7C1FF0448A2
:1057E000FEF7CEFF0028FAD103B05DF804FB00BF3E
:1057F0000081024038B5154B154D1A88154892B2F4
:10580000AC5C1A8808210132C2F308021A8002F047
:10581000B3FD114BE4B21A88013A92B21A800F4BD1
:105820001B7863B10E4A0F4913889BB22B440B605F
:1058300001234B6013880133C3F308031380054829
:10584000082102F097FD204638BD00BF86480020A1
:1058500088480020008002408448002082480020C0
:10586000884A00200081024038B5074D08212846AB
:1058700002F082FD054B28461C880821A4B202F0E4
:1058800079FD204638BD00BF0080024084480020DA
:1058900010B5064C0821204602F06EFDFFF7F0FE21
:1058A0002046BDE81040082102F064BD008002409F
:1058B0000F2001F03FBB0F2001F01EBB10B5284B9D
:1058C00086B01870274B0A461970274B28B1274A13
:1058D00092E8030083E8030004E0254903C983E854
:1058E00003002AB146210C22224806F019F914E0DF
:1058F0002149204CC87A8B7A4A7A0090097B03A808
:1059000001911E4905F05EF930212046042206F07F
:1059100007F903AB03CB6060A160194C002023683A
:10592000DB6E9847174B186023681B6E984701225F
:10593000154B10B115490A7002221A7000F016FFBB
:1059400002F050F908B902F087F91320192103F089
:105950000BFB4FF40040002103F09AFA06B010BD93
:10596000087200208E4A0020F4710020402F002091
:105970005C250020FC71002038720020A7DA41006D
:105980002C720020F07100208A4A00208B4A0020EF
:1059900008B50B4B1B780BB1FEF7A8FD04F090FF88
:1059A00030B902F07BFF014610B9802003F070FA95
:1059B000BDE808404FF40040002103F069BA00BF81
:1059C0008C4A0020014B1870704700BF8D4A0020A0
:1059D00008B5074B1B78012B04D1064B1B68D3F885
:1059E00090309847BDE808401320192103F0BCBA55
:1059F0008A4A00202C720020013838B54D1E0C1840
:105A0000A54208D000F0D2FD0028FBD015F8010F08
:105A100000F006FEF4E738BD00F006BE00F005BE5B
:105A200008B5064B1B7843B1054B1B782BB102F030
:105A300069F9BDE8084000F003BE08BD8C4A0020AB
:105A40008F4A0020164B174A187830B5937820B14A
:105A5000042B05D0052B1FD105E0042B03D030BD4E
:105A60000D23114901E0114910230C46104D14F883
:105A7000010B25F8020B601AC0B29842F7D30D490A
:105A80005B0002330B709BB293819160D28893428A
:105A900004D9044B9A8101E0002030BD012030BDC3
:105AA0000872002014720020BE2E0020AD2E0020AF
:105AB000CE2E0020CC2E0020014B01201870704704
:105AC0008C4A0020014B00221A7070478C4A00203B
:105AD000014B0120187070478F4A0020014B0022B3
:105AE0001A7070478F4A002008B100F09FBD00F087
:105AF0009EBD000007B500F0EBFC80B100F024FD76
:105B0000084B02A91B7801F8010D23B108460121B9
:105B1000FFF758FEEFE7012003F0F0F8EBE703B0E2
:105B20005DF804FB924A002008B50B4B1B781BB1B3
:105B3000BDE80840FFF7CEB9084B1B780BB1022037
:105B400008BD03F0C1F80028F9D1054B1B689B6F15
:105B50009847C0B208BD00BF8B4A00208D4A002084
:105B60002C72002008B5064B1B781BB1BDE808401D
:105B7000FFF7C0B9034B1B68DB6F9847C0B208BD85
:105B80008B4A00202C72002008B5084B1B781BB1F3
:105B9000BDE80840FFF7B8B9054B1B68D3F8803063
:105BA0009847003018BF012008BD00BF8B4A002075
:105BB0002C720020034B1B780BB1FFF7A7B9FFF73E
:105BC00067B800BF8B4A0020034B1B780BB1FFF76F
:105BD000C7B9FFF77FB800BF8B4A00200A4B0821E6
:105BE00018701A68084852001A60DA78D20741BF64
:105BF000B0F8012082F4815282F00102A0F8012065
:105C00000139EED1704700BF09720020024B4FF0FE
:105C1000FF325A709A70704709720020014BB3F836
:105C20000100704709720020F8B50D4B07460E467B
:105C30001C464FF0FF325A709A700025ABB2B34247
:105C400005F1010503D2F85CFFF7C8FFF6E7002075
:105C5000FFF7C4FF0020FFF7C1FFB4F80100F8BD53
:105C60000972002008B5094B1A780A2A0AD10120C6
:105C7000FFF7A8FE03F0E6FB03F08EFCBDE808404A
:105C800003F0ECBE00221A7008BD00BF914A00204C
:105C900003F030BE08B503F061FE04F01BF80D4BB5
:105CA00018601A680C4B1B689A4204D3A4200B4955
:105CB000002203F0BFF803F0FDF830B9084B1B7861
:105CC0001BB903F04DFE04F001F8BDE8084003F0F5
:105CD00047BE00BF10720020000C0000B8DA41007F
:105CE000934A002004F00FB908B503F0F3FF034B0B
:105CF0001860032004F007F9FBE700BF10720020D2
:105D0000FFF77ABE08B504F0E5F8FDF75DFA044B3D
:105D100001221A701020BDE8084003F051B900BFFD
:105D2000904A002038B5394B04461B780D4653B1D4
:105D300002296AD1002868D1354A142013786421D9
:105D40000133137016E0FDF7FDFF14B1012C3CD0B8
:105D500038BD012D12D002D3032D1ED038BD2046F0
:105D6000012104F0EBF82B4B1B78002B4DD11020B8
:105D70004FF4C871BDE8384003F0F6B8204621461C
:105D800004F0DCF80C2003F03DF900283DD004F0CD
:105D9000A3F8BDE8384003F0AFBE1E4D287860B9C7
:105DA000014604F0CBF804F095F8102003F008F950
:105DB000FDF70AFA01232B7038BD2046214604F076
:105DC000BDF8BDE83840FDF729BA032D1DD8DFE83E
:105DD00005F0020814180F4B1B78B3B101200146DF
:105DE00007E0FCF7EBF9014610B10D209621C1E761
:105DF0000120BDE8384004F0A1B8BDE83840FDF707
:105E000083BFBDE83840FCF73FB938BD934A002056
:105E1000914A0020904A002008B504F05DF8BDE8E2
:105E2000084003F069BE002004F0CABD002004F061
:105E3000F5BD0120002104F081B8012004F0C0BDAF
:105E4000012004F0EBBD000008B5064B1B782BB910
:105E500004F042F8BDE8084003F04EBEBDE808403B
:105E6000FDF7DCB9904A002003F032BF10B50446BC
:105E700003F074FD054B20461B681B6F98470446D2
:105E800003F06EFD201C18BF012010BD2C720020F5
:105E900038B5324B1B78002B3FD104F013FD052899
:105EA00003D1BDE8384003F027BEFFF7A6F810B9CC
:105EB0000120FFF717FF002004F0B6FD0C2032216F
:105EC00003F052F803F0D2FD01F008F8FBF7CEFB27
:105ED00010204FF4C87103F047F8214B5B780BB1E9
:105EE00003F00AFE012004F0A9FD062003F0DCF90E
:105EF00018B1BDE8384003F0FDBE072003F0D4F927
:105F000018B1BDE83840FDF7CFBB082003F0CCF94D
:105F100010B3BDE8384003F05DBF03F0C4FF0120BB
:105F200003F096FD012003F0BFF90446052003F0BD
:105F3000BBF90546092003F0B7F920B1FBF782FB56
:105F4000084B01241C7020462946FFF7B7FCBDE82A
:105F50003840012004F072BD38BD00BF934A0020D4
:105F600000F84100924A00201FB503F0D5FD04F06F
:105F7000A7FC274B274C187002F0A6FF02F0B0FBDD
:105F8000FEF7A6FFFBF7E8FFFCF7B5FC03F082FB8A
:105F900004F00AFD002003F085FF04F051F904F03D
:105FA000C1FBFFF72AF823689B6D9847022801D0B0
:105FB00003F070FD236801A81B6898470A2003F0CE
:105FC00073F928B101A803F011FC134803F018F984
:105FD00002A8FFF74BFF022003F066F930B10F482B
:105FE00003F00EF904F060F803F038FD042003F02C
:105FF0005BF930B10A4803F003F903F023FA03F028
:106000002DFD04F0A9FB02F017FF002004B010BD25
:10601000934A00202C720020D3DA4100E0DA4100DC
:10602000EFDA410010B503793C2B31D843793C2B92
:106030002ED88379172B2BD841780139C9B20B2977
:1060400026D8037823B301228A4040F6D521114097
:1060500031B912F4A56F05D112F0020204D117E094
:106060001F2B18E01E2B16E04288910712D16424E2
:10607000B2FBF4F104FB112189B239B94FF4C874B1
:10608000B2FBF4F104FB112292B21AB91D2B02E00B
:10609000002010BD1C2BFBD8024B1B685B6F984780
:1060A000012010BD2C72002008B5002000F0DAFE9F
:1060B00000F0FCFE0028FBD008BD000008B5FFF78B
:1060C000F3FF00F00BFF074A074BDA6200F00CFF0A
:1060D0000028FBD0012000F04BFFBDE8084000F095
:1060E00051BF00BF023F0F0000040E4008B5FFF78C
:1060F000DBFF00F0E3FE084A084B9A6200F0E6FE80
:106100000028FBD0102000F07FFE02F071FA044B53
:106110004FF480721A6008BD033F0F2000040E4048
:10612000000A0E400120704708B9FFF7FDBC0120AE
:10613000704710B90846FFF715BD0120704708B930
:10614000FFF722BD012070470028024818BF002039
:10615000704700BF40DB410070B506460D4614464F
:1061600000F066FA2EB921462846FFF723FD0446C3
:1061700000E0012400F05EFA204670BD70B50646CE
:106180000D46144600F058FA2EB921462846FFF76E
:106190001BFD044600E0012400F050FA204670BDCB
:1061A000034B187872B6BFF35F8F00221A707047E6
:1061B000F02F002070470020704700207047704784
:1061C00028B1034B01221A70BFF35F8F62B670478C
:1061D000F02F00200D4A002313800D4AA1211170D9
:1061E00020215170022153809380D1801381094A6C
:1061F0006FF03D0113705170D37001211371537111
:10620000082391709371FFF763BC00BFBA4F002061
:106210002C4D0020944A0020244BF7B51A781D46D7
:10622000002A40D101F044FD214E348880B101F0B4
:1062300071FD844237D0FFF7B3FF1E491E4B0C7827
:106240001B78E4B23BB9B4FA84F35B090B7005E048
:1062500001F058FDEDE7B4FA84F4640901232B70D2
:10626000FFF7AEFF154B33F814501F46B5F5A07578
:1062700018BF01254DB101F01BFD10B101F04AFD21
:1062800001E001F03FFD308000E035800C4A37F836
:10629000143000920B4A29464FF4A075842005FB68
:1062A000042201F0B9FE03B0F0BD00BF2A4D00206A
:1062B000264D00209B4A0020B94F00209C4A002018
:1062C000CD624100A04A0020FFF7A6BF68B9074B86
:1062D000074A1B78B3FA83F35B0922F81300054BD6
:1062E0001870054B1870FFF797BF70479B4A002046
:1062F0009C4A0020B94F00202A4D0020024B00226A
:106300001A70FFF7EBBB00BF294D002008B5144BF6
:106310001A7812F0800F02F0600208D0202A1DD1F6
:106320005A78212A1AD1DA88072A17D111E0202AAF
:1063300014D15A78202A07D0222A0FD1987800F059
:106340000100FFF7D1FB07E0DA88072A06D10549EB
:10635000196105499A819960012008BD002008BD96
:1063600014720020BF614100944A0020064A074B86
:106370001B881178064A9BB232F81100984294BFEC
:1063800000200120704700BF284D0020244D002030
:10639000204D0020F7B5FFF703FF1949194A0C7883
:1063A00013780746E4B203F0FF0543B9164EDFF851
:1063B00064E033883EF814E09BB29E4504D9384629
:1063C000FFF7FEFE002019E0B4FA84F35B09358084
:1063D0000B7001231370FFF7F3FE2846FFF7C6FF8B
:1063E00008B1FFF787FB094A4FF4A0730092084AEF
:1063F0000520012103FB042201F00EFE03B0F0BDD5
:10640000284D0020B84F0020244D00207D6441001D
:10641000384D0020204D00200E4B10B500241C707C
:106420000D4B1C700D4B1C700D4B1C805C800D4B7C
:106430001C80FFF7F1FE0C4B1C700C4B1C700C4BBE
:106440001C800C4B1C80FFF7A5FF0B4B18701878B5
:1064500010BD00BF2A4D0020B94F00209B4A0020EC
:106460009C4A0020264D0020B84F0020284D0020D7
:10647000204D0020244D0020294D002013B5D8B90F
:106480000E4B1A78B2FA82F2520959B90C490D4CE6
:106490004FF4A073009103FB02420121052001F09B
:1064A000BBFD09E0084B23F81210084B187002B02E
:1064B000BDE81040FFF76EBF02B010BD284D0020B0
:1064C0007D644100384D0020204D0020B84F002051
:1064D0000020FFF74BBF000038B5154B00249D7915
:1064E000A5F109035D425D411249134B0A881B78EF
:1064F0001248DBB230F8130092B2904206D8104B2B
:106500001B7803F0FF00002BEED138BD4FF4A070D4
:1065100000FB03230B480132C35C92B21C430A8088
:10652000FFF738FF15B124020025DDE7204638BD0E
:10653000944A0020244D0020284D0020204D0020AA
:10654000294D0020384D00200020FFF7C5BF000076
:1065500070B5124C124B22781E4633F81220B2F559
:10656000A07F18D10F4D2B786BB9FFF719FE0E4B9A
:106570001B7833B901232B702378B3FA83F35B09BB
:106580002370FFF71DFE237836F81300B0F5A070D6
:1065900018BF012070BD012070BD00BF9B4A0020C4
:1065A0009C4A0020B94F00202A4D00200020FFF710
:1065B000CFBF000070B50D46144B9C79A4F10903C0
:1065C0005C425C410020FFF7C3FF30B9104B1B78E1
:1065D00003F0FF00002BF5D170BDFFF7E1FD0D4B7F
:1065E0000D491B78DBB231F81320561C21F81360DB
:1065F0004FF4A07101FB0323084AD554FFF7E0FDD7
:1066000014B12D120024DDE7012070BD944A002052
:10661000294D00209B4A00209C4A0020A04A0020CF
:1066200001460020FFF7C6BF7047704770477047AC
:1066300003F03CBC03F044BC03F038BC03F040BCA6
:1066400070470000024B987800F07F0001F032BBE9
:106650001472002030B5114B1B780BB9002030BDEF
:106660000F4B1B681B681A798242F7D90D4A1360D9
:106670005C881C449C420ED95D78042D08D19D781D
:10668000854205D1DD788D4202D11360012030BDF5
:106690001D782B44EEE71360E0E700BFC34F0020F6
:1066A000BC4F0020C84F0020084B1B681A68538855
:1066B0001A4403781844824205D94378042B02D047
:1066C000052BF6D100E00020704700BFBC4F002032
:1066D00070B50546FFF7BEFFB8B10D4B1C682046EC
:1066E000FFF7E2FF044638B18078E178A28801F034
:1066F00019FB0028F3D108E0064B1B685B6853F8D0
:106700002530BDE870401B681847002070BD00BFF1
:10671000C84F0020BC4F002070B500210446FFF791
:1067200099FF08B900251AE00E4B1B685B6853F807
:106730002460F368984701462046FFF78BFF054623
:106740000028EFD0084B1C682046FFF7ADFF044639
:1067500018B1807801F05AFBF6E77368984728462D
:1067600070BD00BFBC4F0020C84F002001F03CBAF4
:1067700038B50A4B1A781C4622B90023084A237000
:10678000138038BD0025074BE8B21B6801351B6834
:106790001B798342F1D9FFF7BFFFF4E7C34F002015
:1067A000C04F0020BC4F002010B50A4B1B7803B926
:1067B00010BD0024084B1A6813681979E3B2994296
:1067C00007D9526852F823301B6903B19847013446
:1067D000F0E710BDC34F0020BC4F00202DE9F04171
:1067E000964C0023A3812361636123785AB2002A67
:1067F00003DAE188002900F06F8113F0600140F0B6
:106800004281002A80F29E80E5888C4E002D00F0A7
:106810003A8113F01F035ED17378062B09D0082B41
:1068200051D0002B40F02F81022D40F02C81844864
:106830004DE073881D0A022D08D0032D16D0012DBE
:1068400040F021817F4B1868017832E07D4ADBB24D
:106850001168497C994240F21681526852F833001F
:10686000418801F059FAB3685D7024E0DBB2032B74
:106870000BD8DFE813F007000E0004002B011021F5
:10688000714B08E07148042113E0FFF7DBF890B981
:10689000F9E06F4B0A211A466E4D12F8010B25F8EC
:1068A000020BD01AC0B28842F7D349006A480231BD
:1068B000017001F031FAE388A2899A4240F209811D
:1068C0005E4A938105E1012D40F0DD806348294651
:1068D00001F022FAFDE0012B23D173780A2B40F05E
:1068E000D280012D40F0CF805C4B1B78002B00F054
:1068F000CA805B4B35791E6833681B79AB4240F226
:10690000C2802846FFF7A6FE002800F0BC8073680E
:1069100053F82530DB689847524B01211870184610
:10692000D6E7022B40F0AF807378002B40F0AB80AD
:10693000022D40F0A880307901F088FA4A4B188087
:106940001846C4E713F01F034ED16378013B082BB0
:1069500000F29980DFE803F00D97979705979797D6
:106960001C00E388002B40F08E80404A334B1A61B4
:10697000AFE0E388002B40F08680304B5B88012B32
:1069800040F081802E4A138823F002031380A0E098
:10699000E5882A4F002D76D101F0A8F9002872D0A1
:1069A000284EBA7833685B7C9A426CDCFFF7E0FED5
:1069B000BB782A4A1370002B00F08B80284A71683C
:1069C000164603F10053013B01EBC3031360336828
:1069D000E8B21B681B7983427BD90021FFF778FE60
:1069E00001350028F3D14EE0012B16D16278134B0C
:1069F0000B2A48D1DA88002A45D1184A1278002A91
:106A000041D01D795E882846FFF786FE00283AD0DF
:106A10002846F1B2FFF75CFE34E0022B33D16378F5
:106A2000064D012B02D0032B22D02CE0EB8853BB68
:106A30006B8843BB287901F087FA23E014720020A9
:106A4000C04F0020F4710020AA2F0020EC2F00205E
:106A5000BB2F0020CA2F0020C82F0020C34F0020CA
:106A6000BC4F0020C24F0020C44F002045664100AB
:106A7000EB8843B96B8833B9287901F055FB287945
:106A800001F00CFA48BB237803F01F03012B23D13C
:106A9000134B1B7803B3134B1C79134B1D682B68E6
:106AA0001B79A34218D920460021FFF7D3FD98B1E6
:106AB0006B6853F82450EB68984701462046FFF76F
:106AC000C9FD48B1AB68BDE8F04118470C21074B40
:106AD000E1E60120BDE8F0810020BDE8F08100BFC3
:106AE000C34F002014720020BC4F0020FC71002016
:106AF000B1F1C05F10B542642DD007D8B1F1006F7D
:106B000015D0B1F1805F1DD071BB10BDB1F1205F18
:106B10002BD005D8B1F1005F26D1036F13431FE0DE
:106B2000B1F1405F21D0B1F1605F1ED01CE0D343D2
:106B3000016F046F214019400167416F446F21408C
:106B40000B4010E0036F13430367436F416F0B402B
:106B500023EA020307E0036F016F0B4023EA0203FD
:106B60000367436F13434367426010BDD30741641B
:106B70004CBF4166016612F00A0F14BF0162416208
:106B8000930702D5C0F8801003E0130748BFC0F890
:106B9000841041610160704710B5029C41640CB1E2
:106BA000416600E001660BB1016500E041650AB194
:106BB000016300E041630161016010BDB1F1005F5C
:106BC000F7B507460C4615461E4618D009D8B1F150
:106BD000805F14D0B1F1C05F11D0B1F1006F27D147
:106BE0000DE0B1F1405F14D0B1F1605F11D0B1F1AF
:106BF000205F1DD111461A46FFF7B8FF16E02A465E
:106C000038462146FFF774FFF2074CBF7D663D66AC
:106C10000CE006F00103009304F148435A425A4144
:106C200038462946C6F38003FFF7B6FF012000E08F
:106C3000002003B0F0BD12B1C0F894107047C0F846
:106C400090107047D3060ED59306C0F8B0104CBF15
:106C5000C0F8D410C0F8D01053064CBFC0F8C01014
:106C6000C0F8C4107047C0F8B4107047C36C01641A
:106C7000704741647047C06C7047806C704743092F
:106C800003F5001303F207735B02DA6B00F01F03D6
:106C900022FA03F000F001007047430903F50013E6
:106CA00003F2077300F01F0001225B0282401A63A7
:106CB0007047430903F5001303F2077300F01F0048
:106CC00001225B0282405A637047F7B545090E46C0
:106CD00005F5001501F0F04105F20775B1F1005F0F
:106CE0004FEA45251ED009D8B1F1805F1AD0B1F125
:106CF000C05F17D0B1F1006F37D113E0B1F1405F41
:106D00001FD0B1F1605F1CD0B1F1205F2DD100F038
:106D10001F030124284604FA03F13246FFF726FF39
:106D2000204623E000F01F00012404FA00F73A4651
:106D30002846FFF7DDFEF20701D42F66F0E76F6605
:106D4000EEE7012406F0605206EA0403009302F124
:106D500048435A4200F01F015A41284604FA01F103
:106D6000C6F38003FFF718FFDAE7002003B0F0BD99
:106D700070B505460E46FFF77EFF04462846FFF72E
:106D80007CFF044012D00A4D55F80C3CB3420AD1A6
:106D900055F8081C214206D02B683046984755F814
:106DA000083C24EA03041035002CEDD170BD00BF6F
:106DB000DC4F0020F8B50C4E3468062C12D8DFF8F2
:106DC0002CE027014EF8071006990EEB07056A60C4
:106DD000E960AB60114601341A463460FFF732FFB8
:106DE0000020F8BD0120F8BDCC4F0020D04F00207E
:106DF00001480B21FFF7BCBF000E0E4001480C21DB
:106E0000FFF7B6BF00100E400F4B1A6B22F0700256
:106E1000104340F601021863986E0B49000703D433
:106E2000013AF9D1012070470A6B22F0030242F0C7
:106E300002020A6340F60102996E090702D4013A80
:106E4000FAD1EFE70020704700040E40044A136AAD
:106E500023F45C1323F0080343F45C1313627047BC
:106E600000040E400C4B1A6A28B10C4911400C4A20
:106E70000A431A6270470B4911400B4A0A431A62CF
:106E8000996E054AC907FBD5136A43F09B7343F417
:106E900080331362704700BF00040E40FCFFC8FE41
:106EA00002003701FCC0C8FF013F3700024B986E5B
:106EB00000F48030704700BF00040E40024B4FF0DA
:106EC00000529A62704700BF00040E40024B986E59
:106ED00000F00200704700BF00040E40014B00228A
:106EE000DA62704700040E40024B986E00F0040016
:106EF000704700BF00040E40222815D81F280C4AF6
:106F00004FF0010306D891698340194099420DD092
:106F100013610BE0D2F808112038834019409942E0
:106F200004D0C2F8003101E0012070470020704712
:106F300000040E40222815D81F280C4A4FF00103E8
:106F400006D891698340194099420DD151610BE0F7
:106F5000D2F80811203883401940994204D1C2F870
:106F6000041101E0012070470020704700040E402A
:106F7000000200F47060024B40F00100986370471B
:106F800000040E40014B80221A60704700040E403E
:106F9000014B80225A60704700040E40034A000CE7
:106FA000136F000403431367704700BF00040E40D3
:106FB000034B187872B6BFF35F8F00221A707047C8
:106FC000F02F0020034A0023136153619381024A8A
:106FD0001370704714720020AD5000200D4B052235
:106FE0001A700D4A82B0136B0093009B43F04F035D
:106FF0000093009B43F020030093009B1363002346
:107000000193019B0E2B03D800BF019B0133F7E7CF
:1070100002B07047AD500020004003400D4B0322EA
:107020001A700D4A82B0136B0093009B43F04F031C
:107030000093009B43F010030093009B1363002315
:107040000193019B0E2B03D800BF019B0133F7E78F
:1070500002B07047AD50002000400340024B1B6956
:1070600003B11847704700BF1472002070B5840048
:1070700004F1402404F54034236B421E03F0420324
:10708000422B164B0ED0216B11F0020F4FF0140162
:1070900001FB02314D7C0ABF01266FF3830566F3C5
:1070A00083054D74142101FB02335A7C12F00C0F3E
:1070B000226B0AD122F00202226368B103280BD0AE
:1070C0005A7C012161F3830205E022F04002226331
:1070D0005A7C6FF383025A7470BD00BF4450002085
:1070E0002DE9F347614E431E142202FB036292F81E
:1070F00011C0CCF3810C20B103280CBF0122022265
:1071000000E00122944501DB0120ABE0142202FBE8
:107110000362D768D2F808E0774507D3547C04F0BF
:10712000400404F0FF02002C00F09B80142202FBBC
:1071300003625468128A04EB0709C2F30902C7EB21
:107140000E04944238BF22464FF0140404FB03643B
:10715000174434BF4FF001084FF00008E76009F111
:10716000080502F10804641B4C44072C26D984004E
:1071700015F808AC04F1402404F54034C4F850A0DC
:1071800015F807AC0835C4F850A015F80EACC4F8D3
:1071900050A015F80DACC4F850A015F80CACC4F80C
:1071A00050A015F80BACC4F850A015F80AACC4F800
:1071B00050A015F809ACC4F850A0D2E722F007049B
:1071C0004C4402F007022244944208D014F801AB68
:1071D000DFF89C9000F1140549F825A0F4E714228B
:1071E00002FB0362547C0CF1010C6CF383045474B5
:1071F00051B9B8F1000F21D0142202FB0362517C77
:107200006FF38611517419E0800000F1402000F501
:107210004030026B0092009A42F04F020092009AB6
:1072200042F010020092009A026300220192019A39
:107230000E2ADED800BF019A0132F7E77745FFF446
:1072400063AF142202FB03635A7C02F0400202F097
:10725000FF00002A7FF458AF5A7C42F080025A7433
:1072600000E0104602B0BDE8F08700BF44500020A7
:107270000040034028B1034B01221A70BFF35F8F17
:1072800062B67047F02F00202DE9F043614E8BB0BD
:107290003378032B1AD1604A136B0093009B43F0A1
:1072A0004F030093009B23F001030093009B1363A3
:1072B00000230193019B0E2B03D800BF019B0133D8
:1072C000F7E7FFF7CBFEFFF77DFEA0E0022B00D033
:1072D000FEE7524F524D3988AC89641AA4B2002C93
:1072E00028D1504A13880B449BB21380EA889A42F3
:1072F00002D04D4B1B78BBB1474A04233370136B4C
:107300000293029B43F04F030293029B23F001037D
:107310000293029B136300230393039B0E2B76D8E7
:1073200000BF039B0133F7E76B6953B1984740B146
:107330003C80AC893F2C04D93B4B00221A7040247E
:1073400002E0394B01221A70B7F80080AD68FFF7F0
:107350002FFEDFF8C4904544D9F8303002469B0731
:1073600001D429461AE0FFF785FF04233370D9F8CA
:1073700030300493049B43F04F030493049B23F0A9
:1073800001030493049BC9F8303000230593059B47
:107390000E2B3CD800BF059B0133F7E74B1BDBB23C
:1073A000A3421D4803D211F8013B0365F6E7036BC6
:1073B00044440693069B3C8043F04F030693069B90
:1073C00043F010030693069B036300230793079B78
:1073D0000E2B03D800BF079B0133F7E70E490B6B59
:1073E0000893089B43F04F030893089B23F0010385
:1073F0000893089B0B6300230993099B0E2B03D86A
:1074000000BF099B0133F7E71046FFF733FF0BB0CE
:10741000BDE8F083AD50002000400340AA5000209A
:107420001472002040500020AC500020437C30B546
:107430000446D80614D56FF30413637423687BB134
:10744000084802F10C0550F825000139050648BF2F
:1074500042F0800248424841A168BDE830401847E8
:1074600030BD00BF004003402DE9F04F2220A5B001
:10747000FFF742FD934B9A6912F4006F1A460AD047
:10748000D9690E0507D54FF400621A62FFF78CF92F
:10749000FEF7C6FA9BE3D2698A4BD50740F13581E6
:1074A0001A6B540740F1A180874D2B781BB1FFF771
:1074B000D5FDFFF787FD834C236BC3F30A43082BED
:1074C00017D0FFF78BFD236B0493049B43F04F030E
:1074D0000493049B23F004030493049B236300237D
:1074E0000593059B0E2B00F2728300BF059B0133B1
:1074F000F6E70023734C754E226DB0469A55013362
:10750000082BF7D1FFF76AF90746B8B9FFF766FD10
:10751000236B0693069B43F04F030693069B23F0D1
:1075200004030693069B23630797079B0E2B00F229
:107530004E8300BF079B01330793F6E796F90030AF
:10754000002B236B31DA0893089B43F04F03089319
:10755000089B43F080030893089B2363002309934F
:10756000099B0E2B03D800BF099B0133F7E7554A4F
:10757000136B0A930A9B43F04F030A930A9B23F071
:1075800004030A930A9B136300230B930B9B0E2B9C
:1075900003D800BF0B9B0133F7E74D4A002313804C
:1075A0004C4A138002232B7022E00C930C9B43F077
:1075B0004F030C930C9B23F004030C930C9B23634D
:1075C00000230D930D9B0E2B03D800BF0D9B0133A1
:1075D000F7E7B8F80630002B55D03D4A002313805A
:1075E0003C4A138001232B70F1E21A6BD00702D5BD
:1075F000FFF74AFEEBE21A6B12F002026CD0324A3D
:107600001278012A10D0022A01D0042A02D1FFF7F1
:1076100025FD01E0FFF7E2FC2A4A136B23F0020389
:107620001363FFF7CFFCD2E22A4C1A6B274823885A
:10763000C2F30A4281899D18A942B8BFCA1A81685B
:1076400092B219440E46751AEDB2954204D21D4D00
:107650002D6D06F8015BF6E713449BB2402A1D4EE0
:10766000238006D11A4DC4882A8818491A449442A6
:107670000CDC83814369134C0BB1984770B1236BC9
:1076800023F002032363FFF7C9FCA0E28A899A4230
:1076900011D14B690B4C0BB1984730B9FFF79EFCE9
:1076A000236B23F00203236391E232882B88134477
:1076B0002B8000233380034A136B23F002031363F0
:1076C00085E200BF00400340AD500020147200204E
:1076D00040500020AA500020196B090715D5196BDE
:1076E0000291029941F04F010291029921F00801A3
:1076F0000291029919630392039B0E2B00F2678299
:1077000000BF039B01330393F6E7A64B01261978CC
:1077100000290CBF4FF0020E4FF0050EA24B4FF0A8
:10772000010B9B690BFA06F818EA030F00F0AA8117
:10773000B40004F1402505F54035286B9B4B771EBE
:107740004FF0140A10F042000AFB073A994641D064
:107750002C6BBAF81010C4F30A44DAF80830DAF8DF
:107760000C00C1F30901DAF80420ACB11B1A9C42E9
:1077700038BF23464FF0140E0EFB079E02441844F8
:1077800038BF4FF0000BCEF80C0013449A4204D0DF
:10779000286D02F8010BF9E7A34630460191FFF787
:1077A00065FC0199BBF1000F02D18C4280F00F8281
:1077B000296B11F0200140F00A827B4B5046C3F840
:1077C0001480142303FB0797FB683246BB60FFF766
:1077D0002DFEFCE12B6B13F0010200F032810AF167
:1077E00010025378C3F38101033161F383035370B3
:1077F000DBB203F0200E0EF0FF01BEF1000F5ED0F1
:1078000013F00C032AD02B6B0E930E9B43F04F0307
:107810000E930E9B43F010030E930E9B2B630F9061
:107820000F9B0E2B04D800BF0F9B01330F93F7E77C
:107830002B6B1093109B43F04F031093109B23F07E
:1078400001031093109B2B6300231193119B0E2BAC
:1078500000F2BD8100BF119B0133F6E72A6B129243
:10786000129A42F04F021292129A22F001021292E0
:10787000129A2A631393139B0E2B03D800BF139BFA
:107880000133F7E72B6B1493149B43F04F031493CE
:10789000149B43F020031493149B2B630023159334
:1078A000159B0E2B03D800BF159B0133F7E714235C
:1078B00003FB07977B7C6FF345137B7487E11B0603
:1078C0000BD55378504661F3C7135370DAF80C3078
:1078D0003246CAF80830FFF7A9FD142303FB0793CB
:1078E000D9689A68914224D35D7C15F04C0520D16B
:1078F000FFF75EFB2C4B04F14024C3F8148004F521
:107900004034FFF7B7FC236B1693169B43F04F03ED
:107910001693169B23F001031693169B236317956A
:10792000179B0E2B00F2538100BF179B0133179357
:10793000F6E7032E6AD0142303FB079707F110051F
:107940006B7813F00C0F33D004F1402404F540346D
:10795000236B1893189B43F04F031893189B43F025
:1079600010031893189B236300231993199B0E2B64
:1079700003D800BF199B0133F7E7236B1A931A9BB7
:1079800043F04F031A931A9B23F001031A931A9B97
:10799000236300231B931B9B0E2B32D800BF1B9B22
:1079A0000133F7E7087200200040034044500020F4
:1079B00001213046FFF794FB014648B96B78324607
:1079C00060F3C7136B70FB685046BB60FFF72EFD7A
:1079D00004F1402404F54034236B1C931C9B43F0BA
:1079E0004F031C931C9B23F001031C931C9B2363DC
:1079F00000231D931D9B0E2B03D800BF1D9B01333D
:107A0000F7E730460021FFF76BFBE0E0304601214D
:107A1000FFF766FB6F4A136B1E931E9B43F04F03E9
:107A20001E931E9B23F001031E931E9B13630023D2
:107A30001F931F9B0E2B00F2CA8000BF1F9B0133B8
:107A4000F6E72B6B1F071DD52B6B2093209B43F074
:107A50004F032093209B23F008032093209B2B634C
:107A60002192219B0E2B04D800BF219B013321932F
:107A7000F7E72B6B03F4E063B3F5807F00F0A7809A
:107A80002B6BA4E00136F6B276457FF647AE524B3B
:107A90009A69920402D5DA6994040DD49B69980519
:107AA00003D54D4BDB699A0506D44B4A93695B05B8
:107AB00015D5D3695F0512D5474C4FF400514FF4EB
:107AC00000724FF48063216222622362616162610D
:107AD0006361424B01221A70FDF7A0FF71E09269C9
:107AE0003D4BD50518D5DA69D40515D54FF480720C
:107AF0001A625A614FF400521A614FF400721A610F
:107B00004FF480621A612220FFF714FA334B0022EF
:107B10001A70FDF781FF5AE02F4BDA69D00456D571
:107B200000294FF480521A6214BF05260226002352
:107B30005D1C2B4AECB2142000FB032001212246DD
:107B4000FFF774FCB4422B46F2D3FEF711FE224B32
:107B50005A681C4622F001025A605A6822F002025A
:107B60005A609A6842F480729A609A6822F07F02A2
:107B70009A601A6B2292229A42F04F022292229A23
:107B800022F4074222F080022292229A42F400421A
:107B90002292229A1A6300222392239B0E2B04D84E
:107BA00000BF239B01332393F7E7236B43F4004388
:107BB0002363FFF7FDF901232361FFF75BFBFFF769
:107BC00001FA4FF4807323614FF40063236125B001
:107BD000BDE8F08F0C40034000400340A850002057
:107BE000445000200020704710B5FFF7E1F904462B
:107BF0002220FFF781F9FEF761FA134B502283F838
:107C0000222304225A60114B00221B78002B14BF40
:107C1000052002200E49142303FB0213597C013274
:107C200001F083016FF3C7115974D3B28342F1D3CA
:107C30004FF48020FFF7B2F9064B00222046BDE842
:107C400010401A70FFF716BB00E100E00872002038
:107C500044500020A850002010B5FFF7A9F90446B1
:107C6000114B012222201A70FFF746F90F4B2046D4
:107C7000BDE810405A6F22F480725A675A6F42F47E
:107C800000725A674FF480721A614FF400521A6101
:107C90004FF400721A614FF480621A614FF400626F
:107CA0001A61FFF7E7BA00BFA85000200040034068
:107CB000002070470C4B5A6822F001025A609A6803
:107CC00022F480729A6070B19A6800F07F0022F00E
:107CD0007F02104398609A6842F480729A605A68F2
:107CE00042F001025A60704700400340044B58685C
:107CF00010F001001CBF986800F07F00704700BFC3
:107D000000400340024B1868C0F30A00704700BFF0
:107D10000040034000207047014B986099817047F4
:107D200014720020364BF7B51B7800F00F04002BBF
:107D300014BF052302239C425FD8A50005F140250E
:107D400005F540352B6B13F4004356D101F00306C3
:107D5000012E03D1002C50D0032C4ED0231F012B19
:107D600094BF4FF4007340239A4246DC254F631EB4
:107D70004FF0140E0EFB03731F8A03F1100662F31B
:107D800009071F825B7CC00903F07F036FF3451373
:107D900073701EBFDBB26FF3830373701A4B012243
:107DA0009E6AA24042EA06049C629C6A24EA02029D
:107DB0009A622B6B0093009B43F04F030093009B50
:107DC00023F4074323F080030093009B08B141F0A4
:107DD0000401090201F4E06141F4004119430091FA
:107DE000009B2B6300230193019B0E2B03D800BF44
:107DF000019B0133F7E7012000E0002003B0F0BD54
:107E00000872002044500020004003400D4B00F059
:107E10000F021B78002B14BF05230223934210D3BB
:107E2000930003F1402303F54033196B142021F430
:107E300000411963044B511E00FB01300121FFF783
:107E4000F5BA70470872002044500020104B00F033
:107E50000F001B7810B5002B14BF052302238342AB
:107E600013D30C49431E142404FB03135B7C9B06B1
:107E700009D4094B0C3053F8203013F0280F14BFED
:107E80000120002010BD012010BD002010BD00BF4A
:107E9000087200204450002000400340274B37B5B3
:107EA0001B7800F00F05002B14BF05230223AB4203
:107EB000044640D3FFF77CF8230619D5204B05F183
:107EC0000C0153F821306A1E13F0100F1D4B07D11F
:107ED000142101FB0231497CC1F38101012907DD35
:107EE000142101FB02335A7C42F020025A7419E03B
:107EF000AB0003F1402303F540331A6B0092009A64
:107F000042F04F020092009A42F020020092009A42
:107F10001A6300230193019B0E2B03D800BF019B22
:107F20000133F7E70124064B04FA05F21A61FFF763
:107F3000A1F9204600E0002003B030BD0872002007
:107F400000400340445000207FB5304B00F00F0547
:107F50001B78002B14BF05230223AB4253D32C4ABA
:107F60006E1E142101FB06214B7C6FF345134B74ED
:107F7000AB0003F1402303F54033196B8C0640D569
:107F8000196B0091009941F04F010091009921F087
:107F900020010091009919630021019101990E2996
:107FA00003D800BF01990131F7E71A4C0120A16AFB
:107FB000A8400143A162A16A21EA0000A062196BF6
:107FC0000291029941F04F010291029820F00800BD
:107FD00002900299196300230393039B0E2B03D88D
:107FE00000BF039B0133F7E7142303FB06F153188B
:107FF0005A7CD00605D56FF304125A74044B5B58B3
:108000009847012000E0002004B070BD08720020F5
:1080100044500020004003402DE9F04F1D463F4BE7
:1080200000F00F061B7885B0002B14BF0523022338
:10803000B3428246019102926CD3B30003F1402B0C
:108040000BF5403BDBF8300010F4004063D0741EA9
:108050004FF0140808FB04F8314F07EB080999F8B2
:10806000111001F0200101F0FF00002952D1DBF8CE
:10807000301011F0200303934DD1FEF799FF99F8CA
:1080800011E00EF0100303F0FF0113B1FFF7F2F857
:1080900040E099F811E003914EF0100E89F811E0DC
:1080A000FFF7E8F8029B0399C9F804300E9A019B88
:1080B000C9F80850C9F80C1047F808201BB9B5FAE0
:1080C00085F56D0900E00125142202FB0474627C31
:1080D00065F386126FF3C7126274FEF769FF012120
:1080E000104A05461AF0800F01FA06F010610CD014
:1080F000DBF8303013F0110407D13046FEF7F0FF03
:1081000018B130462146FEF7EBFF2846FFF7B2F8DC
:10811000012000E0002005B0BDE8F08F08720020CB
:1081200044500020004003407FB5424B00F00F0454
:108130001B780646002B14BF05230223A34276D3E7
:10814000FEF736FF01253C4BA5405D61FFF792F835
:1081500036064FD5A30003F1402303F540331A6BD5
:10816000D0060DD41A6B0292029A42F04F0202928C
:10817000029A22F001020292029A1A63002327E077
:108180006CB91A6B0092009A42F04F020092009A6A
:1081900022F010020092009A1A63002210E0032CD1
:1081A000EFD01A6B22F010021A631A6BD106FCD4BE
:1081B0001A6B42F010021A631A6BD206FCD5E0E784
:1081C0000192019A0E2ACDD800BF019A0132F7E739
:1081D0000393039B0E2B03D800BF039B0133F7E7E8
:1081E0001649631E142000FB03135A7C6FF38302AD
:1081F0005A740BE0104B04F10C0253F8223013F0C8
:10820000420F03D02046FEF731FFF3E70A4B14205C
:108210009A6A01212A439A629A6A22EA05059D62B6
:10822000064B621E00FB02302246FFF7FFF804B047
:1082300070BD00BF08720020004003404450002081
:10824000174B00F00F021B7810B5002B14BF05234D
:108250000223934222D3940004F1402404F54034D5
:10826000236B13F400401AD00E4B013A142000FB8C
:108270000230407C10F0100F10D1246BA40601D402
:10828000800608D5142042439818447C995044F045
:108290001004447400E08847012010BD002010BD88
:1082A00008720020445000200A4BC0F8E43000233C
:1082B00043604362836288230360242303604FF496
:1082C000807303604FF4002303604FF400330360B6
:1082D000704700BF00415355F8B50D460646144699
:1082E000FFF7E2FF184900230B6055B32A68B4EB8F
:1082F000021F2CBF102008204243E40004EB52046C
:10830000B4FBF2F44FF6FE72E3085F1E974218D8F2
:10831000082808BF726804F0070404BF42F4002272
:10832000726043EA0444AA686B6834621A432B699A
:1083300000201A43EB68134372680B6013437360A9
:10834000F8BD0120F8BD00BFB050002010B50446B4
:10835000FFF7C2FF30B9636823F00F0343F0020355
:10836000636010BD012010BD4023036070471023DF
:108370000360704781607047C16070474069704713
:108380004069C0F34000704743699B0743BFC1F396
:108390000801C1610020012070470000332002491C
:1083A000002200F047BD00BFB9DC41003420024983
:1083B000002200F03FBD00BFDCDC41003520024957
:1083C000002200F037BD00BF15DD41003620024914
:1083D000002200F02FBD00BF47DB410037200249DB
:1083E000002200F027BD00BF70DB410038200249A9
:1083F000002200F01FBD00BFACDB41003920024964
:10840000002200F017BD00BF3DDD41003A200249C7
:10841000002200F00FBD00BF16DC41003B200249E6
:10842000002200F007BD00BF5DDC41003E20024994
:10843000002200F0FFBC00BFCADC41003F2002491F
:10844000002200F0F7BC00BF53DD4100402002498C
:10845000002200F0EFBC00BFF3DC410041200249E4
:10846000002200F0E7BC00BF04DD410042200249C9
:10847000002200F0DFBC00BFE2DB410043200249E4
:10848000002200F0D7BC00BF05DC410044200249B7
:10849000002200F0CFBC00BF4CDC41004520024967
:1084A000002200F0C7BC00BF72DC41004620024938
:1084B000002200F0BFBC00BF5DDB41005320024939
:1084C000002200F0B7BC00BFCFDB410054200249BE
:1084D000002200F0AFBC00BFF3DB41005520024991
:1084E000002200F0A7BC00BFA7DC410056200249D3
:1084F000002200F09FBC00BF2ADC41005720024947
:10850000002200F097BC00BF3BDC4100592002492B
:10851000002200F08FBC00BF88DB41005A200249D6
:10852000002200F087BC00BF2CDD41006220024920
:10853000002200F07FBC00BFBDDB41006420024987
:10854000002200F077BC00BF96DC410065200249A4
:10855000002200F06FBC00BF99DB41006620024999
:10856000002200F067BC00BF85DC410008B5174B56
:1085700083F30888164A174B9A4202D0043A1946E8
:1085800001E0154A07E015488142FAD252F8040F7B
:1085900041F8040BF7E712498A4203D2002142F85E
:1085A000041BF8E70F4A23F0604323F07F03936036
:1085B0000D4BB3F5004F3EBF936843F000539360FB
:1085C00003F094F9FDF7D0FCFEE700BFF87F002030
:1085D000ACE54100002400209834002098340020AD
:1085E0008472002000ED00E00024000070470000CD
:1085F0002D4A10B5136B03F00303012B2B4B0DD049
:1086000003D3116ACC011AD525E029494969080626
:108610004CBF4FF400414FF4FA4131E0116AC901F7
:108620000BD424491960116A01F07001102902D09D
:10863000202902D025E0204922E0204920E01D49E0
:108640001960116A01F07001102902D0202902D0AE
:1086500003E0194900E019491960116B124801F053
:10866000030102290ABF816AC16A806AC1F30A4410
:10867000196818BFC06A04FB0111C0B2B1FBF0F168
:108680001960126B02F07002702A03BF1A6803218E
:10869000B2FBF1F2044A1FBF116B1A68C1F3021159
:1086A000CA401A6010BD00BF00040E40F42F002025
:1086B00010140E4000093D0000127A00001BB700A4
:1086C000034607B5054A694610680090186801908E
:1086D000082000F04FFB03B05DF804FB7ADD410099
:1086E00010B5064C00212046602203F019FA092338
:1086F00023804FF4C853638010BD00BFB6500020E4
:10870000F7B5244C074623780E461546002B3BD080
:10871000FAF7F0FC0023237003238DF804301E4B7E
:108720001C78182C19D0192C21D0042C2ED1398862
:108730001A4B8AB21A817888120A5881B8888DF843
:108740000540988130888DF80620D88170888DF892
:1087500007101882B088588212E0FAF7B3FB030AB8
:108760008DF805408DF806308DF8070008E00B4BBA
:108770008DF805405D862B0A8DF806308DF8075080
:1087800001A8FFF79DFF01E0184600E0012003B0BB
:10879000F0BD00BF16510020B4500020B65000209C
:1087A00007B501784278104B42EA01229A86817817
:1087B000C27842EA0122DA860179427942EA01224C
:1087C0001A8703238DF804301A238DF805300378B7
:1087D0008DF80630437801A88DF80730FFF770FF59
:1087E00003B05DF804FB00BFB650002007B50323BB
:1087F0008DF8043020238DF805308DF80700002314
:1088000001A88DF80630FFF75BFF03B05DF804FBAD
:1088100007B503238DF8043022238DF805308DF839
:108820000700002301A88DF80630FFF749FF03B0C9
:108830005DF804FB07B503238DF804301F238DF882
:1088400005308DF80700002301A88DF80630FFF7EA
:1088500037FF03B05DF804FB01280DD006D30228D2
:108860000FD1094B588CC0F340007047064B93F86A
:10887000220000F001007047034B588CC0F38000C9
:1088800070470020704700BFB6500020024B588C44
:10889000C0F3C000704700BFB6500020024B588C98
:1088A000C0F38010704700BFB65000207FB503783A
:1088B000022B03D0032B00F0D980FBE1C278817832
:1088C0008DF8043043788DF806108DF8072002EB00
:1088D0000121A3F10A028DF8053089B21E2A00F2A7
:1088E000C380DFE802F010C1C189891DC1348989C4
:1088F0008989898DC1C1C1C1C1A6C1C1C1C1C1C15F
:10890000C1C1C1C1B800A74B9982C90705D50020D4
:10891000FAF7B6FBF3F75AFCA6E0FAF7EBFBA3E095
:10892000A04DAB8B6C8BE98343EA04449E4B9C4285
:10893000C0F09A8003F588339C4280F095802046F1
:10894000023401F07FFB230C6B83AC838CE0954DEC
:10895000CA0769844FEA112405D5E30700F19D8118
:108960000F20FEF79AF90120FFF776FF40B1630769
:108970004FF0170002D4FEF790F901E0FEF799F9E5
:108980000220FFF769FF40B1A6074FF0100002D4A4
:10899000FEF783F901E0FEF78CF9FFF777FF40B1AE
:1089A00021074FF0110002D4FEF783F901E0FEF732
:1089B00074F9FFF773FF002856D004F0400404F068
:1089C000FF06ACB902238DF8083011238DF8093069
:1089D0006B8C02A81A0A8DF80A208DF80B30FFF76D
:1089E0006FFE64206E8403F003FC01F085F83BE029
:1089F0000020FEF752F937E06A4A22F8131033E0FC
:108A0000684B02A89A8CD9858DF80E20DA8C01F576
:108A1000FA618DF80D201A8DADF80A108DF80C2032
:108A20005A8D9B8D8DF808208DF80930FDF7FAFAE4
:108A30001AE05C4BCA07598716D5002001F094FF55
:108A4000052000F0BDFA002001F09EFF57480821E4
:108A5000FEF70FF908E0534B11F0010018BF012099
:108A6000A3F85010FCF78CFD01A821E18DF800302F
:108A700043784F4A2F2B8DF80130137000F211818B
:108A80009A1E2D2A00F20581DFE812F02E00380030
:108A90008200030103010301030103010301030138
:108AA0000301030103014500530003016A000301B0
:108AB0000301030103010301820082008900030115
:108AC000030103019800A900AC00AF00B300B60099
:108AD0000301B800BA00BC000301C500D000DB00F0
:108AE000E600F100F500FA00324B01A81B681B6894
:108AF00098479DF804409DF8053008E02D4B01A8EB
:108B00001B681B6898479DF806409DF8073003EBEB
:108B10000424A4B2C6E0234B598B988B09040C5A49
:108B20000A180232DC83110C64BAA4B259839A8306
:108B3000B8E001F009FF84B201F00EFF08B144F083
:108B400002041320FEF79BF808B144F0040414203B
:108B5000FEF795F8002800F0A58044F00804A1E095
:108B600002A8FDF783F90F4B9DF80D209DF80E40EC
:108B7000DA849DF80C201A859DF808205A859DF806
:108B800009209A85BDF80A20A2F5FA62DA8589E003
:108B9000094B012200201A70FAF772FA8AE0F8F7FE
:108BA0006FFD87E0B650002000FC410000100E4031
:108BB000B45000202C72002016510020FCF71DFA42
:108BC00000286ED0FCF764FAFCF766FB1E2003F069
:108BD0000FFBFCF7D5FB84B2FCF78EFA62E0F8F7E6
:108BE0006FFD67E0F8F71EFD64E002A8FDF73EF9AF
:108BF00044E0F8F755FD5DE02F4839E006203BE002
:108C0000072039E02D4B0124A3F84E402C4B1B6864
:108C10005B6D984746E02A4B03201B68D3F89C30D5
:108C20009847264B84B2A3F852403BE0244B0220E5
:108C30001B68D3F89C309847204B84B2A3F854406B
:108C400030E01F4B01201B68D3F89C3098471B4B2A
:108C500084B2A3F8564025E0194B00201B68D3F8D6
:108C60009C309847154B84B2A3F858401AE0154839
:108C700000F0C6FA02E0052000F09EFA84B211E08E
:108C800000F08AFC68B10E4B01241B685B6D9847AD
:108C900008E00A4A32F8134004E00F20FEF709F812
:108CA00061E600246846230A8DF802308DF80340FF
:108CB000FFF706FD04B070BD65DD4100B650002031
:108CC0002C7200206FDD4100024B93F84E0000F043
:108CD00001007047B6500020024B187D00F00100E3
:108CE000704700BFB650002000F006BF024B0020C6
:108CF000187000F065B900BF1D51002038B50C4D4B
:108D000002462B781C18102C0DDC0A48E4B21844DB
:108D100002F090FE082C2C7009D1BDE838400420E8
:108D2000002100F0B5B8BDE83840FFF7DFBF38BD1F
:108D30001D5100201F51002008B50A4B1B78082B3D
:108D40000CD109480949042202F042FE30B9FFF76C
:108D5000CDFFBDE808400648FFF7A8BDBDE80840C4
:108D6000FFF7C4BF1D5100201F5100207ADD4100D4
:108D70002351002010B5074C034624781CB9BDE8E8
:108D80001040FCF7BDBF0846BDE810401946F9F792
:108D900075BE00BF1E51002010B586B00DF1030056
:108DA0000121F9F7ADFD002838D01D4C2378012BA7
:108DB00009D002D3022B11D02DE09DF80330552BA2
:108DC000ECD1012328E09DF80330AA2B4FF00003DB
:108DD00022D102222270134A1370DFE711499DF855
:108DE00003000A780AB95528EBD0531CDBB20B708C
:108DF0000D49032B8854D1D90C4B012218680190DE
:108E0000019B086802930390094B08200DEB0001B9
:108E10001A70FFF773FF00232370BFE706B010BD81
:108E20001751002018510020195100207EDD41000B
:108E30001E510020FCF758BFF8B5134B1A881F4687
:108E4000E2B10026012400F089FD3B8814EA030505
:108E50000BD00D4A23EA0403138000F081FD0B4B75
:108E60001B689B5903B19847012500F079FD640008
:108E70003C2EA4B202D00436002DE4D0FCF708FF4B
:108E8000FCF708FFD9E700BF30510020F82F002081
:108E900010B5044651B900F061FD054A138844EA53
:108EA0000300BDE81040108000F05ABD10BD00BFA7
:108EB00030510020024B1888003018BF0120704745
:108EC000305100207047000000230548002220F8A0
:108ED00013200133162BF8D1024B1A7000F08EBD0F
:108EE0003251002060510020F8B51B4D1B4E2C78EC
:108EF00054B333889BB233B3002400F02FFD184ADB
:108F000032F814300BB9002709E0013B9BB222F87C
:108F10001430002BF7D12B780127013B2B7000F088
:108F20001FFD27B10F4B53F8243003B1984701348C
:108F3000162CE2D100F012FD3388013B9BB2338046
:108F400000F00EFDD5E7F8BD00F008FD3480BDE867
:108F5000F84000F005BD00BF605100205E510020C8
:108F600032510020A4DD4100152838B504460D46D5
:108F700017D800F0F3FC0E4B33F814201AB90D4942
:108F80000A7801320A701DB9012223F8142004E086
:108F9000094A1288A91823F81410BDE8384000F0D7
:108FA000DFBCDE2005490022BDE83840FFF742BFA4
:108FB00032510020605100205E51002082DD4100CE
:108FC000152810B5044610D800F0C8FC0A4A32F83B
:108FD000143033B109490B78013B0B70002322F8A0
:108FE0001430BDE8104000F0BBBCFF200449002253
:108FF000BDE81040FFF71EBF325100206051002035
:109000008CDD4100152808B503D8064B13F8100075
:1090100008BD40F2151004490022FFF70BFF0020A5
:1090200008BD00BF3251002095DD41002DE9F84315
:10903000804608460D4616461C4602F0FBFE5FFAC7
:1090400080F9414628464A4602F022FFE0B9C5B2FF
:1090500008EB09077B5D0D2B10D12246304600211D
:1090600002F05EFD621ED2B2AA423046394628BFE7
:109070002A4602F057FF0120BDE8F8830A2BECD006
:109080000130002BE3D1E8E70020BDE8F8830000C1
:109090002DE9F04F414C87B00193236881468A4601
:1090A000DB693F483F4915469847A04610B1002468
:1090B00027466DE004460746D8F800303A4E1B6A52
:1090C0003748314698473346002861D1727A002AE2
:1090D0005ED0002F5CD1327AD206EDD403F10900C4
:1090E0002E2102F053FF83460028E5D002F0A2FEB5
:1090F000C3B2042B0246DFD12C4B0BF1FF31D3F866
:1091000000C00BF1030E11F8013F0CEB0300407897
:1091100000F00300022808BF203B71450B70F2D11C
:1091200058462349D2B202F0B3FE83460028C3D189
:10913000D9F800309C4228D11E490C22504602F03A
:10914000F1FEB388F28803F01F01A970C3F3431145
:109150005B0A143B2B7002F01F035B006B71C2F3C0
:109160004513D20A2B716970EA7059460D2202A884
:1091700002F0D6FC0F490D2202A802F0D3FE02A88D
:109180000199F9F725FB012796E70134A4B293E78B
:109190003846C9F8004007B0BDE8F08F2C720020B7
:1091A00064510020E7D74100805100204430002066
:1091B000BDDE41008951002010B51B28ADF50A7DA8
:1091C00001D9002415E0182343430C4A6846D418FB
:1091D000D158012200F022FB0028F2D1611D227932
:1091E000684600F057FBB0FA80F46846640900F066
:1091F00033FB20460DF50A7D10BD00BFD0DF4100D6
:1092000038B5084D2B689B6B9847B0FA80F4064B35
:1092100064091B78012B03D12B68D3F89030984751
:10922000204638BD2C7200208A4A002018232DE9E0
:10923000F04343431B4DADF5117DEF5806463946CB
:1092400006A8002205EB030800F0E8FA044608B17E
:10925000002422E098F8049006A802A94A4601AB2F
:1092600000F00AFB60B9019A4A4508D102A808F14A
:10927000050102F0ADFBB0FA80F4640900E0044699
:1092800006A800F0E9FA002CE2D0182000FB0650F6
:10929000437D13B13846FFF7B3FF20460DF5117D2E
:1092A000BDE8F083D0DF41001B2801D8FFF7BEBF27
:1092B0000020704770B5ADF50C7D05460E4602A83E
:1092C0000C49002200F0AAFA044670B902A83146FF
:1092D0002A4601AB00F0D0FA18B9019B5B1B5C4237
:1092E0005C4102A800F0B8FA00E0002420460DF529
:1092F0000C7D70BDB3D7410030B50446ADF50B7D94
:1093000010480D46FFF77CFF68460E49012200F029
:1093100085FA90B929462246684600F0BBFAB0FAB1
:1093200080F4684600F098FA074B02211B680A4651
:109330001B6C04486409984700E0002420460DF5A2
:109340000B7D30BDB3D741002C72002010B5ADF5B8
:109350000A7D01460022684600F060FA044668462D
:1093600000F07AFAB4FA84F040090DF50A7D10BDD8
:1093700007B50A4B01A91B686A46DB6A084898478B
:1093800010F0FF0F09BF009B00209878019B04BFDD
:109390005843400803B05DF804FB00BF2C72002066
:1093A000E7D741002DE9F043224E87B0336880466D
:1093B000DB6921482149984708B1002436E04FF67F
:1093C000FF7504462F4633681B481B6A6946984759
:1093D00060BB9DF809304BB3029B194A23F0FF0391
:1093E0009342F0D19DF80830DB06ECD45CB94046DE
:1093F0000DF109010D2202F095FD0124BDF8045084
:10940000BDF80670DFE7BDF80490A94504D3DAD1B2
:10941000BDF80630BB42D6D240460DF109010D22FF
:1094200002F080FD4D46BDF80670CCE7204607B03F
:10943000BDE8F0832C72002064510020E7D7410082
:10944000004C4F4770B540F2FF34002686F001060D
:109450003146002000F0F8FC0A4BC4F57F751B680C
:109460000F2C05F1030598BF2146D3F8943088BF2F
:1094700010212846103C984700F03CFA631CE5D1C7
:1094800070BD00BF2C72002000B589B008A84FF055
:10949000FF3340F81C3D05A903AA02ABFFF7F8FD16
:1094A000BDF8040009B05DF804FB13B502AC44F844
:1094B000040D2046FFF7ECFD02B010BD034610B5C9
:1094C000ADF50A7D0C4668461946002200F0A6F963
:1094D00018B9039B2360012400E00024684600F0D3
:1094E000BBF920460DF50A7D10BD0000F0B507461A
:1094F000ADF50D7D0E46144602A8394600221D46E4
:1095000000F08CF988B90B4B02A81B6831465B69E7
:10951000984710F0FF0F05D102A82946224601AB5B
:1095200000F0AAF902A800F097F901200DF50D7DD1
:10953000F0BD00BF2C720020034630B5ADF50B7DA9
:109540000C46154668461946012200F067F980B9B5
:10955000094B68461B6803995B69984710F0FF0F39
:1095600004D168462946224600F094F9684600F086
:1095700073F90DF50B7D30BD2C72002038B5054612
:1095800008460C4602F056FC224601462846BDE835
:109590003840FFF7D1BF000008B5064B00201B681C
:1095A0000146DB6C4FF400729847B0FA80F0400936
:1095B00008BD00BF2C72002008B5054B1B689B6DD1
:1095C0009847022803D0BDE8084000F0C7B908BD9D
:1095D0002C72002008B5054B1B689B6D984702282C
:1095E00003D0BDE8084000F0BBB908BD2C720020D4
:1095F000F0B5164CADF50B7D23680646DB691448C3
:109600001449984718B123681248DB6B9847002526
:1096100011492A46304601F0D5FA23683146012225
:10962000DB68684698470746FFF7C6FF2368684629
:109630009B699847FFF7CEFF17F0FF0F02D1013566
:10964000FF2DE5D10DF50B7DF0BD00BF2C72002084
:109650006451002075DE41007CDE410010B50446F7
:10966000ADF50A7DFFF7A8FF094B21461B680B22C9
:10967000DB68684698470446FFF7ACFF684600F091
:10968000EBF8E0B2B0FA80F040090DF50A7D10BDAC
:109690002C72002030B52448ADF52D7DFFF756FE25
:1096A00010B3214801A9FFF709FFE8B1019C792C0B
:1096B0001AD122A81C49002200F0B0F8A0B922A8B3
:1096C00003A9019A02AB00F0D7F840B9224603A8DB
:1096D000164902F07DF9041C18BF012400E00124A2
:1096E00022A800F0B9F8E4B1114CFFF765FF236838
:1096F0000D49DB680B2222A898470546FFF76AFF51
:1097000015F0FF0F0DD10949792222A800F0C2F807
:1097100022A800F0A1F8236801211B6C02480A4628
:1097200098470DF52D7D30BD8FDE4100FCDD4100F9
:109730002C720020F8B5002407462546E6B206F153
:109740000C00C0B2FFF7B0FD08B13E700125013436
:10975000102CF3D12846F8BD2DE9F041ADF51C7D64
:1097600080460F46164612A81D4900221D4600F0ED
:1097700055F878BB02AC12A821463F2201AB00F09D
:109780007BF808B1002421E0019B1649E0544246D1
:1097900020463B46FFF74AFC0128F3D1234614F844
:1097A000012B0D2A03D00A2A01D0002AF6D118462F
:1097B00013F8012B0D2AFAD00A2AF8D02B460A49B1
:1097C0003246FFF733FC431E5C425C4112A800F0B6
:1097D00043F800E0002420460DF51C7DBDE8F08133
:1097E0009ADE4100A7DE4100ADDE410010B5ADF5C7
:1097F0000A7D044608496846012200F00FF838B98E
:1098000068462146032200F045F8684600F024F837
:109810000DF50A7D10BD00BFB6DE410070B50646ED
:109820000D460C4C2AB923680122DB689847C4B264
:109830000AE0FFF7C1FE23683046DB6829461322A1
:109840009847C4B2FFF7C6FE002C14BFFF200020CB
:1098500070BD00BF2C72002010B50446FFF7ACFEAF
:10986000044B20461B689B699847BDE81040FFF7F2
:10987000B1BE00BF2C72002010B5054C24682469CD
:10988000A047C0B2002814BFFF20002010BD00BFB9
:109890002C72002013B5064B1B689C6A01ABA047D5
:1098A000C0B2002814BFFF20002002B010BD00BFCE
:1098B0002C72002007B50E4B0DF107011B680DF14E
:1098C00006005B6898471320FDF7D9F901280BD0F3
:1098D0002320FDF7D4F9012807D09DF80630002B8E
:1098E00014BF0220032000E0002003B05DF804FB59
:1098F0002C7200200148FBF747B800BF50140E40FF
:1099000010B512484FF40041FBF71EF84FF6FF73F5
:109910009842044605D140F20F200D490022FFF77E
:1099200089FAA2B213464FF030210A48FBF720F81B
:10993000094B10220021C3F88020C3F8802183F84E
:109940000413BDE810401A60FFF7D4BFC0E1E40083
:1099500070E2410050140E4000E100E072B6704722
:1099600062B6704770B506460D460024012001F02E
:1099700075F801281AD0CCB92B68BBB1013B2B601C
:109980000A2002F035FC00F09BFF0446FFF7B2FF0F
:10999000ECE784B92B6873B1013B2B600A2002F01D
:1099A00027FC00F08DFF0446FFF7A4FF012001F023
:1099B00055F80028EDD1347070BD000008B50C4892
:1099C0000021FAF7BAFFC30610D50A4A4FF4007017
:1099D0001388002101339BB21380FFF759FA064B1D
:1099E0001B781BB1BDE8084000F0ACBA08BD00BF51
:1099F000000001405E5100209851002010B5124C2B
:109A00001720FDF779FA2046002144F20302FAF705
:109A100063FF2046002140F6C412FAF780FF0B4B8B
:109A20004FF400022021C3F88021204683F8171349
:109A30001A6000211022FAF779FF2046BDE8104095
:109A40000021FAF757BF00BF0000014000E100E02D
:109A5000014B1870704700BF9851002008B50248AC
:109A6000F7F748FCFEE700BF00140E4008B5084BAE
:109A70005A6F22F400725A675A6F42F480725A6722
:109A8000FDF786FABDE808402220FDF753BA00BF73
:109A90000040034008B502224FF080431A601220B4
:109AA000FDF748FA4FF040511C20FDF70EF94FF03A
:109AB00040511D20FDF709F94FF040511E20FDF7E0
:109AC00004F94FF040511F20FDF7FFF84FF04051CF
:109AD0001A20FDF7FAF8BDE808401B204FF040516E
:109AE000FDF7F3B808B5002000F03EFFBDE80840E0
:109AF000002000F049BF000008B50648FAF7DEFE76
:109B00000448FAF7E4FE72B6FFF7ECFFFFF7F2FE47
:109B1000FCE700BF10140E4010B5EFF30882614B54
:109B2000934204D24FF0CD3143F8041BF8E75E4B6B
:109B300001241A685D4B1A60FCF7D8FAFDF786F924
:109B40005B4A5178137803EB01239178D27803EBC9
:109B5000014303EB0263574AC2F88830564B1C702E
:109B6000BFF35F8F62B60B20FDF7C6F90C20FDF73F
:109B7000C3F94FF000610C20FDF7A7F84FF000612A
:109B80000D20FDF7A2F84FF000610E20FDF79DF8C3
:109B90004FF000610B20FDF798F84FF0805109203D
:109BA000FDF793F84FF080510A20FDF78EF84FF043
:109BB00060510F20FDF789F84FF060511720FDF735
:109BC00084F84FF060511020FDF77FF83B491320D7
:109BD000FDF77BF839491420FDF777F8224638481D
:109BE0004FF48011FDF727F84FF000611520FDF7C5
:109BF0006CF834491620FDF768F84FF00061192021
:109C0000FDF763F84FF000611820FDF75EF84FF0A4
:109C100000610320FDF759F84FF000610420FDF7C3
:109C200054F84FF020512020FDF74FF84FF020510D
:109C30002220FDF74AF821492320FDF746F84FF08E
:109C400040511120FDF741F81F492046FDF73DF82E
:109C50004FF040512D20FDF738F84FF060510020B3
:109C6000FDF733F84FF020512120FDF72EF84FF08B
:109C700040511220FDF729F84FF080512E20FDF7BA
:109C800024F84FF040510220FDF71FF8FBF7B2FB1C
:109C9000FFF736FEFFF70EFE032801D1FFF72CFF7A
:109CA00010BD00BFF87300201C0040002C72002083
:109CB0008800400000240020F02F002040000028F1
:109CC000000E0E40010000087000002830BF7047F1
:109CD00070470000054B06481A46834204D21168BB
:109CE0000433B1F1CD3FF6D0801A7047F8730020ED
:109CF000F87F002037B5354B00252846294602ACB1
:109D0000019304F8055D00F09FF80120014600F082
:109D10009BF82946022000F097F8204601A9FFF79A
:109D200021FE9DF803500DB9019B0BB9FFF796FE7C
:109D30002846012100F088F82946012000F084F827
:109D40002946022000F080F8204601A9FFF70AFE0C
:109D50009DF80350002DE9D1019B002BE6D0284649
:109D6000294600F071F80120294600F06DF8022024
:109D7000012100F069F8204601A9FFF7F3FD9DF8E5
:109D80000340002CD2D1019B002BCFD01048FFF70D
:109D900037FA2046012100F057F80120014600F073
:109DA00053F80220012100F04FF8019B5BB1013B09
:109DB0000A20019302F01CFA00F082FD0028B5D1C0
:109DC000FFF798FDF1E703B030BD00BF905F0100E1
:109DD000DDDE410008B50120FBF7D2FB00200121A8
:109DE00000F032F80120002100F02EF800210220BE
:109DF00000F02AF8642002F0FBF90020014600F090
:109E000023F80120014600F01FF80021022000F095
:109E10001BF8642002F0ECF90020014600F014F871
:109E20000120002100F010F80121022000F00CF8C0
:109E3000642002F0DDF9FFF75DFD00F041FD002830
:109E4000CCD0FFF70BFE000030B50446134B85B0B5
:109E50000D4693E80700022C04AB03E9070007D97D
:109E60000F494020002205B0BDE83040FEF7E2BFB8
:109E70002046FEF7F1FC78B9A40004AB1C4454F86A
:109E80000C0C25B905B0BDE83040FCF706BF05B0A5
:109E9000BDE83040FCF70DBF05B030BD88E24100A1
:109EA00094E241007047F8F76FBA0000034B1A784C
:109EB0001AB901221A70F8F75DBA7047995100205B
:109EC00008B5F8F723FA024B00221A7008BD00BF4C
:109ED00099510020F8F7B0B908B50F20FFF770F8D6
:109EE0000020FFF7B5FD00200146FFF7ADFF012080
:109EF0000021FFF7A9FFBDE8084002200021FFF77D
:109F0000A3BFFFF7E9BF044608B500200121FFF712
:109F10009BFFE20703D501200146FFF795FFA3074A
:109F200003D502200121FFF78FFF642002F060F9C2
:109F3000FFF7D2FF642002F05BF9E6E7F8F746B9D5
:109F4000F8F77AB9F8F742BAF8F76CBAF8F77EBAC8
:109F5000F8F78ABAF8F794BAF8F798BA08B54FF450
:109F60008000FAF74DFD054B1860FFF7F7FCBDE8E0
:109F700008404FF480000621FAF732BD9C510020C2
:109F800008B5054B4FF480001978FAF729FDBDE8B4
:109F90000840FFF7E5BC00BF9C51002038B50F4CCE
:109FA000FFF7DCFC04F57E75FFF7D8FF0022294699
:109FB00013462046FAF7E2FD20460949082201230C
:109FC000FAF72CFD0022294613462046FAF78EFDAB
:109FD000FFF7D6FFFFF7C4FC012038BD00F84100B1
:109FE000307200200349044A0B68012013604B685B
:109FF0005360704700F841003072002038B50F4CB4
:10A00000FFF7ACFC04F2FF35FFF7A8FF002229465A
:10A0100013462046FAF7B2FD20460949442201239F
:10A02000FAF7FCFC0022294613462046FAF75EFDAB
:10A03000FFF7A6FFFFF794FC012038BD00FC4100AC
:10A04000FC2F002037B504460B0A8DF804308DF83C
:10A050000510A51CFFF782FCFFF780FF00222946B0
:10A0600013462046FAF78AFD01A920460222012361
:10A07000FAF7D4FC0022294613462046FAF736FDAB
:10A08000FFF77EFFFFF76CFC012003B030BD00003E
:10A0900008B503494422034801F0CCFC012008BD67
:10A0A00000FC4100FC2F002008B5FFF757FF0120FE
:10A0B000FAF7C6FDBDE80840FFF762BF10B5064CD1
:10A0C00048212046FBF7B0FD2146A4F848004A206D
:10A0D000BDE81040FFF710B93872002070B58EB09F
:10A0E0000C240021202206A801F01AFD002122469E
:10A0F0000DEB040001F014FD224B0EAE186833F88E
:10A10000042F02909978204B01209871D871029801
:10A11000ADF804208DF806105522D973A5211A70C8
:10A12000C3F809000222BDF80400D9743C215A701A
:10A13000197500221E219A701A715A711A745A7474
:10A140009A745A75DA75DC701C72A3F80D00997553
:10A1500006AA03F11C05144603CCB44228606960CA
:10A16000224605F10805F6D103AA03CA074CD863B5
:10A17000106800226160A06083F8482083F84920BD
:10A180000EB070BDA2E2410038720020747200204F
:10A1900070B50C4605468CB00021202204A801F0C1
:10A1A000BFFC0C2201A8002101F0BAFC552323704A
:10A1B000022363700023A3702B780CAEE3706B78DE
:10A1C0002371AB786371EB78A3712B79E3716B79B1
:10A1D0002372D5F80630C4F809302B4633F80A2F1D
:10A1E000A4F80D209B78E3736B7B2374EB89A4F8B0
:10A1F00011302B7CE3746B7C2375AB7C6375EB7C3B
:10A20000A3752B7DE375D5F8153004F11C05A3610A
:10A2100004AB1A4603CAB24228606960134605F1CE
:10A220000805F6D101AB03CBE063186821646064D4
:10A2300048212046FBF7F8FCA4F848000CB070BD9C
:10A24000F0B59A4BAFB01B78102B0CD0984B102266
:10A250001A7000225A709A70DA701A715A719A71D3
:10A26000DA71FFF79BFE1BAF4A203946FFF722F851
:10A2700068B138464821FBF7D7FCBDF8B4308342BB
:10A280000AD139464A228B4801F0D4FB6BE11C20ED
:10A2900004A9FFF70FF810B9FFF720FF63E104A846
:10A2A0001A21FBF7C1FCBDF82A308342F4D104A87F
:10A2B0003946FFF76DFF7F4839464A2201F0BAFB65
:10A2C00001257C4C2378552B03D0FFF707FF012392
:10A2D00000E000236278022A02D1764A927812B115
:10A2E000FFF7FCFE0123207A724A48B9D17939B9C7
:10A2F000917929B9D17819B9117909B95279DAB1B5
:10A30000E1786C4A17290FD811793B290CD851797B
:10A310003B2909D8917901391E2905D8D279013A0A
:10A320000B2A01D8632807D90023E37023716371D6
:10A33000A371E37123720123227C012A82BF5D4B4A
:10A3400000221A74627D88BF0123012A04D9594B67
:10A3500000225A75012502E0002B18BF0125E27882
:10A36000544B4AB91A793AB95A792AB99A791AB929
:10A37000DA790AB91B7A3BB10023E3702371637168
:10A38000A371E371237201254B4E4C4831460422E0
:10A3900001F01EFB40B13378012563727378A3721C
:10A3A000B378E372F3782373627B424B2AB99A7BCA
:10A3B000092A02D1DB7B192B06D000236373092302
:10A3C000A3731923E37301250DF10300FFF7B2F91D
:10A3D00038B1FFF75DFE9DF80320394B5A75FFF742
:10A3E0000DFE0BA8202101AA0C23FFF7B5F908B335
:10A3F000FFF74EFEDFF8D0E00BAB0DF14C0C1A4628
:10A4000003CA6245CEF80000CEF8041013460EF1E0
:10A41000080EF4D1DFF8A8E001AB03CBCEF836008C
:10A420001868CEF83A10CEF83E00FFF7E7FD254851
:10A43000FEF7E6FE737DFF2B06D1FFF729FE204BCA
:10A4400000225A75FFF7DAFD0023F218917D1F2BC9
:10A45000B1FA81F14FEA511103D001330029F4D050
:10A4600016E0A9B9202213A801F05AFBFFF710FE4D
:10A47000DFF854E013AB1A4603CABA42CEF8000024
:10A48000CEF8041013460EF1080EF4D1FFF7B6FD16
:10A490000023F21892F836100B2BB1FA81F14FEA33
:10A4A000511113D001330029F3D022E000F841000C
:10A4B000307200203872002000FC41004172002000
:10A4C000FC2F00209ADE41001230002089B9284E6E
:10A4D0000C2213A801F024FBFFF7DAFD13AB03CB2A
:10A4E000C6F836001868C6F83A10C6F83E00FFF7FE
:10A4F00085FD2048204901F061FB50B11D4B1E4AEB
:10A5000003F1200153F8040B8B4242F8040BF9D1FC
:10A5100001251A4F1A4E3846314601F04FFB30B133
:10A520003B68012533607B687360BB68B360154B83
:10A530000DF102001B6813A95B6898479DF8023073
:10A540006BB19DF84C3023B9237C012B07D001223D
:10A5500002E0237C1BB100220B4B1A7400E025B1F2
:10A56000FFF7ACFD01E00025ABE62FB0F0BD00BF6A
:10A57000FC2F002016FC41005472002036FC4100E4
:10A58000747200202C72002038720020FFF796BDF4
:10A59000F8B50446FFF726FD134B9F78D8781E794F
:10A5A00059799D79DA79238840EA0720184463882D
:10A5B00041EA06211944A38842EA05221A440B4BBA
:10A5C00080B289B292B240F30724D870597141F336
:10A5D000072042F307219C7018719971DA71BDE868
:10A5E000F840FFF7DBBC00BF00F8410030720020EC
:10A5F00008B5FFF74DFD034BB3F84200431E584228
:10A60000584108BDFC2F002008B5FFF741FD054B60
:10A61000012283F84220002283F84320BDE808404D
:10A62000FFF7ECBCFC2F002073B504464821FBF774
:10A63000FBFAB4F84830834230D1E27852B923793A
:10A6400053B9637943B9A37933B9E37923B9237A49
:10A6500013B923E0172A21D820793B281ED8617925
:10A660003B291BD8A679731E1E2B17D8E5796B1EC4
:10A670000B2B13D8237A632B10D803F5FA638DF8CC
:10A68000050068468DF800608DF80150ADF8023085
:10A690008DF806208DF80410FBF7C4FC02B070BDE5
:10A6A00010B50446FFF79EFC024B5C70BDE81040FD
:10A6B000FFF774BC3072002038B5184B04461A7886
:10A6C0001D462AB100F048F910B1154B01221A704D
:10A6D000287818B1124B1B7823B116E040F693236B
:10A6E0009C4219D840F60C239C4210D840F68A139D
:10A6F0009C420ED840F62E139C420CD840F6071010
:10A7000084428CBF0420052038BD002038BD0120C4
:10A7100038BD022038BD032038BD00BF934A002059
:10A72000B551002008B5F8F743FB00F0EDF8084BF1
:10A7300001221A7000F008F948B1064B5B7833B17A
:10A74000BDE8084015204EF66021FEF70DBC08BD9F
:10A750004030002000F84100114B10B51B7893B138
:10A76000104BB3F81130B3F57A6F0CD90E4B1C783F
:10A770004CB900F0F1F810B10C4B1C7010BD052065
:10A7800042F6E06107E00A4B002201201A7000F057
:10A79000EBF806200A21BDE81040FEF7E5BB00BF3C
:10A7A000934A00203872002040300020B051002031
:10A7B000B1510020024B012202201A70F8F716BB9B
:10A7C000B451002070B5314C2578F8F77BFB237825
:10A7D0002F4A0133DBB2082B22F8150023701546EF
:10A7E00052D100242B4B20461C7000F0BDF82046AF
:10A7F000234635F81020013008281344F9D140F6DB
:10A800001C44C3F3CF00244B44431880234BC4F3B0
:10A81000CF241A78224E234D82B100221A70FFF7FE
:10A820004BFF05283070A5F8114002D10120FFF739
:10A8300037FF10200021FEF72BFB10E01A4B1B788E
:10A8400023B9B5F81130A34204D808E0B5F81130A7
:10A85000A34204D2FFF730FFA5F8114030703378DF
:10A86000052B07D1104B1B7823B90120FFF718FFE8
:10A87000FBF7EAFA052042F6E061FEF775FBBDE85A
:10A8800070400220F8F7CCBA70BD00BFB151002073
:10A89000A0510020B4510020B251002040300020CF
:10A8A000B051002038720020934A0020034B1B78DF
:10A8B0001BB108200021FEF7EBBA7047B45100200D
:10A8C00000F042B8014B1878704700BFB05100202B
:10A8D000014BB3F8110070473872002008B500F042
:10A8E00033F828B1BDE8084080200021FEF7D0BA37
:10A8F00008BD0020FFF7D4BE0C2803D1082901D1E0
:10A90000FFF7ECBF7047000013B50C4B0C4C0093E5
:10A910000822402320460C21FCF74CFA204608214F
:10A92000FCF7A4F9074B4FF480522021C3F8802193
:10A9300083F80C131A6002B010BD00BFF9A84100E3
:10A9400000100E4000E100E008B52320FCF797F965
:10A95000431E5842584108BD08B52220FCF78FF924
:10A96000431E5842584108BD10B50446FDF796FFF6
:10A9700048B911201CB9BDE81040FCF79AB9BDE8F0
:10A980001040FCF78AB910BD10B50446FDF786FFEC
:10A9900040B91CB9BDE81040FCF78BB9BDE81040C8
:10A9A000FCF77BB910BD000008B500F079F8002075
:10A9B00000F054F8014B187008BD00BFB6510020DC
:10A9C000012838B5044626D800F048F8124B195D26
:10A9D000884220D0E51C51B9204601221A55FBF7C8
:10A9E000A1F9E8B29621BDE83840FEF7BDBA0022D1
:10A9F00020460121EDB21A55FBF794F92846FEF7DF
:10AA000001FB40B12846FEF7DBFA2046BDE838409E
:10AA10000221FBF787B938BDB6510020012802D8C2
:10AA20000321FBF77FB97047012804D80130C0B279
:10AA30000521FEF799BA704700F010B800F064B82D
:10AA40000B280AD1B1F5002F01D1002003E0B1F5A8
:10AA5000801F02D10120FFF7E7BF7047034607B50B
:10AA60000D4A012B92E8030002AA02E9030009D86B
:10AA700002EB830353F8080CFCF701F9003018BF10
:10AA8000012005E09B2005490022FEF7D3F90120B3
:10AA900003B05DF804FB00BFACE24100B4E241004A
:10AAA00013B5164C0B214FF4002240230094144898
:10AAB000FCF780F9134B4FF400622021C3F880218A
:10AAC000012083F80B131A60FFF7C8FF012801D19A
:10AAD000FFF7AAFF00940B214FF48012402308488F
:10AAE000FCF768F9074B4FF400622021C3F880217E
:10AAF00083F80B131A6002B010BD00BF41AA4100D9
:10AB0000000E0E4000E100E008B558B10B484FF4CC
:10AB10000021FCF7ABF8BDE8084008484FF480116D
:10AB2000FCF7A4B805484FF40021FCF7A2F8BDE8F3
:10AB3000084002484FF48011FCF79BB8000E0E400D
:10AB400070B5051C0C1C101C002A03D00E22835E5D
:10AB5000013302D0002C14D11CE0828982239B0097
:10AB60001A42F7D00668002909D0311C221C2B7824
:10AB70000B7001310135013A002AF8D1361906600F
:10AB800008E02878013500060016FAF771F8013C54
:10AB9000002CF6D170BC01BC0047000030B581B07C
:10ABA000041C01F047F9051C201C291C0022FFF79A
:10ABB000C7FF0A20FAF75CF8281C01B030BC02BCC1
:10ABC0000847C0460EB400B598B019AB04CB199233
:10ABD0006946822292008A8100900490094A02927A
:10ABE000059201225242CA811793074A1068199AA6
:10ABF00000F00CF8009A0023137018B008BC03B0E2
:10AC000018470000FFFFFF7F70340020F0B55F465B
:10AC100056464D464446F0B4AFB002908A461E1CDC
:10AC2000904600220492089200E0099E4246137862
:10AC3000002B09D0252B07D0444601342378002B64
:10AC400003D0252B01D0F8E744464346E51A002DF2
:10AC500007D04046291C5246FFF772FF049A52194A
:10AC600004920023E356002B00D1FEE20134A046FB
:10AC700000226B46B7331A700392059201235B42A0
:10AC8000069300E01E1C42461278120612169346E6
:10AC90000123984400E005915B46203B582B00D9E6
:10ACA00030E29B00C74A9B589F46C74A08928FE1F3
:10ACB0006A46B7320023D356002BE4D12023137009
:10ACC000E1E70123039A1A430392DCE7331D366858
:10ACD0000596002ED6DA724205921E1C0423039AB2
:10ACE0001A430392CFE72B226B46B7331A70CAE799
:10ACF00042461378012290441B061B162A2B06D0CD
:10AD00009B461A1C303A092A0DD900211AE0331D3E
:10AD100036680696002E04DA1E1C01235B42069359
:10AD2000B1E71E1CAFE700218B005B185B00991890
:10AD30004246127812061216934601239844303A7E
:10AD4000092AF1D900290691A6DA01225242069277
:10AD5000A2E78023039A1A43039294E700215B46FB
:10AD6000303B8A0052185200991843461B781B0644
:10AD70001B169B4601229044303B092B8BD8EEE7F3
:10AD80004023039A1A4303927DE742460023D35699
:10AD90006C2B06D1012398441023039A1A43039283
:10ADA00071E71023039A1A4303926CE71023039A66
:10ADB0001A43039267E75B46432B02D0039AD206FD
:10ADC00010D500230C930D933268029869463F31E9
:10ADD0000CAB01F0EDF8071C431C00D145E2043632
:10ADE000099606E0321D099232686B463F331A70AD
:10ADF000012700226B46B7331A703F236B449946F4
:10AE00002DE21023039A1A430392039BDB0603D51A
:10AE1000321D099234680BE0039B5B0605D5321D99
:10AE2000099233681B041C1402E0331D0993346833
:10AE3000002C01DB0121ECE064422D226B46B7338C
:10AE40001A700121E5E0039AD20605D5331D099356
:10AE50003368049A1A60E8E6039B5B0606D5321D48
:10AE6000099233686A46128A1A80DEE6331D099316
:10AE70003368049A1A60D8E61023039A1A4303929F
:10AE8000039BDB0603D5321D0992346809E0039B5E
:10AE90005B0603D5321D0992348802E0331D099305
:10AEA00034680021B1E0321D099234680223039A0C
:10AEB0001A43039278239B460221434A0892A4E056
:10AEC000069C00226B46B7331A70331D099336680F
:10AED000B146002E00D1BFE15A46532A02D0039B4F
:10AEE000DB0643D54D460E9500230A930B93002CA9
:10AEF00018DB002700250E9B5A59002A1FD0029804
:10AF000069463F310AAB01F053F8421C00D1ACE175
:10AF1000C019A04213DC0435844201D1271C0EE085
:10AF2000071CE8E70AAB0093029800210EAA002351
:10AF300001F068F8071C431C00D196E10E95002F24
:10AF400000D1EEE000250A950B956C4667340AABFC
:10AF500000930298211C0EAA3B1C01F053F8874273
:10AF600000D082E1E555A1460795E0E0002C0CDB1E
:10AF7000301C0021221C00F0E1FC002800D1D3E0AD
:10AF8000871BA74200DDCFE0CBE0301C00F052FF72
:10AF9000071C64E11023039A1A430392039BDB0608
:10AFA00003D5321D0992346809E0039B5B0603D583
:10AFB000321D0992348802E0331D0993346801215F
:10AFC00023E00000CCE2410050E44100AC4A08928A
:10AFD000039BDB0603D5321D0992346809E0039B0D
:10AFE0005B0603D5321D0992348802E0331D0993B4
:10AFF0003468039AD20707D5002C05D00223039AA0
:10B000001A430392022100E0022100226B46B7336B
:10B010001A70069B002B03DB8023039A9A4303924A
:10B02000002C02D1069B002B50D0012909D0012908
:10B030000CD302293AD0069A0792924B99461927C7
:10B0400075E0092C1CD86D46673529E067226A44F3
:10B05000914601235B4299440723234030334A46FB
:10B060001370E408002CF4D1039AD20743D5302B97
:10B0700041D001235B42994430234A4613703AE0A1
:10B080006D466735013D201C0A2100F01DF9303165
:10B090002970201C0A2100F00DF9041C0928F1D8A0
:10B0A000013DA946231C30332B7024E067236B44F9
:10B0B00099460122524291440F232340089A9B5CF7
:10B0C0004A4613702409002C15D0F2E7002903D05A
:10B0D00067236B4499460EE0039AD20703D4672393
:10B0E0006B44994607E030216A463F322723D1540A
:10B0F00066226A4491466B4667334A469F1A069B0E
:10B10000079314E05A46002A00D1AEE069463F3169
:10B110000A7000226B46B7331A70099689460127D8
:10B120009DE00023079302E0069F002207923E1C49
:10B13000079B9F4200DA1E1C6B46B7331B781B0629
:10B140001B16002B01D0013603E0039A920700D5AD
:10B1500002368423039D1D4012D1059B9C1B002CAD
:10B160000EDD102C07DD484810215246FFF7E8FCA1
:10B17000103C102CF7DC4448211C5246FFF7E0FC41
:10B180006846B7300023C356002B04D00121524635
:10B19000FFF7D6FC0CE0039A920709D568463D30CC
:10B1A000302303705B46437002215246FFF7C8FC10
:10B1B000802D16D1059A941B002C12DD102C0ADD6F
:10B1C000314B1D1C1035281C10215246FFF7B8FCCE
:10B1D000103C102CF7DC2C481030211C5246FFF795
:10B1E000AFFC079BDC1B002C12DD102C0ADD264B6C
:10B1F0001D1C1035281C10215246FFF7A1FC103CE5
:10B20000102CF7DC20481030211C5246FFF798FC28
:10B210004846391C5246FFF793FC039A520712D551
:10B22000059B9C1B002C0EDD102C07DD1648102101
:10B230005246FFF785FC103C102CF7DC1248211C0D
:10B240005246FFF77DFC331C059A964200DA131C28
:10B25000049AD2180492E8E40C4B994606273E1E45
:10B2600000DA0026002207926FE704982FB03CBC5A
:10B2700090469946A246AB46F0BC02BC0847000087
:10B2800064E4410078E4410030E4410094E441008A
:10B2900030B581B0041C0D1C131C054A1068211C1C
:10B2A0002A1CFFF7B3FC01B030BC02BC0847000009
:10B2B00070340020002902D0B0FBF1F0704708B1D3
:10B2C0004FF0FF3000F008B80029F8D00246B0FB7C
:10B2D000F1F000FB11217047704700BFD0400B1CFC
:10B2E0001141203A03D49C4613411843634652420D
:10B2F00093401843704700BF7BB972B90029BEBFA5
:10B3000000204FF0004106E008BF00281CBF6FF08E
:10B3100000414FF0FF30FFF7DFBF82B0EC462DE970
:10B32000005000F005F8DDF804E002B00CBC7047F6
:10B330002DE9F041069C904606460F461D4600F05A
:10B3400027F808FB01FCA8FB002300FB05C5B21A87
:10B350002B4467EB03038646C4E90023BDE8F08174
:10B360002DE9F843089E1746804689461D4600F0A1
:10B3700065F900FB05F3A0FB074507FB0137B8EBB8
:10B3800004043D4469EB0505C6E90045BDE8F883C2
:10B3900000292DE9F043C0F2A8800026002BC0F25E
:10B3A0009E8081468E4690469C46174604460D4632
:10B3B000002B3DD18A4259D9B2FA82F33BB1C3F195
:10B3C00020029D4020FA02F29F4015439C40390C18
:10B3D000B5FBF1F01FFA87FE01FB10550EFB00F3E1
:10B3E000220C42EA0545AB4209D9ED1900F1FF32C2
:10B3F00080F00B81AB4240F2088102383D44ED1AE7
:10B40000B5FBF1F301FB13550EFB03FEA4B244EAB6
:10B410000545AE4508D9ED1903F1FF3280F0F780FC
:10B42000AE4540F2F480023B43EA0043002203E0D1
:10B430008B420FD900221346341C18BF01246042EE
:10B440004FF0000565EB4501584051400019694136
:10B45000BDE8F083B3FA83F2002A40F089808B4282
:10B4600002D3804500F2E2800123E5E712B901230F
:10B47000B3FBF2F7B7FA87F8B8F1000F3BD1ED1B39
:10B480004FEA174C1FFA87FE0122B5FBFCF00CFBBC
:10B4900010550EFB00F3210C41EA0545AB4207D9DC
:10B4A000ED1900F1FF3102D2AB4200F2C380084631
:10B4B000ED1AB5FBFCF30CFB13550EFB03FEA4B217
:10B4C00044EA0545AE4507D9ED1903F1FF3102D233
:10B4D000AE4500F2AD800B4643EA0043ACE7524272
:10B4E0006FEA060663EB43035BE7404261EB410111
:10B4F0004FF0FF3652E707FA08F7C8F1200225FAA5
:10B5000002F34FEA174CB3FBFCF11FFA87FE0CFB6A
:10B51000113324FA02F205FA08F50EFB01F92A4369
:10B52000100C40EA0343994504FA08F407D9DB19E3
:10B5300001F1FF3078D2994576D902393B44C9EB05
:10B540000303B3FBFCF00CFB10330EFB00F592B2CF
:10B5500042EA03439D4207D9DB1900F1FF325FD273
:10B560009D425DD902383B445D1B40EA01428CE7B5
:10B57000C2F1200328FA03F10CFA02FC41EA0C0C98
:10B580004FEA1C402EFA03F1B1FBF0F51FFA8CF7DD
:10B5900000FB151129FA03F30EFA02FE07FB05F969
:10B5A00043EA0E0E4FEA1E4343EA0141894508FA79
:10B5B00002F808D911EB0C0105F1FF3332D28945AD
:10B5C00030D9023D6144C9EB0101B1FBF0F300FB4E
:10B5D000131107FB03F71FFA8EFE4EEA014E774563
:10B5E00008D91EEB0C0E03F1FF3117D2774515D9A0
:10B5F000023BE64443EA0543A3FB0889C7EB0E0E72
:10B60000CE4509D305D0002216E71046F7E61346CB
:10B610000AE794404445F6D2013BF4E70B46E9E7DC
:10B620001046A1E71D46CEE7014688E7134603E72B
:10B63000023B51E702383D443AE700BF2DE9F043B1
:10B64000002B44D18A42154604464FD9B2FA82F7FC
:10B650000E464FB1C7F12003B94020FA03F602FAB3
:10B6600007F50E4300FA07F42F0CB6FBF7F01FFAAC
:10B6700085FE07FB10620EFB00F1260C46EA024332
:10B68000994209D95B1900F1FF3280F0EE809942AE
:10B6900040F2EB8002382B44591AB1FBF7F307FB59
:10B6A00013110EFB03FEA4B244EA01418E4508D9F2
:10B6B000491903F1FF3280F0DA808E4540F2D780DD
:10B6C000023B43EA004000263146BDE8F0838B424E
:10B6D00047D8B3FA83F6002E48D18B4202D3824278
:10B6E00000F2CF8001203146BDE8F08312B9012578
:10B6F000B5FBF2F5B5FA85FCBCF1000F78D1491B1A
:10B700002F0C1FFA85FE0126B1FBF7F007FB101185
:10B710000EFB00F2230C43EA01418A4207D9491982
:10B7200000F1FF3302D28A4200F2BC801846891A27
:10B73000B1FBF7F307FB13110EFB03FEA4B244EABF
:10B740000142964508D9521903F1FF3180F09180EA
:10B75000964540F28E80023B43EA00403146BDE808
:10B76000F083002630463146BDE8F083C6F1200460
:10B7700022FA04F5B3402B4321FA04F74FEA1348A9
:10B78000B7FBF8FC1FFA83F908FB1C7720FA04FECC
:10B7900001FA06F509FB0CF44EEA05054FEA154ED1
:10B7A0004EEA0747BC4202FA06F204D9FF180CF130
:10B7B000FF3168D38C463F1BB7FBF8F408FB1477C6
:10B7C00009FB04F9ADB245EA0741894504D9C91816
:10B7D00004F1FF355DD32C4644EA0C44A4FB02235C
:10B7E000C9EB0101994249D345D0204600266BE7B9
:10B7F000CCF1200405FA0CF521FA04F32A0CB3FB72
:10B80000F2F61FFA85FE02FB163820FA04F701FA59
:10B810000CF10EFB06F90F433C0C44EA0843994532
:10B8200000FA0CF407D95B1906F1FF3138D29945BB
:10B8300036D9023E2B44C9EB0303B3FBF2F002FB03
:10B8400010330EFB00F1BFB247EA0343994207D918
:10B850005B1900F1FF3721D299421FD902382B44DE
:10B860001746591A40EA06464EE7104614E71346B3
:10B8700027E70B4670E7B0409042B6D2601E002624
:10B8800022E7304620E7BC4294D9ACF1020C1F44B9
:10B8900091E789459FD9023C19449DE73846DFE787
:10B8A0000E46C8E70238294441E700BF10B491FBB7
:10B8B000F2F4002902FB141306DB002B0EDB0460FC
:10B8C00043605DF8044B7047002BC4BF04F1FF34A4
:10B8D0009B18046043605DF8044B704701349B1A69
:10B8E000046043605DF8044B704700BF70B50F4EB5
:10B8F0000F4D761BB61018BF002405D0013455F843
:10B90000043B9847A642F9D10A4E0B4DFCF76EFE58
:10B91000761BB61018BF002406D0013455F8043B3E
:10B920009847A642F9D170BD70BD00BFA4E54100A3
:10B93000A4E54100A4E54100A4E54100830770B4FB
:10B94000C9B240D0541E002A3FD003788B4218BFA2
:10B95000431C05D11CE0ECB10278013C8A4217D0AF
:10B9600013F0030F184603F10103F4D1032C14D88C
:10B9700084B103788B420BD00519431C02E0027896
:10B980008A4205D0AB42184603F10103F7D10020EB
:10B9900070BC7047204670BC7047024641EA0126E1
:10B9A00046EA0646136810467340A3F1013525EABE
:10B9B000030313F0803F02F10402D9D1043C032CAD
:10B9C0001046EFD8D4E71446D0E71046E0E700BFB2
:10B9D000032A70B426D940EA01039B0711D00478EA
:10B9E0000D78AC4222D10244431C05E013F8014B10
:10B9F00011F8015FAC4219D19342F7D1002070BC1D
:10BA000070470C4603461E6825681846AE4221461C
:10BA100003F1040304F1040404D1043A032A184690
:10BA20002146F0D8002ADAD11046E8E7601B70BC46
:10BA3000704700BF844641EA000313F0030349D175
:10BA4000403A23D30B6803604B6843608B68836084
:10BA5000CB68C3600B6903614B6943618B69836188
:10BA6000CB69C3610B6A03624B6A43628B6A836270
:10BA7000CB6AC3620B6B03634B6B43638B6B836358
:10BA8000CB6BC36340304031403ADBD230320BD312
:10BA90000B6803604B6843608B688360CB68C3604E
:10BAA00010301031103AF3D20C3205D351F8043B68
:10BAB00040F8043B043AF9D2043208D0D2071CBF44
:10BAC00011F8013B00F8013B01D30B88038060466D
:10BAD000704700BF082A13D38B07B1D010F00303BF
:10BAE000AED0C3F10403D21ADB071CBF11F8013B2F
:10BAF00000F8013BA4D331F8023B20F8023B9FE75A
:10BB0000043AD9D3013A11F8013B00F8013BF9D2CC
:10BB10000B7803704B7843708B7883706046704766
:10BB200070B4840746D0541E002A41D0CDB20346DB
:10BB300002E0621EE4B3144603F8015B9A07F8D1F1
:10BB4000032C2ED9CDB245EA05250F2C45EA054533
:10BB500019D9264603F11002103E0F2E42F8105C50
:10BB600042F80C5C42F8085C42F8045C02F11002F6
:10BB7000F2D8A4F1100222F00F0204F00F041032E8
:10BB8000032C13440DD91E462246043A032A46F8D4
:10BB9000045BFAD8221F22F003020432134404F09B
:10BBA00003042CB1C9B21C4403F8011BA342FBD10E
:10BBB00070BC704714460346C2E700BF80EA010C20
:10BBC0001CF0030F37D110F0030C20F0030021F01C
:10BBD000030150F8042B08BF51F8043B0ED08CF041
:10BBE000030C6FF07F434FEACC0C23FA0CFC51F8A6
:10BBF000043B42EA0C0243EA0C0300BFA2F1013C01
:10BC00009A4201BF2CEA020C1CF0803F50F8042B32
:10BC100051F8043BF2D04FEA02604FEA12220128A9
:10BC200028BFB0EB036F08BF1B0AF4D003F0FF037B
:10BC3000000EC01A704710F0030F0AD010F8012B45
:10BC400011F8013B012A28BF9A42F4D0A2EB03006D
:10BC500070474DF8045D50F8042B01F0030521F006
:10BC6000030151F8043B022D26D04DD822F07F4528
:10BC7000B5EB132FA2F1013C2CEA020C0DD11CF004
:10BC8000803C08BF51F8043B0AD185EA0205B5EBB8
:10BC9000036F0CD150F8042BE8E74FEA13235BE065
:10BCA0003CF07F4C54D10B784FEA126554E04FEAD8
:10BCB000126503F0FF034FE04FEA0245A2F1013C99
:10BCC0004FEA15452CEA020CB5EB134F18D11CF0C6
:10BCD000803C08BF51F8043B07D185EA0205B5EB6B
:10BCE000034F09D150F8042BE6E75FEA0C4C2FD143
:10BCF0000B884FEA12452FE04FEA03434FEA124503
:10BD00004FEA134328E000BF02F0FF05B5EB136FC5
:10BD1000A2F1013C2CEA020C0DD11CF0803C08BFC2
:10BD200051F8043B0AD185EA0205B5EB032F0AD18D
:10BD300050F8042BE8E74FEA13630DE012F0FF0F11
:10BD400006D051F8043B4FEA122523F07F4303E06D
:10BD50004FF0000020BC704705F0FF0203F0FF0029
:10BD6000012828BF904204BF2D0A1B0AF4D0A2EB81
:10BD7000000020BC704700BF80EA0102844612F038
:10BD8000030F4FD111F0030F32D14DF8044D11F0D4
:10BD9000040F51F8043B0BD0A3F101329A4312F087
:10BDA000803F04BF4CF8043B51F8043B16D100BF60
:10BDB00051F8044BA3F101329A4312F0803FA4F1F1
:10BDC00001320BD14CF8043BA24312F0803F04BF78
:10BDD00051F8043B4CF8044BEAD023460CF8013BE5
:10BDE00013F0FF0F4FEA3323F8D15DF8044B70478F
:10BDF00011F0010F06D011F8012B0CF8012B002ACD
:10BE000008BF704711F0020FBFD031F8022B12F0BB
:10BE1000FF0F16BF2CF8022B8CF8002012F47F4F76
:10BE2000B3D1704711F8012B0CF8012B002AF9D17E
:10BE3000704700BF20F0030110F00300C0F10000C4
:10BE400051F8043B00F1040C4FEACC0C6FF00002F7
:10BE50001CBF22FA0CF213434FF0010C4CEA0C2CDD
:10BE60004CEA0C4CA3EB0C0222EA030212EACC12BD
:10BE700004BF51F8043B0430F4D0C2F1000102EADF
:10BE80000102B2FA82F2C2F11F0200EBD200704747
:10BE9000002A3CD040EA010313F00303F0B425D19B
:10BEA000032A23D904680D68AC421FD1043A30D06C
:10BEB000A4F1013525EA040414F0803F2CD1071DBC
:10BEC0000D1D0DE057F8043B0E68A3F10134B34299
:10BED00024EA03040AD1043A1BD014F0803F1ED197
:10BEE000032A2946384605F10405EBD803780C7877
:10BEF000013AA34208D162B173B110F8013F11F8C1
:10BF0000014F013AA342F6D0181BF0BC704710460F
:10BF100070471046F0BC70471846F0BC70470020D0
:10BF2000F3E700BF40EA01039B0770B42BD1032A5B
:10BF300029D90C460346214654F8046BA6F1013575
:10BF400025EA060515F0803F05D1043A032A43F897
:10BF5000046B2146EFD8A2B10C78013A1C70013174
:10BF600001333CB16AB111F8014B013A03F8014BBE
:10BF7000002CF7D12AB11A44002103F8011B934287
:10BF8000FBD170BC70470346E5E700BF71B138B51F
:10BF900003460C46002501E00546431C1846214691
:10BFA00000F04EF80028F7D1284638BD00F048B818
:10BFB0002DE9F041054686B01E460C46A1B1104B56
:10BFC0001746D3F8008000F037F800960346214664
:10BFD0003A462846C047431C03D100228A233260D8
:10BFE0002B6006B0BDE8F081054B1F6800F024F817
:10BFF000009603462246284603A9B847EBE700BF50
:10C000007434002010B582B0049C8DE818004FF005
:10C01000FF3300F07BF802B010BD00BF21B1FF2A52
:10C0200004D80A7001207047084670478A230360CD
:10C030004FF0FF30704700BF004870477834002051
:10C04000C9B270B4002933D0850710D00378002B13
:10C0500059D0994218BF431C06D127E013F8012B91
:10C06000002A4DD0914221D09A071846F6D141EAD4
:10C070000126036846EA064601E050F8043F83EAD9
:10C080000605A5F10134A3F1013224EA050422EAF0
:10C090000303234313F0803FEFD0037823B932E04A
:10C0A00010F8013F002B2ED09942F9D170BC704797
:10C0B00084070BD00378002BF8D0431C03E00278F0
:10C0C0000133002AF2D099071846F8D10268A2F18C
:10C0D000013323EA020313F0803F08D150F8042F04
:10C0E000A2F1013323EA020313F0803FF6D0037874
:10C0F000002BDBD010F8013F002BFBD170BC704748
:10C10000104670BC7047184670BC70472DE9F04F60
:10C110008DB0DDF85880179DD2F800A0002952D0CC
:10C12000B8F1000F5CD0002B5CD000241E4689467D
:10C13000A3460691079205902B68DAF80040039316
:10C140006B680493284B1F68FFF776FF224603466F
:10C150000095059809A9B847431C2AD000EB0B02AB
:10C1600042451DD8069B93B100280CDD00F1FF3E2F
:10C1700009A9CE4409F1FF3311F8014B03F8014F2F
:10C180007345F9D1814407990B6804330B605AF861
:10C19000043BDBB1424514D2013E12D09346CBE7BB
:10C1A0005C46039B2B60049B6B6020460DB0BDE892
:10C1B000F08F05998A2200230A602B600DB0BDE83C
:10C1C000F08F1446F1E74FF0FF38ACE7069909B15C
:10C1D00007990B600023501E2B600DB0BDE8F08F57
:10C1E0004446E2E71C46E0E774340020000000000B
:10C1F00001B40248844601BC604700BFCD24002042
:10C200005245462E545854005261636B6574207237
:10C21000656620696E20666C617368203A20005262
:10C2200061636B657420726566206C697374203A73
:10C230000A00095374723D2573205261636B657463
:10C2400031503D256420436F65663D25640A0050EA
:10C25000726F6475637420666F756E6420696E20FA
:10C260006C697374203A20004E6F6E650A00437546
:10C270007272656E7420537472756374203A200074
:10C280004261626F6C617420504C4159205075724C
:10C29000652044726976650000000000000000001F
:10C2A000FF004261626F6C617420504C4159204123
:10C2B00065726F50726F20447269766500000000ED
:10C2C0000000FF004261626F6C617420504C415964
:10C2D0002050757265204472697665204C697465DA
:10C2E00000000000F2004261626F6C617420504CEB
:10C2F00041592050757265204472697665202B0083
:10C30000000000000000FF004261626F6C61742059
:10C31000504C41592050757265204165726F000084
:10C320000000000000000000FF024261626F6C61CB
:10C330007420504C4159204165726F204E616461F8
:10C340006C000000000000000000FF01669EA016C7
:10C35000000000009A615FE900000000000000207A
:10C3600000000000669EA01600000000669EA01659
:10C37000A0885D31000000006077A2CE00000000C0
:10C38000EA2BD04500000000A0885D3100000000CD
:10C39000A0885D31000000010002000300040005D8
:10C3A00000060007FF07FF08FF09FE0AFE0BFD0C51
:10C3B000FC0DFC0EFB0FFA10F811F712F613F41433
:10C3C000F215F016EE17EC18E919E71AE41BE01C59
:10C3D000DD1DDA1ED61FD220CD21C922C423BF24E1
:10C3E000B925B426AE27A828A1299A2A932B8B2CED
:10C3F000842D7B2E732F6A30613157324D33433495
:10C4000038352D36223716380939FD39F03AE23BF6
:10C41000D43CC63DB73EA83F98408841774266432A
:10C420005444424530461D470948F548E149CC4A45
:10C43000B64BA04C8A4D734E5B4F43502B5111525B
:10C44000F852DD53C354A7558C566F575258345980
:10C45000165AF85AD85BB95C985D775E565F3360C0
:10C460001161ED61C962A5637F645A6533660C672B
:10C47000E567BD6894696A6A406B166CEA6CBE6DCC
:10C48000926E656F37700871D971AA7279734874AA
:10C490001775E475B2767E774A781579E079AA7ACD
:10C4A000737B3B7C037DCB7D917E587F1D80E2803A
:10C4B000A68169822C83EE83B08470853186F086F4
:10C4C000AF876D882B89E889A48A608B1B8CD58CFB
:10C4D0008F8D488E008FB88F6F902691DC9191924E
:10C4E0004593F993AC945F951196C29673972398F0
:10C4F000D3988199309ADD9A8A9B369CE29C8D9DD7
:10C50000379EE19E8A9F32A0DAA082A128A2CEA205
:10C5100074A318A4BCA460A503A6A5A647A7E8A772
:10C5200089A828A9C8A966AA04ABA2AB3FACDBAC1A
:10C5300077AD12AEACAE46AFE0AF78B010B1A8B1F7
:10C540003FB2D5B26BB300B495B429B5BDB550B602
:10C55000E2B674B705B896B826B9B6B945BAD3BA33
:10C5600061BBEFBB7BBC08BD93BD1FBEA9BE33BF83
:10C57000BDBF46C0CFC057C1DEC165C2EBC271C3EB
:10C58000F7C37BC400C583C507C68AC60CC78EC760
:10C590000FC890C80000000000000000000000006C
:10C5A00000000000000000000000ECFF3333130027
:10C5B0009B551500327717009A99190002BC1B0091
:10C5C00098DD1D00000020000000000000000000B9
:10C5D000000000009A99E9FFCDCCECFF0000F0FFCD
:10C5E0003333F3FF6666F6FF00000000AFE945064F
:10C5F0001E5C7C0C2F069412A7E27D18385D2B1E62
:10C6000073768E234AE69928CD3C412DD6007931A8
:10C6100052CC3635E36571389ED7203BAE823E3D25
:10C62000A02FC53E481BB13F0000004000000000A5
:10C63000FB211900F1433200E1654B00C48764001F
:10C6400098A97D0058CB960002EDAF00900EC9006E
:10C65000FF2FE2004B51FB00717214016C932D010E
:10C6600038B44601D2D45F0136F578015F159201E6
:10C670004B35AB01F554C4015974DD017393F601D8
:10C6800040B20F02BBD02802E2EE4102AF0C5B02C7
:10C690001F2A74022E478D02D863A6021A80BF0299
:10C6A000F09BD80255B7F10245D20A03BEEC230332
:10C6B000BB063D033820560331396F03A25188036E
:10C6C0008869A103DF80BA03A397D303CFADEC033E
:10C6D00061C3050454D81E04A4EC37044D00510472
:10C6E0004C136A049D2583043C379C042548B504FB
:10C6F0005458CE04C567E704747600055E841905B6
:10C700007F913205D39D4B0555A9640503B47D0582
:10C71000D7BD9605D0C6AF05E7CEC8051BD6E10547
:10C7200066DCFA05C5E1130634E62C06AFE94506DA
:10C7300033EC5E06BBED770644EE9006C9EDA90624
:10C7400048ECC206BBE9DB0620E6F40672E10D0701
:10C75000AEDB2607CFD43F07D2CC5807B3C371074F
:10C760006EB98A07FFADA30763A1BC079693D507EF
:10C770009384EE0757740708DE62200824503908B6
:10C78000253C5208DE266B084B10840867F89C088D
:10C7900030DFB508A0C4CE08B5A8E7086A8B000949
:10C7A000BC6C1909A74C3209272B4B0937086409BF
:10C7B000D5E37C09FDBD9509AA96AE09D86DC709D8
:10C7C0008543E009AC17F90949EA110A59BB2A0A5D
:10C7D000D78A430AC0585C0A1025750AC3EF8D0A30
:10C7E000D5B8A60A4380BF0A0946D80A220AF10A28
:10C7F0008CCC090B428D220B404C3B0B8209540B15
:10C8000006C56C0BC77E850BC0369E0BEFECB60BD6
:10C8100050A1CF0BDE53E80B9604010C74B3190C36
:10C820007560320C940B4B0CCEB4630C1E5C7C0C0C
:10C830008201950CF5A4AD0C7346C60CF9E5DE0C2F
:10C840008383F70C0E1F100D94B8280D1350410D63
:10C8500086E5590DEB78720D3D0A8B0D7899A30D85
:10C860009826BC0D9AB1D40D7B3AED0D35C1050E5D
:10C87000C6451E0E2AC8360E5C484F0E5AC6670EB5
:10C880001E42800EA7BB980EEF32B10EF3A7C90E61
:10C89000AF1AE20E208BFA0E41F9120F0F652B0F23
:10C8A00086CE430FA3355C0F619A740FBEFC8C0FCC
:10C8B000B45CA50F40BABD0F5F15D60F0D6EEE0F1D
:10C8C00046C4061007181F104B6937100EB84F10DA
:10C8D0004E046810064E801032959810D0D9B010D2
:10C8E000DA1BC9104E5BE1102798F91063D21111C1
:10C8F000FC092A11F03E42113A715A11D7A0721167
:10C90000C4CD8A11FCF7A2117C1FBB113F44D31187
:10C910004366EB1184850312FDA11B12ACBB3312DD
:10C920008CD24B1299E66312D1F77B122F06941228
:10C93000AF11AC124F1AC4120920DC12DB22F41220
:10C94000C1220C13B61F2413B8193C13C31054137F
:10C95000D2046C13E3F58313F2E39B13FACEB31303
:10C96000F8B6CB13E99BE313C97DFB13945C131456
:10C9700046382B14DD10431453E65A14A5B872142C
:10C98000D1878A14D153A214A31CBA1442E2D11441
:10C99000ACA4E914DC630115CF1F191581D830153B
:10C9A000EE8D481513406015ECEE7715769A8F15CD
:10C9B000AC42A7158CE7BE151189D6153827EE15A0
:10C9C000FDC105165D591D1653ED3416DD7D4C165F
:10C9D000F70A64169D947B16CB1A93167E9DAA16B1
:10C9E000B21CC2166498D9168F10F116318508173B
:10C9F00046F61F17C9633717B8CD4E170F346617A1
:10CA0000CA967D17E6F594175F51AC1731A9C31785
:10CA100059FDDA17D34DF2179C9A0918B0E3201884
:10CA20000C293818AB6A4F188AA86618A7E27D1837
:10CA3000FC189518874BAC18447AC3182FA5DA1840
:10CA400045CCF11882EF0819E30E2019642A371932
:10CA500001424E19B855651984657C1961719319A5
:10CA60004D79AA19447DC119427DD8194479EF192D
:10CA70004571061A44651D1A3B55341A28414B1A54
:10CA80000729621AD40C791A8CEC8F1A2BC8A61AB3
:10CA9000AF9FBD1A1273D41A5342EB1A6C0D021BCE
:10CAA0005CD4181B1E972F1BAE55461B0A105D1B2E
:10CAB0002DC6731B15788A1BBD25A11B23CFB71B61
:10CAC0004274CE1B1815E51BA0B1FB1BD849121CE4
:10CAD000BBDD281C476D3F1C78F8551C4A7F6C1C39
:10CAE000B901831CC47F991C65F9AF1C996EC61CE3
:10CAF0005EDFDC1CAF4BF31C89B3091DE916201D5A
:10CB0000CB75361D2CD04C1D0826631D5C77791D16
:10CB100024C48F1D5D0CA61D0450BC1D158FD21D95
:10CB20008CC9E81D67FFFE1DA130151E385D2B1E48
:10CB30002885411E6DA8571E05C76D1EEBE0831E9C
:10CB40001DF6991E9606B01E5412C61E5319DC1E01
:10CB5000901BF21E0719081FB5111E1F9605341FE2
:10CB6000A8F4491FE6DE5F1F4EC4751FDCA48B1FAF
:10CB70008C80A11F5C57B71F4829CD1F4CF6E21FC0
:10CB800065BEF81F90810E20CA3F24200FF939207E
:10CB90005BAD4F20AC5C6520FE067B204DAC902049
:10CBA000974CA620D8E7BB200D7ED120320FE7207E
:10CBB000449BFC204022122123A42721E8203D2170
:10CBC0008D9852210F0B68216A787D219BE092217C
:10CBD0009E43A82171A1BD210FFAD221764DE821F3
:10CBE000A39BFD2192E412223F282822A8663D2221
:10CBF000CA9F5222A0D3672228027D225E2B922256
:10CC0000404FA722CA6DBC22F886D122C89AE622DC
:10CC100036A9FB223EB21023DFB5252314B43A23F4
:10CC2000DAAC4F232EA064230D8E792373768E23E6
:10CC30005E59A323CA36B823B30ECD2317E1E123EF
:10CC4000F3ADF62343750B240437202432F3342448
:10CC5000CCA94924CC5A5E2431067324F7AB87242F
:10CC60001B4C9C2499E6B0246F7BC5249A0ADA24D5
:10CC70001594EE24DF170325F39517254F0E2C2569
:10CC8000EF804025D1ED5425F15469254CB67D2522
:10CC9000DF119225A767A625A0B7BA25C801CF2521
:10CCA0001B46E3259784F72537BD0B26FAEF1F2691
:10CCB000DB1C3426D9434826EF645C261A80702694
:10CCC00058958426A6A49826FFADAC2662B1C0264E
:10CCD000CBAED42637A6E826A397FC260C831027D4
:10CCE0006E682427C847382715214C2752F45F2740
:10CCF0007DC173279388872790499B277204AF27AC
:10CD000034B9C227D567D6275210EA27A7B2FD2724
:10CD1000D04E1128CCE42428987438282FFE4B28B4
:10CD200090815F28B6FE7228A07586284AE6992869
:10CD3000B150AD28D2B4C028AB12D428376AE72846
:10CD400075BBFA2861060E29F84A2129378934294A
:10CD50001CC14729A3F25A29C91D6E298C42812979
:10CD6000E8609429DB78A729618ABA297895CD29CA
:10CD70001C9AE0294C98F3290390062A3F81192A2E
:10CD8000FD6B2C2A3A503F2AF32D522A2505652A9D
:10CD9000CED5772AEA9F8A2A77639D2A7120B02A06
:10CDA000D6D6C22AA386D52AD52FE82A69D2FA2A4E
:10CDB0005C6E0D2BAC03202B5592322B551A452B54
:10CDC000A89B572B4D166A2B3F8A7C2B7DF78E2B09
:10CDD000035EA12BCEBDB32BDD16C62B2B69D82B42
:10CDE000B6B4EA2B7CF9FC2B79370F2CAA6E212CD8
:10CDF0000E9F332CA0C8452C5EEB572C46076A2C9F
:10CE0000551C7C2C872A8E2CDA31A02C4C32B22C6B
:10CE1000D92BC42C7F1ED62C3A0AE82C09EFF92C0A
:10CE2000E8CC0B2DD5A31D2DCD732F2DCD3C412D41
:10CE3000D2FE522DDAB9642DE26D762DE81A882DD6
:10CE4000E7C0992DDF5FAB2DCBF7BC2DAA88CE2D87
:10CE50007812E02D3495F12DD910032E6685142E0D
:10CE6000D8F2252E2C59372E60B8482E70105A2E25
:10CE70005A616B2E1CAB7C2EB3ED8D2E1B299F2E81
:10CE8000535DB02E588AC12E27B0D22EBECEE32ECF
:10CE900019E6F42E37F6052F14FF162FAF00282FB2
:10CEA00003FB382F0FEE492FD1D95A2F45BE6B2FD8
:10CEB000699B7C2F3A718D2FB63F9E2FDA06AF2FDC
:10CEC000A3C6BF2F0F7FD02F1C30E12FC7D9F12F62
:10CED0000C7C0230EB1613305FAA233067363430F7
:10CEE00000BB443028385530DBAD6530181C763037
:10CEF000DC82863023E29630ED39A730368AB730AF
:10CF0000FBD2C7303B14D830F34DE8301F80F830E7
:10CF1000BFAA0831CFCD18314CE9283135FD383161
:10CF2000860949313E0E5931590B6931D6007931A4
:10CF3000B2EE8831EAD498317CB3A831668AB83130
:10CF4000A559C8313721D83118E1E7314899F7316F
:10CF5000C349073287F2163291932632E02C3632DB
:10CF600070BE4532404855324CCA643293447432E4
:10CF700012B78332C7219332B084A232C9DFB132F3
:10CF80001133C132857ED03224C2DF32EAFDEE3267
:10CF9000D531FE32E35D0D3311821C335E9E2B339F
:10CFA000C6B23A3348BF4933E2C3583390C06733FF
:10CFB00051B5763322A2853301879433EC63A333D2
:10CFC000E038B233DB05C133DCCACF33DE87DE3372
:10CFD000E13CED33E2E9FB33DF8E0A34D52B193423
:10CFE000C3C02734A64D36347BD24434414F53342A
:10CFF000F5C36134953070341F957E3490F18C34D4
:10D00000E7459B342192A9343CD6B7343612C63456
:10D010000C46D434BD71E2344695F034A5B0FE34EC
:10D02000D8C30C35DDCE1A35B1D1283552CC3635C2
:10D03000BFBE4435F4A85235F18A6035B2646E350E
:10D0400036367C357AFF89357DC097353C79A535F4
:10D05000B529B335E7D1C035CE71CE356809DC3599
:10D06000B598E935B11FF7355B9E0436B01412361A
:10D07000AF821F3655E82C36A0453A368E9A473691
:10D080001DE754364C2B623617676F367E9A7C3616
:10D090007DC5893614E896363F02A436FD13B136B5
:10D0A0004C1DBE362A1ECB369516D8368A06E53676
:10D0B00009EEF1360ECDFE3698A30B37A571183761
:10D0C0003337253740F43137CAA83E37CE544B3773
:10D0D0004CF8573741936437AC25713789AF7D37AA
:10D0E000D8308A3796A99637C219A3375981AF37F6
:10D0F0005AE0BB37C236C8379084D437C3C9E0374B
:10D100005706ED374B3AF9379E6505384D8811388B
:10D1100056A21D38B9B3293871BC35387FBC4138A7
:10D12000E0B34D3892A2593894886538E365713878
:10D130007E3A7D38630689388FC994380284A038D6
:10D14000BA35AC38B4DEB738EF7EC3386916CF389D
:10D1500020A5DA38132BE63840A8F138A41CFD3896
:10D160003F8808390EEB133910451F3942962A398A
:10D17000A4DE3539331E4139EE544C39D382573948
:10D18000E0A7623914C46D396CD77839E8E1833986
:10D1900085E38E3942DC99391CCCA43913B3AF39FD
:10D1A0002591BA394F66C5399132D039E8F5DA3967
:10D1B00054B0E539D261F039600AFB39FDA9053A6E
:10D1C000A840103A5FCE1A3A1F53253AE8CE2F3ABC
:10D1D000B9413A3A8EAB443A670C4F3A4264593AF5
:10D1E0001DB3633AF8F86D3ACF35783AA369823ABD
:10D1F00070948C3A36B6963AF3CEA03AA6DEAA3AA6
:10D200004CE5B43AE5E2BE3A6FD7C83AE8C2D23A42
:10D210004EA5DC3AA17EE63ADF4EF03A0516FA3A20
:10D2200014D4033B09890D3BE234173B9ED7203BC6
:10D230003D712A3BBB01343B18893D3B5307473BBB
:10D24000697C503B5AE8593B234B633BC4A46C3B7D
:10D250003CF5753B873C7F3BA67A883B97AF913B7B
:10D2600057DB9A3BE7FDA33B4417AD3B6E27B63B2C
:10D27000622EBF3B1F2CC83BA420D13BF00BDA3BF6
:10D2800001EEE23BD5C6EB3B6C96F43BC45CFD3B48
:10D29000DC19063CB2CD0E3C4578173C9419203C75
:10D2A0009EB1283C6040313CDAC5393C0A42423CE0
:10D2B000EFB44A3C881E533CD47E5B3CD1D5633CE2
:10D2C0007E236C3CD967743CE2A27C3C96D4843CBF
:10D2D000F6FC8C3CFF1B953CB0319D3C093EA53CC7
:10D2E0000741AD3CAA3AB53CF02ABD3CD911C53C3A
:10D2F00062EFCC3C8BC3D43C528EDC3CB74FE43C59
:10D30000B807EC3C53B6F33C895BFB3C57F7023D56
:10D31000BC890A3DB712123D4892193D6C08213D67
:10D320002375283D6CD82F3D4532373DAE823E3DBA
:10D33000A4C9453D28074D3D373B543DD2655B3D73
:10D34000F686623DA39E693DD7AC703D92B1773DB4
:10D35000D2AC7E3D969E853DDE868C3DA865933D94
:10D36000F23A9A3DBD06A13D07C9A73DCF81AE3D2A
:10D370001331B53DD4D6BB3D0F73C23DC505C93D84
:10D38000F38ECF3D990ED63DB584DC3D48F1E23DAC
:10D390004F54E93DCAADEF3DB8FDF53D1844FC3DA5
:10D3A000E980023E2AB4083ED9DD0E3EF7FD143E68
:10D3B00082141B3E7921213EDB24273EA81E2D3EF0
:10D3C000DE0E333E7CF5383E82D23E3EEFA5443E33
:10D3D000C16F4A3EF92F503E94E6553E92935B3E14
:10D3E000F336613EB4D0663ED7606C3E59E7713E7D
:10D3F0003A64773E78D77C3E1441823E0CA1873E4A
:10D400005FF78C3E0D44923E1587973E76C09C3E5A
:10D410002FF0A13E3F16A73EA632AC3E6345B13E7B
:10D42000754EB63EDB4DBB3E9443C03EA02FC53E7D
:10D43000FE11CA3EADEACE3EADB9D33EFC7ED83E2B
:10D440009A3ADD3E87ECE13EC194E63E4733EB3E3F
:10D450001AC8EF3E3853F43EA1D4F83E544CFD3E7A
:10D4600050BA013F951E063F21790A3FF5C90E3F8C
:10D470000F11133F704E173F15821B3FFFAB1F3F2D
:10D480002ECC233F9FE2273F53EF2B3F4AF22F3F03
:10D4900081EB333FFADA373FB3C03B3FAB9C3F3FB2
:10D4A000E36E433F5937473F0DF64A3FFEAA4E3FD2
:10D4B0002C56523F96F7553F3C8F593F1D1D5D3FFF
:10D4C00038A1603F8D1B643F1C8C673FE3F26A3FCD
:10D4D000E34F6E3F1BA3713F8AEC743F302C783FC3
:10D4E0000C627B3F1E8E7E3F65B0813FE2C8843F69
:10D4F00092D7873F77DC8A3F8FD78D3FDAC8903F3E
:10D5000058B0933F078E963FE861993FFB2B9C3FB5
:10D510003EEC9E3FB2A2A13F554FA43F28F2A63F4A
:10D520002A8BA93F5B1AAC3FBB9FAE3F481BB13F64
:10D53000028DB33FEAF4B53FFF52B83F40A7BA3F70
:10D54000ADF1BC3F4632BF3F0A69C13FF995C33FC9
:10D5500013B9C53F58D2C73FC6E1C93F5EE7CB3FCD
:10D5600020E3CD3F0BD5CF3F1EBDD13F5A9BD33FCC
:10D57000BE6FD53F4A3AD73FFEFAD83FD9B1DA3F1E
:10D58000DC5EDC3F0502DE3F559BDF3FCB2AE13FFF
:10D5900067B0E23F2A2CE43F129EE53F1F06E73FBB
:10D5A0005264E83FA9B8E93F2603EB3FC743EC3F8D
:10D5B0008C7AED3F76A7EE3F84CAEF3FB6E3F03FAB
:10D5C0000BF3F13F84F8F23F20F4F33FE0E5F43F42
:10D5D000C3CDF53FC8ABF63FF17FF73F3C4AF83F7C
:10D5E000AA0AF93F3AC1F93FEC6DFA3FC110FB3F7F
:10D5F000B8A9FB3FD138FC3F0CBEFC3F6939FD3F69
:10D60000E7AAFD3F8812FE3F4A70FE3F2DC4FE3F51
:10D61000320EFF3F594EFF3FA184FF3F0BB1FF3F4A
:10D6200096D3FF3F43ECFF3F11FBFF3F000000405C
:10D63000010101010101010101010101010101FFDC
:10D64000FFFFFFFFFFFFFFFFFFFFFFFFFFFF0000E8
:10D6500000002000FFFFFFFFFFFF3030303000559B
:10D66000AA55AA000055AA55AAC04041007EDADC9E
:10D67000EDEDA97AC0C04041007EACAFEFEEBB84B7
:10D68000C0C04041007EDADCEDEDA97AC0C0404167
:10D69000007EACAFEFEEBB84C0C04041007EADEF7A
:10D6A000ACEDA1A6C0C04041007EDEADD0D0835815
:10D6B000C0C0DBDC6500DA0F040001000011DAC035
:10D6C000C04041007EDEADD0D08358C0C0DBDC65F9
:10D6D00000DA0F040001000011DAC0C0480000B7F2
:10D6E0005E8CC0C0C88205B002002C00010003702F
:10D6F000000003022400000002003B0004009B0025
:10D700000600520008004B000A002D0010000F0018
:10D71000140028002000300024000D0028000E0016
:10D7200046000B004C00030062000C0070000D006E
:10D73000800002000001040000020100000000005F
:10D7400032BBC0C0480000B75E8CC0C0C98205AF04
:10D7500001002C00010003700000030224000000FF
:10D7600002003B0004009B000600520008004B0032
:10D770000A002D0010000F001400280020003000C7
:10D7800024000D0028000E0046000B004C00030092
:10D7900062000C0070000D00800002000001040017
:10D7A0000002010000000000A8B7C0C0500000AF98
:10D7B00053D1C0557365725061722E696E66002533
:10D7C00073202573004261626F6C617420504C417C
:10D7D0005900303A5C4C4F47253033642E42494E55
:10D7E0000025735C257300303A000000000004053A
:10D7F00053454E5343414C2E5458540050524F44BD
:10D80000203A0A0009415A203A202568640A000992
:10D810004758203A202568640A00094759203A20D1
:10D820002568640A0009475A203A202568640A00DE
:10D830004150504C49203A0A00414C474F20434147
:10D840004C43200A000200434F554E540020202034
:10D8500020202020202020202020202020202020C8
:10D860002020202020202002014143435800202076
:10D8700020202020202020202020202020202020A8
:10D880002020202020202020200201414343590055
:10D890002020202020202020202020202020202088
:10D8A000202020202020202020202002014143434E
:10D8B0005A0020202020202020202020202020204E
:10D8C000202020202020202020202020200201476E
:10D8D00059525800202020202020202020202020C5
:10D8E0002020202020202020202020202020200256
:10D8F000014759525900202020202020202020209C
:10D900002020202020202020202020202020202017
:10D910002002014759525A00202020202020202098
:10D9200020202020202020202020202020202020F7
:10D9300020202002005049455A4F3100202020204D
:10D9400020202020202020202020202020202020D7
:10D95000202020202002005049455A4F320020202C
:10D9600020202020202020202020202020202020B7
:10D970002020202020202002005049455A4F33000B
:10D980002020202020202020202020202020202097
:10D9900020202020202020202002005049455A4FDE
:10D9A0003400202020202020202020202020202083
:10D9B0002020202020202020202020020050494527
:10D9C0005A4F3500202020202020202020202020F9
:10D9D0002020202020202020202020202002005055
:10D9E00049455A4F3600202020202020202020208A
:10D9F0002020202020202020202020202020200245
:10DA0000005049455A4F3700202020202020202058
:10DA10002020202020202020202020202020202006
:10DA20002002005049455A4F380020202020202055
:10DA300020202020202020202020202020202020E6
:10DA400020202002005642415454206D56002020D0
:10DA500020202020202020202020202020202020C6
:10DA600020202020200100494E464F002020202069
:10DA700020202020202020202020202020202020A6
:10DA800020202020202020AF24324656FE128990EC
:10DA900078BC2980340100AF24324656FE128990AA
:10DAA00078BC29803501012530325825303258257F
:10DAB00030325825303258004150505F4B45525F4C
:10DAC0004C6F77506F7765724D616E6167656D65FC
:10DAD0006E7400303A4657555645522E4B45590004
:10DAE000303A42545F53414D42412E4B455900302C
:10DAF0003A44454C535049464C2E4B455900000082
:10DB0000E1164100B1334100398D4100C5A7410004
:10DB1000915E41002D534100C58E410029364100E0
:10DB2000C58E4100E98E4100691F4100998D410079
:10DB3000C58E4100C58E4100C58E410091594100FE
:10DB400022506C617922004275734661756C745F76
:10DB500048616E646C65725F5765616B0055415238
:10DB600054315F48616E646C65725F5765616B002C
:10DB700055736167654661756C745F48616E646C6E
:10DB800065725F5765616B005443315F48616E6435
:10DB90006C65725F5765616B0043524343555F4844
:10DBA000616E646C65725F5765616B005356435FCD
:10DBB00048616E646C65725F5765616B00444143F8
:10DBC000435F48616E646C65725F5765616B0048C6
:10DBD000534D43495F48616E646C65725F57656180
:10DBE0006B005744545F48616E646C65725F5765A3
:10DBF000616B00545749305F48616E646C65725FB9
